:100000000C9413210C9444210C9444210C9444210D
:100010000C9444210C9444210C9444210C944421CC
:100020000C9444210C9444210C9444210C944421BC
:100030000C9444210D94E33A0C9444210C944421F3
:100040000C9444210C9432D80C9444210C944421F7
:100050000C9444210C9444210C94F9D40D94993AB5
:100060000C9444210C94414A0C94374A0C9444213A
:100070000C9444210C9444210C9444210C9444216C
:100080000C9444210C9444210C9444210C9444215C
:100090000C9444210C9444210C9444210C9444214C
:1000A0000C9444210C9444210C9444210C9444213C
:1000B0000C9444210C9444210C9444210C9444212C
:1000C0000C9444210C9444210C9444210C9444211C
:1000D0000C9444210C9444210C9444210C9444210C
:1000E0000C944421084AD73B3BCE016E84BCBFFD33
:1000F000C12F3D6C74319ABD56833DDA3D00C77FF8
:1001000011BED9E4BB4C3E916BAAAABE0000008090
:100110003F05A84CCDB2D44EB93836A9020C50B91F
:10012000918688083CA6AAAA2ABE000000803F004B
:100130000D942C340D941B340C94EE210C943681C8
:100140000D94BC340C94CF4A0C94C7AF0D94073572
:100150000D9478330C9457810C946CC90D947C33B6
:100160000C94C0AE0C940C780C9456780D949F337C
:100170000C94D0AE0C9490AE0C942F7A0C94CA7F51
:100180000C94BE7F0C94AE7F0C9446210C94847822
:100190000C9486C70C9470A70C94DA770C94E5C77E
:1001A0000D948E340C940B7A0C94B14A0D94AD33AB
:1001B0000C9445770C947DC20C94794A0D9461336C
:1001C0000C945B960D94D0340C946F750D94803321
:1001D0000C94787D0C94F3910C942F880C94A7BB0D
:1001E0000C946D780C941BB20C9400840C94A07940
:1001F0000C94D74A0C949B790C9407850C946580D9
:100200000C94C47A0C94677B0C942B7A0C94F4BAFB
:100210000C94067B0D94C6340C9493770C94637BFA
:100220000D94A2340C94A8AE0C940D850D94E23379
:100230000C94869F0C94D0C60C94DD7B0D942034D6
:100240000D94D9460C947D800C9458A10D943C34A7
:100250000D947A130C947EAE0C94EDC60C94AE778C
:100260000C9410850C9494790C94A8B20D9491334D
:100270000C9416B20C94FC790C94C67F0C940F8BE2
:100280000C94F0840C94CAC70C9496AE0C94A18183
:100290000C94FC800D9432340C9491850C94E87D80
:1002A0000D94FD340C94C7770D94B7330C94A88249
:1002B0000D9466330C9447780C9473850C94F99DD7
:1002C0000D94C7330D9411350D94B3330C94A57967
:1002D0000C94F1930C9401B60C94CB4A0C94567B7D
:1002E0000C94048A0C94AEAE0C9447BB0C94E64A72
:1002F0000C94F8830C94C6BB0C940E7A0D949B332B
:100300000C948A810C9466BB0C9420810C94B27F6F
:100310000C94C6AE0D9468460C9480770C944D9C5A
:100320000C94B1800D94E9340C946D7B0C94967907
:100330000C9484AE0C9475C80C94C74A0C94D27F6C
:100340000C94CE7F0C9401850C9475800C946B7B7F
:100350000D9498340C9488750C942C770C94E78148
:100360000C9430750C94A2AE0C9490970D94F334C9
:100370000C94267A0C94657B0C9449210C945022A1
:100380000C9404850C94FE840C9433B20C9430903D
:100390000D94DA340C940A850C941D850C947685A2
:1003A0000C946A790D94AC340C9423790C94DB4A48
:1003B0000C94D34A0D9484330C9456360C94779A4B
:1003C0000C947F790C945F7B0C94B4AE0C94707D8C
:1003D0000D9497330C94CA800C9457A40C94B67F58
:1003E0000C948E750C9415850C94F94A0C94158117
:1003F0000C9425750C94157B0C94C04A0D94B43460
:100400000C9429980C94F2830C94F1960D94A933D2
:100410000C949CAE0C94A2C80C94747D0C94BA7F7E
:100420000C94E2B20C94C27F0C94BAAE0C94227D70
:100430000C94DF4A0C947EC20C94D1C30C94C52159
:100440000C941A850C9409840D94BB460C94EF9D72
:100450000D9489340C94117A0C94167D0C947B9530
:100460000C9465C70D942B130C9463C80C948E8D5B
:100470000C9411B20C94E3800C94F14A0D948134E5
:100480000C94F3770C94728C0C942E780C94148446
:100490000C948AAE0C9406990C94F3310C94772248
:1004A0000C949C750D94A5330C94697B0C94E279A3
:1004B0000C94C5AB0C946D770C94D5BA0C94FB845A
:1004C0000C940CB20C9451C60C941B780D945813D8
:1004D0000C9473790C944C210D9447340C943FA6E2
:1004E0000C9417850C94FBC10D9487330C949B7866
:1004F0000D948D330C94F0BB0C94AA790C945E7718
:100500000C9492790C9402750C94147A0D941B350A
:100510000C94A24A0C94617B4E414E494E49545969
:10052000494E46CDCCCC3D0AD7233C17B7D13877BE
:10053000CC2B329595E6241FB14F0A0000204100D4
:1005400000C84200401C4620BCBE4CCA1B0E5AAE1E
:10055000C59D7400407A10F35A00A0724E1809002D
:1005600010A5D4E80000E87648170000E40B540218
:100570000000CA9A3B000000E1F505000080969853
:1005800000000040420F000000A0860100000010A3
:100590002700000000E803000000006400000000E5
:1005A000000A00000000000100000000002C76D8C6
:1005B00088DC674F0823DFC1DFAE59E1B1B796E5AC
:1005C000E3E453C63AE651997696E8E6C28426EB10
:1005D000898C9B62ED407C6FFCEFBC9C9F40F2BA23
:1005E000A56FA5F490055A2AF75C936B6CF9676DBB
:1005F000C11BFCE0E40D47FEF520E6B500D0ED9010
:100600002E0300943577050080841E080000204EDC
:100610000A000000C80C333333330F986E12831175
:1006200041EF8D2114893BE65516CFFEE6DB18D14C
:10063000844B381BF77C1D901DA4BBE4242032841E
:10064000725E228100C9F124ECA1E53D27434F4DA4
:100650004D554E49434154494F4E0044525952550D
:100660004E004552524F525300494E464F004543AB
:10067000484F004572726F722077726974696E67B5
:1006800020746F20454550524F4D210A0053544F5E
:10069000505045442E20005072696E74657220736C
:1006A000746F707065642064756520746F20657266
:1006B000726F72732E2046697820746865206572A7
:1006C000726F7220616E6420757365204D393939FF
:1006D00020746F20726573746172742E20285465C3
:1006E0006D706572617475726520697320726573CF
:1006F00065742E2053657420697420616674657278
:100700002072657374617274696E67290A004E6F96
:1007100020436865636B73756D2077697468206C1E
:10072000696E65206E756D6265722C204C61737404
:10073000204C696E653A20004E6F20436865636BFC
:1007400073756D2077697468206C696E65206E75AD
:100750006D6265722C204C617374204C696E653A31
:100760002000636865636B73756D206D69736D61DF
:100770007463682C204C617374204C696E653A2058
:10078000004C696E65204E756D626572206973203C
:100790006E6F74204C617374204C696E65204E75C9
:1007A0006D6265722B312C204C617374204C696E24
:1007B000653A20004D3131300053657269616C201B
:1007C000737461747573206D69736D617463680A05
:1007D00000776169740A0053442072656164206582
:1007E00072726F720A00486F74656E642049646C9F
:1007F000652054696D656F757400486F74656E642B
:100800002049646C652054696D656F75740A002118
:1008100021204B494C4C20636175736564206279DB
:10082000204B494C4C20627574746F6E2F70696E4A
:100830000A002121204B494C4C206361757365648B
:1008400020627920746F6F206D75636820696E6116
:1008500063746976652074696D65202D20637572F7
:1008600072656E7420636F6D6D616E643A20004D29
:10087000656469612052656D6F766564004D6564DD
:10088000696120496E736572746564004D31303062
:10089000305300627573793A207061757365642016
:1008A000666F7220696E7075740A00627573793AAA
:1008B0002070617573656420666F72207573657250
:1008C0000A00627573793A2070726F636573736999
:1008D0006E670A00506C65617365205265736574BC
:1008E000005052494E5445522048414C5445440012
:1008F00025533A20255300706F7765726F66660046
:100900004B494C4C45442E20005072696E74657200
:100910002068616C7465642E206B696C6C282920DA
:1009200063616C6C6564210A006563686F3A004519
:1009300072726F723A000A4D656173757265642058
:10094000706F696E74733A0A00357835206D65737F
:10095000682E205A206F66667365743A20005072C4
:10096000696E74696E67204F626A6563740025530F
:10097000202569002F2F616374696F6E3A007374CC
:1009800061727400656E6400486F74656E642074F3
:100990006F6F20636F6C640A0053656E64204D3185
:1009A000303820746F20726573756D650A00496E6A
:1009B000736572742066696C616D656E7420616E1A
:1009C000642073656E64204D3130380A00526568CA
:1009D00065617420446F6E65005265686561746975
:1009E0006E672E2E2E005265686561740048656141
:1009F0007465722054696D656F75740053656E641B
:100A0000204D31303820746F2068656174206E6F1E
:100A10007A7A6C650A004E6F7A7A6C652050617242
:100A20006B65640070617573656400506175736512
:100A300000726573756D656400526573756D696EDE
:100A400067004732362043616E63656C656400471A
:100A500032362048656174696E67204E6F7A7A6C11
:100A600065004732362048656174696E67204265CB
:100A7000640057616974696E6720666F72206865EB
:100A8000617475702E0A004669786564204C656E45
:100A9000677468205072696D6500446F6E65205000
:100AA00072696D696E67004D616E75616C20707260
:100AB000696D696E672E2E2E004C656176696E67D2
:100AC00020473236003F537065636966696564206C
:100AD000582C5920636F6F7264696E617465206F62
:100AE0007574206F6620626F756E64732E0A003F06
:100AF00028522965706561742076616C7565206E79
:100B00006F7420706C61757369626C653B206D75E4
:100B10007374206265206174206C65617374203188
:100B20002E0A003F537065636966696564206E6FC5
:100B30007A7A6C652074656D706572617475726522
:100B4000206E6F7420706C61757369626C652E0A1B
:100B5000003F5370656369666965642066696C610E
:100B60006D656E742073697A65206E6F7420706C89
:100B700061757369626C652E0A003F537065636925
:100B800066696564207072696D65206C656E677456
:100B900068206E6F7420706C61757369626C652E6D
:100BA0000A003F537065636966696564206E6F7AF9
:100BB0007A6C652073697A65206E6F7420706C6141
:100BC000757369626C652E0A003F526574726163C9
:100BD00074696F6E204D756C7469706C69657220F4
:100BE0006D757374206265207370656369666965ED
:100BF000642E0A003F53706563696669656420521C
:100C0000657472616374696F6E204D756C74697080
:100C10006C696572206E6F7420706C6175736962A7
:100C20006C652E0A003F53706563696669656420D0
:100C30006C6179657220686569676874206E6F748D
:100C400020706C61757369626C652E0A0043292EF1
:100C50000A003F5370656369666965642062656474
:100C60002074656D7065726174757265206E6F7445
:100C700020706C61757369626C65202834302D00BA
:100C8000473236207374617274696E672E2E2E0A95
:100C9000004F46460A0046616465204865696768FA
:100CA000742000426564204C6576656C696E67202F
:100CB000004661696C656420746F20656E61626CCA
:100CC0006520426564204C6576656C696E670A0034
:100CD0004D65736820426564204C6576656C2064C0
:100CE0006174613A0A00496E76616C6964206D65D1
:100CF00073682E0A00206E6F7420656E74657265CD
:100D0000642E0A0050726F62696E6720506F696EC0
:100D1000740025532025692F256900206F66200067
:100D20004D424C2047323920706F696E7420002983
:100D30000A004A206F7574206F662072616E6765C5
:100D40002028302D00290A0049206F7574206F6615
:100D50002072616E67652028302D004732384C3094
:100D6000004D6573682070726F62696E6720646FF2
:100D70006E65004D6573682070726F62696E6720E2
:100D8000646F6E652E0A005374617274206D657312
:100D9000682070726F62696E6720776974682022BC
:100DA000473239205331222066697273742E0A004B
:100DB0004732395332004732384C300A47323953C0
:100DC0003200686173206E6F20646174612E0A00C6
:100DD0004D65736820426564204C6576656C696E6C
:100DE00067200053206F7574206F662072616E67F4
:100DF000652028302D35292E0A004D657368207036
:100E00006F696E74206F7574206F662072616E67F3
:100E1000650A004D34323120696E636F727265630A
:100E20007420706172616D6574657220757361679D
:100E3000650A004F4646004F4E0020204D61783A2B
:100E40002000200020204D696E3A2000536F667408
:100E500020656E6473746F70733A20004D323420D5
:100E600053256C642054256C64004739322E392098
:100E700045257300473120462564004739322E3915
:100E8000205A2573004731205A3020463230300036
:100E90004731205825732059257320463330303090
:100EA000004D34323020532569205A2573004D31CE
:100EB00030362050256920532569004D32303020CE
:100EC0004425730047323852305859004739322E82
:100ED00039204530205A300A47315A2573004D31A8
:100EE000303920532569004D3139302053256900B0
:100EF0004D343230205330205A300020496E766114
:100F00006C6964206578747275646572200047327C
:100F10002F47332062616420706172616D65746572
:100F200072730A00536C6565702E2E2E004D65732A
:100F30006820706F696E74206F7574206F66207200
:100F4000616E67650A004D302053746F70004D313B
:100F50002053746F7000436C69636B20746F205270
:100F60006573756D652E2E2E004E6F204D6F766564
:100F70002E00456E642066696C65206C6973740A86
:100F800000426567696E2066696C65206C697374E0
:100F90000A004E6F206D656469610A0052657375C1
:100FA0006D696E6720534400286E6F2066696C651A
:100FB000290043757272656E742066696C653A200B
:100FC000005072696E742074696D653A20000A538E
:100FD000746174733A2046696C616D656E74207536
:100FE0007365643A20002C204C6F6E676573742023
:100FF0006A6F623A2000546F74616C2074696D6589
:101000003A200053746174733A20002C20466169C1
:101010006C65643A20002C2046696E6973686564CB
:101020003A20005072696E74733A200053746174F0
:10103000733A2000436F6F6C696E672E2E2E004846
:10104000656174696E672E2E2E0045202553006F52
:101050006B006F6666006E06690662065B064D06EB
:1010600044454255473A004D3131332053004265E3
:101070006420436F6F6C696E672E2E2E004265648C
:101080002048656174696E672E2E2E005375506579
:10109000522043522D3230204F46462E002F2F0033
:1010A0004D31343520533C696E6465783E206F7550
:1010B00074206F662072616E67652028302D31299B
:1010C0000A00205200416363656C65726174696F48
:1010D0006E3A2050005741524E494E4721204C6FE6
:1010E00077205A204A65726B206D6179206C6561AA
:1010F0006420746F20756E77616E74656420706112
:10110000757365732E0A004D3230362058004652F2
:101110003A0020466C6F773A20004D424C204164E3
:101120006A757374205A0020643A0020693A0020DE
:10113000703A00496E76616C6964206578747275E6
:101140006465720A0020643A0020693A0020703A0F
:10115000004C434420436F6E74726173743A2000F4
:1011600064697300656E0043290A0061626C6564FE
:1011700020286D696E2074656D702000436F6C646B
:101180002065787472756465732061726520004F04
:10119000666673657473204170706C6965640045A0
:1011A00072723A20546F6F206661722100546F6F23
:1011B000206661722066726F6D2072656665726569
:1011C0006E636520706F696E740A00454550524F1A
:1011D0004D204F4B0A002E0A002028302D31302997
:1011E000002076616C7565206F7574206F662072C3
:1011F000616E676500416476616E6365204B3D00FA
:10120000506F7765722D6C6F7373207265636F76A4
:1012100065727920004D383400446F6E652070721D
:10122000696E74696E672066696C650A004D3737B0
:10123000004D3331004361703A004D4541545041F7
:10124000434B00434F4F4C45525F54454D50455220
:101250004154555245004348414D4245525F544523
:101260004D50455241545552450042414259535404
:10127000455050494E470041524353004D4F544949
:101280004F4E5F4D4F44455300544845524D414CDD
:101290005F50524F54454354494F4E004C4F4E47B8
:1012A0005F46494C454E414D45004155544F5245CE
:1012B000504F52545F53445F53544154555300535D
:1012C000445F5752495445005245504541540053DC
:1012D00044434152440050524F4D50545F53555077
:1012E000504F525400454D455247454E43595F506B
:1012F000415253455200434153455F4C494748547E
:101300005F4252494748544E45535300544F474754
:101310004C455F4C494748545300534F465457413E
:1013200052455F504F574552004255494C445F501B
:10133000455243454E54004C4556454C494E475F37
:1013400044415441005A5F50524F42450052554E5D
:101350004F5554004155544F4C4556454C00505242
:10136000494E545F4A4F420050524F4752455353E3
:10137000004155544F5245504F52545F54454D50C3
:1013800000564F4C554D4554524943004545505227
:101390004F4D0042494E4152595F46494C455F54BA
:1013A00052414E534645520053455249414C5F58B5
:1013B0004F4E5F584F4646004649524D57415245A1
:1013C0005F4E414D453A4D61726C696E20322E3050
:1013D0002E375F4457372E3320544D334420325339
:1013E0004D444E4E2028417072203234203230322B
:1013F000312032303A30303A32352920534F55526D
:1014000043455F434F44455F55524C3A687474708E
:10141000733A2F2F6769746875622E636F6D2F4959
:101420006E73616E6974794175746F6D6174696F03
:101430006E2F4D61726C696E2F747265652F4372E9
:1014400065616C6974794477696E5F322E30205023
:10145000524F544F434F4C5F56455253494F4E3AAB
:10146000312E30204D414348494E455F5459504537
:101470003A53755065522043522D3230204558540E
:1014800052554445525F434F554E543A31205555BD
:1014900049443A63656465326132662D34316132A4
:1014A0002D343734382D396231322D63353563367A
:1014B000326633363766660A0043616E6E6F74209B
:1014C0006F70656E207375626469722000256973A0
:1014D0000025696D20256973002569682025696DDF
:1014E0002025697300256964202569682025696DB8
:1014F000202569730025697920256964202569689C
:101500002025696D202569730023646566696E6511
:101510002044454641554C545F00626564004B646D
:1015200020004B6920004B70200050494420417539
:10153000746F74756E652066696E69736865642181
:101540002050757420746865206C617374204B7032
:101550002C204B6920616E64204B6420636F6E7396
:1015600074616E74732066726F6D2062656C6F7744
:1015700020696E746F20436F6E666967757261745F
:10158000696F6E2E680A00504944204175746F746B
:10159000756E65206661696C6564212074696D658E
:1015A0006F75740A00504944204175746F74756EEC
:1015B00065206661696C6564212054656D70657293
:1015C000617475726520746F6F20686967680A00BE
:1015D000204B643A2000204B693A2000204B703A9F
:1015E000200020436C617373696320504944200AD2
:1015F00000204E6F206F76657273686F6F740A00FB
:101600002054753A2000204B753A2000206D6178F7
:101610003A2000206D696E3A200020643A200020B4
:10162000626961733A2000504944204175746F74B7
:10163000756E652073746172740A005049442041CC
:1016400075746F74756E65206661696C65642120C0
:1016500054656D706572617475726520746F6F206A
:10166000686967680A00504944204175746F747551
:101670006E6500504944204175746F74756E652025
:101680006661696C656421204261642068656174EB
:1016900065722069640A004572723A207574663872
:1016A00020666F6E74206E6F7420696E6974696154
:1016B0006C697A65642E004572723A2075746638DA
:1016C00020666F6E74206E6F7420696E6974696134
:1016D0006C697A65642E004572723A2075746638BA
:1016E00020666F6E74206E6F7420696E6974696114
:1016F0006C697A65642E00FFE0FFD140A0C8A6A205
:101700002FF80023AC00AF10FFFEFF05FFD0FFE075
:10171000FFC1FFD1E240A0C8A6A22FF80023812775
:10172000AC00AFFFD0FF64FFD1A5FFD0FF64FF6422
:10173000FFD1A4FFD0FF16FFFE000C0F00FE070232
:101740002503BB017FFE08FE08FE05080806000011
:1017500040F0C88888987810050808060000C0F88E
:101760008888888888F80505050600012030F8304B
:10177000200508080600002070F820202020E00541
:1017800009090600FF2070A8A8B8888870200705FE
:1017900005070001D86C366CD80509090600FFF86A
:1017A000A88888888888A8F8050A0A0600FE2050BC
:1017B00050505088A8A8887003030306000340A077
:1017C00040FFFFFFFFFFFFFFFFFFFFFFFFFFFFFFE8
:1017D000FFFFFFFFFFFFFF0000000605FF010707F7
:1017E00006020080808080800080030303060105DC
:1017F000A0A0A005060606000050F85050F85005BD
:1018000009090600FF2070A8A07028A8702005070D
:1018100007060000C8C81020409898050707060072
:101820000040A0A040A89068010303060205808044
:10183000800309090601FF2040408080804040204D
:101840000309090601FF8040402020204040800518
:10185000070706000020A8702070A82005050506CF
:1018600000012020F820200203030601FFC0408071
:10187000050101060003F8020202060100C0C005CE
:1018800007070600000810102040408005070706E3
:101890000000708898A8C8887003070706010040F8
:1018A000C040404040E0050707060000708808106F
:1018B0002040F8050707060000F808103008887077
:1018C00005070706000010305090F81010050707B4
:1018D000060000F880F00808887005070706000079
:1018E000304080F0888870050707060000F808106F
:1018F000102020200507070600007088887088885F
:1019000070050707060000708888780810600205D7
:1019100005060100C0C000C0C00206060601FFC0E7
:10192000C000C04080030505060101204080402022
:10193000050303060002F800F8030505060101800F
:101940004020408005070706000070881020200016
:10195000200507070600007088B8A8B88070050742
:1019600007060000708888F8888888050707060041
:1019700000F04848704848F00507070600007088E6
:101980008080808870050707060000F048484848B6
:1019900048F0050707060000F88080F08080F80511
:1019A0000707060000F88080F080808005070706A2
:1019B00000007088808098887005070706000088FE
:1019C0008888F8888888030707060100E0404040BF
:1019D0004040E00507070600003810101010906026
:1019E0000507070600008890A0C0A090880507079B
:1019F000060000808080808080F8050707060000D0
:101A000088D8A8888888880507070600008888C8BD
:101A1000A898888805070706000070888888888845
:101A200070050707060000F08888F08080800507B1
:101A30000706000070888888A890680507070600D8
:101A400000F08888F0A090880507070600007088DD
:101A50008070088870050707060000F82020202005
:101A60002020050707060000888888888888700578
:101A70000707060000888888885050200507070659
:101A8000000088888888A8A85005070706000088F5
:101A90008850205088880507070600008888502055
:101AA000202020050707060000F80810204080F8D5
:101AB0000309090601FFE080808080808080E005C6
:101AC000070706000080404020101008030909069F
:101AD00001FFE020202020202020E0050303060055
:101AE000052050880501010600FEF80303030601E6
:101AF00005804020050505060000700878887805F7
:101B000007070600008080F0888888F00505050634
:101B100000007080808870050707060000080878BC
:101B2000888888780505050600007088F0807005B3
:101B30000707060000304840E04040400507070620
:101B400000FE708888887808700507070600008006
:101B500080F0888888880307070601004000C0409D
:101B60004040E00409090601FE100030101010107A
:101B7000906005070706000080808890E090880349
:101B80000707060100C04040404040E0050505064B
:101B90000000D0A8A8A8A8050505060000B0C888C0
:101BA0008888050505060000708888887005070785
:101BB0000600FEF0888888F080800507070600FE92
:101BC00078888888780808050505060000B0C88070
:101BD000808005050506000078807008F00507077D
:101BE0000600002020F8202020180505050600002A
:101BF0008888889868050505060000888888502030
:101C00000505050600008888A8A8500505050600FA
:101C10000088502050880507070600FE88888850F5
:101C2000204080050505060000F8102040F8030953
:101C3000090601FF20404040804040402001090942
:101C40000602FF80808080808080808003090906F2
:101C500001FF8040404020404040800503030600D3
:101C60000248A890FF554E4C4F41442046494C41F4
:101C70004D454E54004C4F41442046494C414D4542
:101C80004E540046494C414D454E54204348414E28
:101C900047450042656400456E636C6F73757265FD
:101CA000002568753A253032687500253032687530
:101CB0003A25303268750020202020202020002086
:101CC000202020001FE020102010201010201020C5
:101CD0002010201030300840048003001FE03FF047
:101CE0003FF03FF01FE01FE03FF03FF03FF00FC03C
:101CF000078003003FFFF038007030FC3020FC10FC
:101D00002078102030102C00D02E31D02F7BD02FF7
:101D10007BD02E31D02C00D020301020781020FC29
:101D20001030FC303800703FFFF03FFFF03800709B
:101D30003186302387102787902F87D02F03D0201C
:101D400030102078102078102030102F03D02F87EB
:101D5000D02787902387103186303800703FFFF0FE
:101D60001FFFF81FFFF8041040020820020820049B
:101D7000104008208010410010410008208004100D
:101D8000400000001FFFF81FFFF8FFFFFF80000169
:101D90008E00E19F01F19381399F81F99F81F99F25
:101DA000B9F98F28F18038018000019FFFF9917403
:101DB000999B06A99B54A99B56A99B54999FFFF9EF
:101DC000FFFFFF6E6F74696669636174696F6E20EF
:101DD0000063616E63656C005072696E74204162CD
:101DE0006F72746564004469736D6973730055495B
:101DF0002041626F72746564004D323520500A4D87
:101E0000323400526573756D650055492050617517
:101E100073650050617573696E672E2E2E007265B2
:101E200073756D65004D3234004C6F6164206D6DCB
:101E300000556E6C6F6164206D6D0046696C2E20DC
:101E40004469612E004520696E206D6D5E3300414E
:101E50006476616E6365204B004D3330332055311D
:101E60002045256920532569005049442041757457
:101E70006F74756E65202A005049442D44202A0055
:101E80005049442D49202A005049442D50202A0011
:101E900020082046616374002008204D61780020EE
:101EA00008204D696E004F6666004F6E00417574E4
:101EB0006F74656D70005654726176204D696E00C6
:101EC000566D696E00566D6178204500566D6178DB
:101ED000205A00566D6178205900566D617820585F
:101EE00000416D6178204500416D6178205A0041C4
:101EF0006D6178205900416D6178205800412D5462
:101F0000726176656C00412D526574726163740074
:101F1000416363656C0056652D4A65726B00565AC5
:101F20002D4A65726B0056592D4A65726B005658E2
:101F30002D4A65726B00452073746570732F6D6D4B
:101F4000005A2053746570732F6D6D0059205374BF
:101F50006570732F6D6D00582053746570732F6D0D
:101F60006D00416476616E636564205365747469C5
:101F70006E6773003F0043616E63656C00496E6974
:101F800074004D34323800496E697469616C697A45
:101F90006520454550524F4D0046696C616D656E38
:101FA000740054656D706572617475726500537468
:101FB0006570732F6D6D004A65726B0041636365D8
:101FC0006C65726174696F6E0056656C6F636974DD
:101FD000790053657420486F6D65204F66667365A0
:101FE000747300436F6E66696775726174696F6EB2
:101FF000003F004E65787420506F696E7400446F26
:102000006E65004E657874004C6576656C696E6728
:1020100020446F6E6521004D6F7665205A0047326F
:10202000395332004E65787420506F696E74002504
:1020300069202F2025750047323953310047323946
:10204000533200436C69636B20746F20426567698B
:102050006E00486F6D696E672058595A005A2056B5
:10206000616C756500496E646578205900496E643D
:10207000657820580053746F7265205365747469D5
:102080006E6773004C6F61642053657474696E678A
:1020900073004C6576656C20436F726E65727300D9
:1020A000426564205A004661646520486569676836
:1020B00074004F6666004F6E00426564204C657682
:1020C000656C696E670045646974204D65736800CE
:1020D0004C6576656C20426564004D6F74696F6E67
:1020E000003F0043616E63656C204F626A656374F4
:1020F000004E4F005945530043616E63656C204F9D
:10210000626A656374203D004D61696E00426564DA
:10211000004E6F7A7A6C650046616E20537065657B
:102120006400436F6E66696775726174696F6E00F3
:10213000526573746F72652044656661756C747363
:10214000004C6F61642053657474696E677300534B
:10215000746F72652053657474696E677300507292
:102160006568656174202420436F6E66004F666663
:10217000004F6E00506F776572204F757461676510
:10218000004C434420436F6E747261737400416469
:1021900076616E6365642053657474696E6773005D
:1021A0004D61696E004D37303220542564004D3644
:1021B000303020423020542564004D373032203BEF
:1021C0002564004D37303120542564004D373032BE
:1021D000004D373031004D363030204230004D61F7
:1021E000696E005075726765206D6F726500436F90
:1021F0006E74696E756500524553554D45204F50BC
:1022000054494F4E533A005052494E542050415574
:102210005345440020204E6F7A7A6C653A20005076
:1022200061726B696E672E2E2E0000005761697413
:1022300020666F720066696C616D656E74206368FC
:10224000616E676500746F2073746172740057610A
:10225000697420666F720066696C616D656E7420CA
:10226000756E6C6F616400004E6F7A7A6C652068E1
:10227000656174696E6700506C6561736520776194
:1022800069742E2E2E00005072657373206275746F
:10229000746F6E00746F2068656174206E6F7A7A57
:1022A0006C650000496E736572742066696C616DBF
:1022B000656E7400616E6420707265737320627560
:1022C00074746F6E00746F20636F6E74696E7565E1
:1022D000005761697420666F720066696C616D6594
:1022E0006E74206C6F6164000050726573732042DD
:1022F0007574746F6E00746F20726573756D6520F0
:102300007072696E7400005761697420666F722084
:102310007072696E7400746F20726573756D652ECE
:102320002E2E00005761697420666F720066696C1A
:10233000616D656E7420707572676500003E2000E7
:10234000256C642E25696D0045787472756465642A
:1023500020546F74616C003E20004C6F6E67657393
:1023600074204A6F622054696D65003E2000546FEE
:1023700074616C205072696E742054696D650043FD
:102380006F6D706C65746564003A20005072696E00
:102390007420436F756E74003A200031353000357B
:1023A000004245443A204154432031303447542DB3
:1023B000320052756E617761792057617463683AB3
:1023C000204F4E004D61782054656D7000333135DB
:1023D000004D696E2054656D7000350045313A201E
:1023E0004550434F53203130304B00505355004738
:1023F000656E657269630050726F746F636F6C0015
:10240000312E30004261756400323530303030009A
:10241000437265616C69747933442052414D505365
:10242000004D657368204C6576656C696E67004584
:10243000787472756465727300310074696E796DB9
:10244000616368696E657333642E636F6D005375E5
:102450005065522043522D323000323032312D300F
:10246000342D313800322E302E375F4457372E331B
:10247000004D61726C696E005072696E74657220F5
:10248000537461747300546865726D6973746F720C
:102490007300426F61726420496E666F005072690A
:1024A0006E74657220496E666F004D61696E004DF5
:1024B000313030300053746F70205072696E740088
:1024C000526573756D65205072696E7400506F7738
:1024D0006572204F7574616765003F004261636BF0
:1024E0000053746F70005072696E742066726F6D65
:1024F000204D65646961004368616E6765204D65C4
:10250000646961004D32310041626F757420507210
:10251000696E746572004368616E67652046696C18
:10252000616D656E7400436F6E6669677572617484
:10253000696F6E0054656D706572617475726500C7
:102540004D6F74696F6E00486F73742053746172BD
:1025500074004E6F204D6564696100526573756D3E
:1025600065205072696E740043616E63656C204F24
:10257000626A6563740054756E650053746F7020F1
:102580005072696E74005061757365205072696E87
:102590007400496E666F2053637265656E003F007C
:1025A0005374617274205072696E740043616E637B
:1025B000656C005072696E740043616E6E6F7420BA
:1025C000656E746572207375626469723A200002E8
:1025D0002E2E004D61696E002100486F74656E6497
:1025E00020746F6F20636F6C64004261636B0050F6
:1025F000726F63656564004F6666004F6E00536FCF
:10260000667420456E6473746F7073004D6F7469E7
:102610006F6E0044697361626C65205374657070FD
:10262000657273004D383400426564204C657665F0
:102630006C696E6700486F6D65205A004732385AE2
:1026400000486F6D652059004732385900486F6D5A
:102650006520580047323858004175746F20486F24
:102660006D6500473238004D61696E0050726568D3
:10267000656174202420456E640050726568656150
:10268000742024204265640054656D706572617425
:1026900075726500436F6F6C646F776E0050726582
:1026A0006865617420240046616E2053706565641E
:1026B000207E00426564004E6F7A7A6C65004D6141
:1026C000696E004261627973746570205A004164DA
:1026D00076616E6365204B00466C6F770046616ED5
:1026E000205370656564207E00426564004E6F7AF9
:1026F0007A6C6500426564205A0053706565640019
:102700004D61696E00486F6D696E67204661696C46
:102710006564006F70656E005452494747455245E5
:1027200044003A20007A5F6D696E00795F6D696ED2
:1027300000785F6D696E005265706F7274696E67C4
:1027400020656E6473746F70207374617475730A9E
:102750000020746F6F206C6F6E67206578747275DF
:1027600073696F6E2070726576656E7465640A00B9
:1027700020636F6C6420657874727573696F6E2066
:1027800070726576656E7465640A00000000000072
:10279000000000000000005761726E696E673A2009
:1027A000486F6D696E672042756D70204469766967
:1027B000736F72203C20310A000202040000704353
:1027C0000000704300007A43000000410000004117
:1027D0000000004000000001000000010000800037
:1027E000555555000000400033333300AAAA2A0093
:1027F0004992240000002000C7711C00999919001B
:10280000D1451700555515003BB11300244912005E
:1028100011111100000010000F0F0F00E3380E001F
:1028200043790D00CCCC0C00C3300C00E8A20B00A7
:1028300064210B00AAAA0A00703D0A009DD8090075
:10284000427B090092240900DCD308008888080034
:102850001042080000000800F0C107008787070049
:1028600075500700711C07003EEB0600A1BC060076
:102870006990060066660600703E06006118060054
:1028800017F4050074D105005BB00500B290050097
:10289000627205005555050078390500B81E05001F
:1028A000050505004EEC040087D40400A1BD04001A
:1028B00090A7040049920400C17D0400EE69040061
:1028C000C7560400444404005C320400082104009C
:1028D00041100400000004003FF00300F8E0030092
:1028E00026D20300C3C30300CCB503003AA80300FB
:1028F0000A9B0300388E0300C08103009F7503000C
:10290000D0690300505E03001D53030034480300E8
:10291000913D03003333030016290300381F0300E1
:1029200097150300300C0300030303000BFA0200A9
:1029300049F10200BAE802005CE002002DD8020072
:102940002DD0020059C80200B0C0020031B9020007
:10295000DAB10200AAAA0200A0A30200BC9C0200F5
:10296000FA9502005C8F0200DF880200828202007A
:10297000457C02002776020027700200436A0200AD
:102980007C640200D05E02003F590200C85302007E
:10299000FFFDFCFAF8F6F4F2F0EEECEAE9E7E5E325
:1029A000E1E0DEDCDAD9D7D5D4D2D0CFCDCBCAC8DE
:1029B000C7C5C3C2C0BFBDBCBAB9B7B6B4B3B2B065
:1029C000AFADACAAA9A8A6A5A4A2A1A09E9D9C9AC1
:1029D00099989795949392908F8E8D8B8A898887FA
:1029E0008684838281807F7E7D7B7A797877767515
:1029F00074737271706F6E6D6C6B6A69686766650F
:102A000064636261605F5E5D5C5B5A5958585756FB
:102A1000555453525150504F4E4D4C4B4A4A4948D1
:102A2000474646454443424241403F3E3E3D3C3B93
:102A30003B3A393838373635353433323231303045
:102A40002F2E2E2D2C2B2B2A2929282727262525EA
:102A500024232322212120201F1E1E1D1C1C1B1B82
:102A60001A1919181817161615151413131212110E
:102A700011100F0F0E0E0D0D0C0C0B0A0A09090890
:102A80000807070606050504040303020201000007
:102A9000000070430000704300007A430000000013
:102AA000000000000000000053657474696E6773D5
:102AB0002053746F72656400454550524F4D204954
:102AC0006E697469616C697A65640A003B20002054
:102AD000204D36303320002055004C0046696C6193
:102AE0006D656E74206C6F61642F756E6C6F6164C0
:102AF000206C656E677468733A0020204D39303061
:102B0000204B004C696E65617220416476616E6392
:102B1000653A0020204D343133205300506F7765E3
:102B2000722D4C6F7373205265636F766572793ABC
:102B30000020204D3235302043004C434420436F69
:102B40006E74726173743A002044002049002020A2
:102B50004D33303420500020440020490020204DC7
:102B60003330312050005049442073657474696ECD
:102B700067733A0020460020480020204D3134354C
:102B80002053004D6174657269616C2068656174E1
:102B9000757020706172616D65746572733A0020A2
:102BA00020473239205334205A00204A0020204741
:102BB000323920533320490020204D343230205305
:102BC000004D65736820426564204C6576656C69CC
:102BD0006E673A0020204D323036205800486F6D25
:102BE00065206F66667365743A00205800205300B4
:102BF00020204D323035204200416476616E63659D
:102C0000643A20423C6D696E5F7365676D656E74F2
:102C10005F74696D655F75733E20533C6D696E5FCF
:102C200066656564726174653E20543C6D696E5FD3
:102C300074726176656C5F66656564726174653E29
:102C400020583C6D61785F785F6A65726B3E2059F1
:102C50003C6D61785F795F6A65726B3E205A3C6DAE
:102C600061785F7A5F6A65726B3E20453C6D617882
:102C70005F655F6A65726B3E002054002052002041
:102C8000204D323034205000416363656C657261C1
:102C900074696F6E2028756E6974732F7332293AC8
:102CA00020503C7072696E745F616363656C3E2096
:102CB000523C726574726163745F616363656C3EFC
:102CC00020543C74726176656C5F616363656C3E31
:102CD0000020204D3230312058004D6178696D75EB
:102CE0006D20416363656C65726174696F6E202845
:102CF000756E6974732F7332293A0020204D32307B
:102D0000332058004D6178696D756D206665656486
:102D100072617465732028756E6974732F73293A14
:102D20000053746570732070657220756E69743A13
:102D30000020440020204D323030205300204469D0
:102D40007361626C65640A0046696C616D656E74DE
:102D50002073657474696E67733A0020204D3134B6
:102D6000392043203B20556E69747320696E2043DF
:102D7000656C736975730A0020286D6D2900202029
:102D8000473231202020203B20556E697473206922
:102D90006E206D6D0000803B4400803B44000020AD
:102DA00041000096420000A0420000A0420000C87E
:102DB000430000BE42D0070000D0070000640000BE
:102DC000004B00000024F4D43050C38E20C2A24037
:102DD00017828B7011127A910D816CD90AA861E16A
:102DE00008C7586607615143061E4B5D05C145A7DC
:102DF000041A411104093D9803713931034036DB4F
:102E00000265339102D4305402802E1D02632CEEF1
:102E100001752AC501B028A001102781018F256402
:102E2000012B244B01E0223401AC211F018D200D28
:102E300001801FFC00841EED00971DDF00B81CD22E
:102E400000E61BC600201BBC00641AB200B219A821
:102E5000000A19A0006A189900D117910040178B39
:102E600000B516840031167E00B31579003A15734B
:102E700000C7146F0058146A00EE136600881363CD
:102E80000025135E00C7125B006C12570015125428
:102E900000C111510070114F0021114B00D6104993
:102EA000008D1047004610440002104200C00F4041
:102EB00000800F3E00420F3C00060F3B00CB0E3857
:102EC00000930E37005C0E3500270E3400F30D32F0
:102ED00000C10D3100900D3000600D2E00320D2D1F
:102EE00000050D2C00D90C2B00AE0C2900850C29F7
:102EF000005C0C2700350C27000E0C2600E80B2484
:102F000000C40B2400A00B23007D0B23005A0B21CF
:102F100000390B2100180B2000F80A1F00D90A1EE7
:102F200000BB0A1E009D0A1D00800A1D00630A1CCA
:102F300000470A1B002C0A1B00110A1A00F7091A85
:102F400000DD091900C4091900AB0919009209171D
:102F5000007B091800630917004C09160036091692
:102F600000200916000A091500F5081500E00814EC
:102F700000CC081400B8081400A40814009008132A
:102F8000007D0812006B0813005808120046081252
:102F90000034081100230811001208110001081163
:102FA00000F0071000E0071000D0071000C0071065
:102FB00000B0070F00A107100091070E0083070F54
:102FC0000074070F0065070E0057070E0049070E33
:102FD000003B070D002E070E0020070D0013070D04
:102FE0000006070D00F9060C00ED060D00E0060CCA
:102FF00000D4060C00C8060C00BC060C00B0060C81
:1030000000A4060B0099060C008D060B0082060B2F
:103010000077060B006C060B0061060A0057060BD2
:10302000004C060A0042060A0038060A002E060A6C
:103030000024060A001A060A001006090007060AFC
:1030400000FD050900F4050900EB050900E205098A
:1030500000D9050900D0050900C7050900BE05090A
:1030600000B5050800AD050800A50509009C050888
:1030700000940508008C050800840508007C0508FC
:1030800000740508006C050700650508005D05076C
:1030900000560508004E05070047050700400508D3
:1030A0000038050700310507002A0507002305073A
:1030B000001C050600160507000F05070008050699
:1030C0000002050700FB040600F5040700EE0406F5
:1030D00000E8040600E2040700DB040600D504064D
:1030E00000CF040600C9040600C3040600BD0406A0
:1030F00000B7040600B1040500AC040600A60406EF
:1031000000A00405009B0406009504050090040639
:10311000008A04050085040500800406007A040581
:103120000075040500700405006B040500660405C5
:1031300000610405005C0405005704050052040505
:10314000004D04050048040500430405003E040446
:10315000003A04050035040500300404002C040581
:103160000027040400230405001E0404001A0404BC
:103170000016040500110404000D040400090405F0
:10318000000404040000040400FC030400F8030429
:1031900000F4030400F0030400EC030400E803045B
:1031A00000E4030400E0030400DC030400D803048B
:1031B00000D4030400D0030400CC030400C80303BC
:1031C00000C503030024F404D9201BC40C5C0E9832
:1031D00004C4095F0265077101F405F900FB04B33B
:1031E0000048048700C103690058035500030345E4
:1031F00000BE023A008402310053022A002902254F
:103200000004022000E4011C00C8011900AF0117EE
:103210000098011400840113007101100061011075
:103220000051010E0043010D0036010B002B010B74
:103230000020010B00150109000C01090003010821
:1032400000FB000800F3000800EB000700E40006A4
:1032500000DE000600D8000600D2000600CC000503
:1032600000C7000500C2000500BD000400B900044D
:1032700000B5000400B1000400AD000400A9000482
:1032800000A5000300A20003009F0004009B0003B0
:1032900000980003009500020093000300900003D3
:1032A000008D0002008B00030088000200860002EF
:1032B0000084000300810002007F0002007D000204
:1032C000007B000200790002007700010076000216
:1032D000007400020072000100710002006F000221
:1032E000006D0001006C0002006A0001006900022C
:1032F0000067000100660001006500010064000233
:10330000006200010061000100600001005F000236
:10331000005D0001005C0001005B0001005A00013B
:10332000005900010058000100570001005600013B
:10333000005500010054000100530000005300013B
:10334000005200010051000100500001004F000137
:10335000004E0000004E0001004D0001004C000135
:10336000004B0000004B0001004A00010049000131
:10337000004800000048000100470001004600002E
:103380000046000100450000004500010044000126
:103390000043000000430001004200000042000121
:1033A000004100000041000100400001003F00001A
:1033B000003F0001003E0000003E0001003D000013
:1033C000003D0001003C0000003C0000003C00010A
:1033D000003B0000003B0001003A0000003A000101
:1033E00000390000003900010038000000380000FA
:1033F00000380001003700000037000100360000EF
:1034000000360000003600010035000000350000E5
:1034100000350001003400000034000000340001D9
:1034200000330000003300000033000100320000D0
:1034300000320000003200010031000000310000C5
:1034400000310001003000000030000000300001B9
:10345000002F0000002F0000002F0000002F0001AF
:10346000002E0000002E0000002E0001002D0000A4
:10347000002D0000002D0000002D0001002C000098
:10348000002C0000002C0000002C0001002B00008C
:10349000002B0000002B0000002B0001002A000080
:1034A000002A0000002A0000002A00010029000074
:1034B0000029000000290000002900000029000167
:1034C000002800000028000000280000002800005C
:1034D000002800010027000000270000002700004E
:1034E0000027000000270001002600000026000041
:1034F0000026000000260000002600010025000034
:103500000025000000250000002500000025000027
:103510000025000100240000002400000024000019
:10352000002400000024000100230000002300000C
:1035300000230000002300000023000000230000FF
:1035400000230001002200000022000000220000F1
:1035500000220000002200000022000100210000E3
:1035600000210000002100000021000000210000D7
:1035700000210000002100010020000000200000C8
:1035800000200000002000000020000000200000BB
:103590000020000000200001001F0000001F0000AC
:1035A000001F0000001F0000001F0000001F00009F
:1035B000001F0001001E0000001E0000001E000091
:1035C000001E000000232C0000B822000056180046
:1035D000003A0F0000B8080000B1040000710200BA
:1035E000003E01000020436F756E7420583A00427F
:1035F000656400453100626564002C207379737442
:10360000656D2073746F7070656421204865617406
:1036100065725F49443A200048656174696E6720AD
:103620004661696C65640048656174696E6720660F
:1036300061696C6564004D31313220536875746482
:103640006F776E001000C90210012C0140012201A9
:1036500070011801B0010E01F00104015002FA00DE
:10366000B002F0003003E600D003DC009004D2008A
:103670007005C800A006BE000008B400B009AA008A
:10368000D00BA000600E960060118C000015820027
:1036900020197800C01D6E00A0226400B0275A00D7
:1036A000902C500000314600E0343C0010383200CD
:1036B000903A2800603C1E00A03D1400803E0A00A5
:1036C000203F0000544845524D414C2052554E4138
:1036D00057415900546865726D616C2052756E6176
:1036E000776179004572723A204D415854454D50EA
:1036F000004D415854454D5020747269676765729A
:103700006564004572723A204D494E54454D500053
:103710004D494E54454D5020747269676765726516
:103720006400202F002042403A0020403A002057F9
:103730003A0020573A00496E76616C6964206578DA
:103740007472756465720A007C3C3E5E2B3D3F2FAF
:103750005B5D3B2C2A225C0043616E6E6F74206FB0
:1037600070656E207375626469722000534420494D
:103770006E6974204661696C005344206361726411
:10378000206F6B0A006F70656E526F6F74206661F8
:10379000696C65640A00766F6C756D652E696E697B
:1037A00074206661696C65640A004E6F2053442082
:1037B000636172640A000A4D3234004D32332025B1
:1037C000730041425300504C41002E0A006F706557
:1037D0006E206661696C65642C2046696C653A20D0
:1037E0000046696C652073656C65637465640A00E6
:1037F0002053697A653A200046696C65206F7065D0
:103800006E65643A2000454E4420535542524F5550
:1038100054494E450A002220706F730022207061C7
:1038200072656E743A2200535542524F5554494EB8
:10383000452043414C4C207461726765743A220004
:1038400053756263616C6C204F766572666C6F773E
:10385000004578636565646564206D617820535523
:1038600042524F5554494E452064657074683A0081
:103870002E0A0044656C6574696F6E206661696C20
:1038800065642C2046696C653A200046696C6520A9
:1038900064656C657465643A005344207072696EA7
:1038A00074696E67206279746520004E6F742053CE
:1038B00044207072696E74696E670A002F617574B6
:1038C0006F25632E670057726974696E6720746F85
:1038D0002066696C653A2000667265736800646FE3
:1038E000696E67002066696C653A20004E6F77202C
:1038F0000002FD55555555555FFFFFFFFFFFFFFFC8
:10390000FFFFFE00000000003FFFFFFFFFFFFFFF83
:10391000FFFFFD000007FFFFFFFFFFFFFFFFFFFFAF
:10392000FFFFFE07C00555555555555FFFFFFFFFCB
:10393000FFFFFC0A200600000000003FFFFFFFFF22
:10394000FFFFFE141005000007FFFFFFFFFFFFFF52
:10395000FFFFFC28080607C00555555555555FFF64
:10396000FFFFFE5404040A200600000000003FFF91
:10397000FFFFFC600406141005000007FFFFFFFFB7
:10398000FFFFFE50040428080607C005555555558D
:10399000555FFC6004065404040A20060000000081
:1039A000003FFE54041C60040614100500000000D3
:1039B000001FFC28082E50040428080607C0000138
:1039C000F03FFE1410546004065404040A20000260
:1039D000081FFC0A206654041C600406141000052D
:1039E000043FFE07C05428082E5004042808000A8B
:1039F000021FFC00002E141054600406540400152D
:103A0000013FFE00001C0A206654041C60040018DC
:103A1000011FFC00000607C05428082E50040014A3
:103A2000013FFE00000400002E1410546004001832
:103A3000011FFCFFFFFE00001C0A206654041C1539
:103A4000013FFED5555400000607C05428082A0A35
:103A5000021FFC84104600000400002E14105105C3
:103A6000043FFEC41044FFFFFE00001C0A20610258
:103A7000881FFC841046D5555400000607C051012C
:103A8000F03FFE84104484104600000400002A0029
:103A9000001FFCC41046C41044FFFFFE00001C00C1
:103AA000003FFE841044841046D5555400000000A9
:103AB000001FFCD5555684104484104600000000B9
:103AC000003FFCFFFFFCC41046C41044FFFFFFFF93
:103AD000FF9FFE000006841044841046D5555555BE
:103AE00055BFFD555554D555568410448410410496
:103AF000109FFFFFFFFCFFFFFCC41046C4104104F1
:103B000011BFFFFFFFFE0000068410448410410433
:103B1000109FFFFFFFFD555554D5555684104104A5
:103B2000109FFFFFFFFFFFFFFCFFFFFCC4104104DD
:103B300011BFFFFFFFFFFFFFFE00000684104104DE
:103B4000109FFFFFFFFFFFFFFD555554D5555555FD
:103B500055BFFFFFFFFFFFFFFFFFFFFCFFFFFFFF62
:103B6000FF9FFFFFFFFFFFFFFFFFFFFE00000000C2
:103B7000003FFFFFFFFFFFFFFFFFFFFD55555555BE
:103B8000555FFFFFFFFFFFFFFFFFFFFFFFFFFFFF8F
:103B9000FFFFFFFFFFFFFFFFFFFFFFFFFFFFFFFF35
:103BA000FFFFFFFFFFFFFFFFFFFFFFFFFFFFFFFF25
:103BB000FFFFFFFFFFFFFFFFFFFFFFFFFFFFFFFF15
:103BC000FFFFE02EFB7DFBFBCFC1DFBB3EC0E1FE74
:103BD0003C1FFDEE7B39F9F3CF9EDFBB3EDFDEFC01
:103BE000DDE7FDEE3BBBF9EBD7BF5FBB5EDFDEFD84
:103BF000EDF7FDEEBBD3FAEBB73FDFBB4EDFDFFFE8
:103C0000CDF3FDEEDBC7FAEBBB7FC03B6EC0E3FF3D
:103C10001DF3FDEECBEFFADBBB7FDFBB66DFF8FF0A
:103C2000CDF3FDEEEBEFFB5B033F5FBB76DFFE7F8B
:103C3000EDF3FDEEF3EFFB5B79BEDFBB7ADFDE7DFC
:103C4000EDF7FDEEF3EFFBBAFD9EDFBB7CDFDEFDA3
:103C5000CDE7FDEEFBEFFBBAFDC1DFBB7EC0E0FEB2
:103C60001C1F6D61726C696E66772E6F7267003211
:103C70002E302E375F4457372E33001FFFFFFFFFD4
:103C8000FFFF600000000001FF400000000000FF97
:103C90008000000000007F83CF00000C303F87FFD2
:103CA00080000C301F867980000C000F8C30C78399
:103CB0008C30E78C30CFC7CC31F38C30DCECEC337C
:103CC000B98C30D86C6C33198C30D06C0C33198CA7
:103CD00030D86C0C33198C30DC6C0E3B198C30CF27
:103CE0007C079F198C30C77C038F194000000000AF
:103CF0000002600000000000061FFFFFFFFFFFF84A
:103D000070012C0190012701B0012201C0011D01A9
:103D1000F00118011002130130020E0160020901C6
:103D200090020401C002FF000003FA004003F50006
:103D30008003F000D003EB002004E6007004E100F3
:103D4000E004DC004005D700C005D2004006CD00ED
:103D5000D006C8008007C3003008BE00F008B900D4
:103D6000C009B400B00AAF00B00BAA00D00CA50087
:103D7000000EA000500F9B00C01096005012910042
:103D800000148C00C0158700B0178200B0197D00A8
:103D9000D01B7800001E730040206E009022690046
:103DA000F024640040275F0090295A00E02B550062
:103DB000102E500020304B0010324600E0334100FE
:103DC00090353C001037370070383200A0392D0094
:103DD000B03A2800A03B2300603C1E00103D1900B3
:103DE000903D1400103E0F00703E0A00C03E0500DA
:103DF000003F0000403FFBFF803FF6FFC03FF1FF68
:103E00002020506C616E6E65724275666665724206
:103E1000797465733A20002046726565204D656DA2
:103E20006F72793A2000436F6D70696C65643A2057
:103E300041707220323420323032310A00204C611D
:103E4000737420557064617465643A203230323185
:103E50002D30342D3138207C20417574686F723AD2
:103E60002054696E794D616368696E657333440AE5
:103E700000322E302E375F4457372E330A004D6103
:103E8000726C696E0020536F6674776172652052A0
:103E9000657365740A00205761746368646F6720F6
:103EA00052657365740A002042726F776E206F75D9
:103EB000742052657365740A002045787465726ECB
:103EC000616C2052657365740A00506F7765725596
:103ED000700A0073746172740A00473238585900CE
:103EE0004D31303031006572726F722077726974B3
:103EF000696E6720746F2066696C650A00446F6E96
:103F00006520736176696E672066696C652E0A00AC
:103F10004D323900456E6473746F70730025532001
:103F2000256320256320256320256300205A3A005D
:103F300020593A0020583A00656E6473746F7073AC
:103F4000206869743A200000000A0B02090C0D0E6B
:103F5000080703040100000000000000000000004A
:103F60000000000000000000000000000000000051
:103F7000000000121110000000000000000000000E
:103F800000000000000000000000000000004D6F75
:103F900076652025736D6D004D6F766520302E316E
:103FA0006D6D004D6F766520316D6D004D6F7665DE
:103FB0002031306D6D004D6F76652041786973005A
:103FC0004578747275646572004D6F7665205A008D
:103FD0004D6F76652059004D6F7665205800C637C5
:103FE000C2374368616E67652046696C616D656EB6
:103FF0007400556E6C6F61642046696C616D656E0E
:1040000074004C6F61642046696C616D656E74006C
:104010005072656865617420437573746F6D0050EC
:104020007265686561742024004261636B00FFFF64
:10403000FF486F6D652025732573257320466972CF
:1040400073740070726F6D70745F0073686F7700C7
:10405000627574746F6E00626567696E0050757288
:1040600067654D6F72650050617573656400436FDD
:104070006E74696E7565004C6F61642046696C6191
:104080006D656E74205400496E73657274206669A4
:104090006C616D656E7420616E642073656E642062
:1040A0004D3130380A00220A00556E6B6E6F776E04
:1040B00020636F6D6D616E643A2022002042002003
:1040C00050006F6B0053755065522043522D3230B3
:1040D0002052656164792E005072696E74696E6752
:1040E0002E2E2E005072696E7420506175736564B7
:1040F00000204500205A00205900204D3932205818
:104100000020453A00205A3A0020593A00583A0017
:1041100020746F6F206C6F6E672065787472757392
:10412000696F6E2070726576656E7465640A002032
:10413000636F6C6420657874727573696F6E20703C
:10414000726576656E7465640A00526573656E64A7
:104150003A20006E6F74696669636174696F6E20DE
:104160000000002200250028002B002E0031003422
:104170000002010000050108010B010000210024DC
:104180000027002A002D0030003300010100000448
:104190000107010A010505050507050808080802C9
:1041A0000202020A0A0808040404040101010101D0
:1041B0000101010303030303030303040707070CBF
:1041C0000C0C0C0C0C0C0C02020202060606060675
:1041D0000606060B0B0B0B0B0B0B0B010210202022
:1041E000080810204010204080020102010804024B
:1041F00001010204081020408080402010080402C1
:104200000180040201804020100804020108040219
:10421000010102040810204080010204081020401F
:1042200080002001240211241FBECFEFD1E2DEBFA7
:10423000CDBF00E00CBF13E0A0E0B2E0E2E3FAEB98
:1042400002E00BBF02C007900D92AC36B107D9F760
:1042500028E1ACE6B3E001C01D92A63DB207E1F74C
:1042600011E2C2E1D1E200E006C021970109802FEE
:10427000FE010F947659C131D10780E00807A9F7F4
:104280000F942C480D94075D0C940000FC01849160
:104290000895FC018081089590E080E00895CF9317
:1042A000DF93DB01F9019C919130C1F0943080F0F3
:1042B00094509C938830D1F480819181009771F063
:1042C000019791838083480F591FEA01188206C025
:1042D0008C3539F49C5F9C93943041F4DF91CF91FD
:1042E00008958B3339F781E08C93F8CF20813181A9
:1042F000B9016F5F7F4F71836083420F531FEA01E3
:104300008883808191818F3591056CF7E7CF0F937A
:104310001F9381E00091BD161091BE162091BF162B
:104320003091C0164091B9165091BA166091BB16E3
:104330007091BC16041715072607370708F480E0AC
:104340001F910F91089590E080E00895282F90919B
:104350006608833021F495FD0FC094FD0FC0892FAE
:1043600090E0B0E0A0E004C0B695A795979587953A
:104370002A95D2F78170089581E0089580E008952C
:10438000129A0895269A2E9A0895EF92FF920F930B
:104390001F93CF93DF93EC018B017A018A859B8574
:1043A0008617970731F0888199810F94783D1B8794
:1043B0000A87B701888199810F943D2F2E813F8113
:1043C000820F932F911D9F838E8390E080E0DF9179
:1043D000CF911F910F91FF90EF9008959F92AF9210
:1043E000BF92CF92DF92EF92FF920F931F93CF93E2
:1043F000DF93EC018B01942EA52E8A859B85861771
:10440000970731F0888199810F94783D1B870A873F
:1044100088859985019649F5BC800A818E81080FAF
:10442000C880D980D6015596ED91FC91C6011995A9
:10443000B80EE92CFA2C10E0F70121917F0121112F
:1044400027C08E819F81810F911D9F838E8390E075
:1044500080E0DF91CF911F910F91FF90EF90DF905F
:10446000CF90BF90AF909F9008950E811F81692DCE
:104470007A2D888199810F943D2F800F912F911D66
:10448000288539852817390738F681E090E0E1CF93
:104490004B2D602FC6010F94D03D080F180FCCCFC5
:1044A000DF92EF92FF920F931F93CF93DF93EC0174
:1044B000D62E1CAD0BAD7C0184E0E80EF11CE98D1D
:1044C000FA8DC7011995412F480F2D2D602FC70177
:1044D0000F94D03D9BAD890F8BAF81E090E0DF91D1
:1044E000CF911F910F91FF90EF90DF900895AF92C1
:1044F000BF92DF92EF92FF920F931F93CF93DF93C0
:104500008C01EB01D42E79018FE0481709F486C0A5
:10451000A5E14A17B1F1BAE04B130EC0EC81FD8161
:1045200030E020E042E061E0C80119954CE057E13D
:10453000BE01C8010F947B3E0A80DB81C02DF2E3EF
:10454000DF1609F4E2C0FD1508F491C085E1D81624
:1045500009F4E0C0A7E1DA1609F4EFC0B4E1DB1218
:104560007BC0EE81FF818D8190E0880F991F8E0FB7
:104570009F1F11928E179F07E1F7CE010F94983B72
:104580006BC0AA80BB8047EF56E1C8010F947B3E09
:10459000F5014481440F406BBE01C8010F94633E96
:1045A00041E0BE01C8010F946B3ED50116962D91D6
:1045B0003C911797EC81FD8115964C9166E0C801FE
:1045C000199540E0BE01C8010F94733E47EF56E1D4
:1045D000BE01C8010F947B3EF5014481440F4F5F3B
:1045E000406BBE01C8010F94633E41E0BE01C801AB
:1045F0000F946B3ED50115964C91159716962D91FB
:104600003C91240F311DEC81FD8166E0C8011995B4
:1046100040E0BE01C8010F94733E8ECF41E0C80157
:104620000F94733E40E0BE01C8010F946B3E41E819
:10463000BE01C8010F94633EF701408150E05595DB
:10464000479555954795BE01C8010F94633E40E0DC
:10465000BE01C8010F94733E81E0DF91CF911F919D
:104660000F91FF90EF90DF90BF90AF900895E6E438
:10467000DE1609F471C0F7E4DF1609F471C08BE3AC
:10468000D812EACFD70111969C91119713968C916D
:1046900038E0390F813031F0833011F0392F02C00A
:1046A000392F985021E04B81491708F420E041E070
:1046B000391708F040E091E05A81351708F490E08E
:1046C000322F342B932311F4242331F2F70112817A
:1046D00000E0D12C843048F490E0FC01E855FD4F17
:1046E000D0808C559D4FDC010C9117FF04C0B701A1
:1046F000CE010F949F3BF70180818D0D80838181D6
:10470000800F8183110F89F7A7CFB701CE010F94D6
:104710009F3BA2CFCE010F94823B882309F49DCF0B
:10472000EE81FF818D8190E0880F991F8E0F9F1F72
:1047300011928E179F07E1F78FCFD7011C928A81C4
:1047400011968C9311978D81815012968C931297AC
:104750008B8113968C9380CF8D81F70180837CCFE2
:104760008981D7018C9378CFAB01BC014093BD16F2
:104770005093BE166093BF167093C01686E298E100
:104780000C94BACE809323028032B8F5909107053D
:10479000891724F091E0980F909307054091030545
:1047A000509104056091050570910605082E04C01E
:1047B00076956795579547950A94D2F7417040933F
:1047C000521087FD1DC0282F082E000C330B3F937D
:1047D0008F938EE599E09F938F938EE699E09F9358
:1047E0008F931F920E9449B28DB79EB707960FB65E
:1047F000F8949EBF0FBE8DBF089510925210E1CF66
:104800000D9492420F931F93CF93DF9300D01F928A
:10481000CDB7DEB79C0105E318E090E1EDE9F0E1EA
:10482000D80101900D929A95E1F7F901208131812B
:1048300042815381F80160857185828593850F944B
:104840007F59F801608771878287938780E090E0C5
:10485000A0EAB0E489839A83AB83BC83CE0101963E
:104860000E9461F90F900F900F900F90DF91CF9100
:104870001F910F9108952F923F924F925F926F92E6
:104880007F928F929F92AF92BF92CF92DF92EF92E0
:10489000FF921F93CF93DF93CDB7DEB72C970FB660
:1048A000F894DEBF0FBECDBF7A011901DC012D9156
:1048B0003D914D915C912D833E834F835887FB0141
:1048C000408051806280738080909D1090909E10F7
:1048D000A0909F10B090A010A50194016D817E81E1
:1048E0008F8198850F948D5281110EC011E0A30124
:1048F00092016091A1107091A2108091A3109091EB
:10490000A4100F948D52811110E0D1012D913D9191
:104910004D915C9129873A874B875C87F701C0806E
:10492000D180E280F3802091090230910A02409107
:104930000B0250910C02C701B6010F948D528823CF
:1049400009F44EC0C0920902D0920A02E0920B0212
:10495000F0920C028091A9109091AA10A091AB1036
:10496000B091AC104091A1105091A2106091A31091
:104970007091A4108092350890923608A092370862
:10498000B09238084093390850933A0860933B0836
:1049900070933C08C0923D08D0923E08E0923F08D8
:1049A000F09240088093410890934208A0934308F6
:1049B000B093440820E030E040E05FE36091801075
:1049C0007091811080918210909183100F94F35216
:1049D00069837A838B839C83CE0101960E9461F95F
:1049E0002D813E814F8158852093350830933608BC
:1049F00040933708509338084092390850923A084B
:104A000060923B0870923C08D1012D913D914D91EF
:104A10005C916091410870914208809143089091A7
:104A200044080F947F596093410870934208809323
:104A300043089093440811112FC020E030E0A901F1
:104A400069857A858B859C850F948D52811133C041
:104A500060E070E088EC92E469837A838B839C83C6
:104A6000CE0101960E9461F92C960FB6F894DEBF34
:104A70000FBECDBFDF91CF911F91FF90EF90DF90E0
:104A8000CF90BF90AF909F908F907F906F905F90EE
:104A90004F903F902F9008952AEF3EE74AE25FE360
:104AA000609184107091851080918610909187108C
:104AB0000F94F352D1CF60E070E080EA91E4CCCF64
:104AC0008091BF049091C004009731F04AE050E01B
:104AD00070E060E00D94A85060E070E0CB010895B4
:104AE00080915F0982FF0BC063E682E49AE00E9436
:104AF00064B20F948C350E9429B981E0089580E05A
:104B000008958091BF049091C004009731F04AE06D
:104B100050E070E060E00D947A4F60E070E0CB010F
:104B20000895AF92BF92CF92DF92EF92FF920F93D0
:104B30001F93CF93DF93EC015B018A01FB01199571
:104B400087FD16C0C82ED12CF12CE12C2196F8013E
:104B5000C082D182E282F382CE01DF91CF911F9198
:104B60000F91FF90EF90DF90CF90BF90AF9008959E
:104B7000982F907E903CA9F48F7190E0B0E0A0E077
:104B80006C017D0156E0CC0CDD1CEE1CFF1C5A951F
:104B9000D1F7CE010196F50119958F73C82A229697
:104BA000D6CF982F907F903E11F58F7090E0B0E0B7
:104BB000A0E06C017D0136E0CC0CDD1CEE1CFF1C7E
:104BC0003A95D1F7CE010196F50119958F73C82A50
:104BD00046E0CC0CDD1CEE1CFF1C4A95D1F7CE0143
:104BE0000296F50119958F73C82A2396B0CF982F96
:104BF000987F903F79F5877090E0B0E0A0E06C017D
:104C00007D0186E0CC0CDD1CEE1CFF1C8A95D1F7E3
:104C1000CE010196F50119958F73C82A96E0CC0C48
:104C2000DD1CEE1CFF1C9A95D1F7CE010296F50112
:104C300019958F73C82A26E0CC0CDD1CEE1CFF1CD6
:104C40002A95D1F7CE010396F50119958F73C82ADD
:104C500024967DCF982F907C903841F4807C8038CA
:104C600069F42196CE01F5011995F8CF8E7F8D3F1D
:104C700028F02196CE01F5011995F8CFC12CD12C41
:104C8000760165CF9CE0899F802D112491E0980FDB
:104C9000909308052CE0280F20932F0830E02E5F1A
:104CA0003F4F409187164217130619F014F080E029
:104CB0000895209189169217D0F7662341F08E5FF0
:104CC0000F94923C80912F088E5F0F94923C8091BC
:104CD0002F0890918716891750F32091891690918B
:104CE0000805291720F310928A1680938B1681E00D
:104CF00008952091F904022E000C330B821713063D
:104D000041F08093F90469E377E183E596E10D943E
:104D1000783D08951F93CF93DF931F92CDB7DEB7F1
:104D20008F3F910519F014F08FEF90E088379105CF
:104D300014F488E790E09093520280935102182F68
:104D400080918C16811105C081E080938C160F94A0
:104D5000B93B609155167091561619839E012F5FCD
:104D60003F4F4FE083E596E10F94B53B0F90DF9105
:104D7000CF911F910895CF938091FA0481114FC074
:104D800010928A1610928B1610928C16109258164A
:104D90001092571610925A161092591610925C16CD
:104DA00081E080935B1682E280935D16109262161A
:104DB00010926116E6E7F6E124E836E18FEF819381
:104DC0002E173F07E1F7C1E0C093731628E231E0E8
:104DD0003093691620936816C0936A1610926B166A
:104DE00010926C1690E490936D1610926E1626E653
:104DF00032E0309385162093841626E132E030931A
:104E000056162093551699E1909378169BE190934E
:104E10007716809376160F94B93BC093FA0480916D
:104E20005102909152020E948A2681E08093FB04F5
:104E300087EF96E19093C6158093C5151092C8151B
:104E40001092C715CF910895CF92DF92EF92FF9203
:104E50000F931F93CF93DF93CDB7DEB72C970FB689
:104E6000F894DEBF0FBECDBF6F3F71058105910580
:104E700009F0D0F48FE496E10E945022E091571699
:104E8000F09158163196849190E02C960FB6F894D4
:104E9000DEBF0FBECDBFDF91CF911F910F91FF906D
:104EA000EF90DF90CF900895F0908A16E0908B16E7
:104EB0002091FB0421110FC047ED56E16E2D8F2D7F
:104EC0000F943C3E90E080E0F80EF0928A16E0925B
:104ED0008B169927DACFC0905716D090581623E535
:104EE00036E13A8329832F2D30E03C832B832E2D0E
:104EF00030E03E832D8318861F822FEF3FEF3A87E5
:104F000029871C861B860EEE11E29E012F5F3F4F04
:104F1000AB01BC01C6010F947925B60183E596E18A
:104F20000F94783D8F819885CFCFCF93DF93FC018D
:104F300025AD211104C021E025AF0F94B93BC091EC
:104F40005516D0915616E0918416F091851682E0A0
:104F50001995E0918416F091851681E0199530E05D
:104F600020E044E1BE0183E596E10F94B53B26E8DD
:104F700036E147E1BE0183E596E10F94B53BE09150
:104F80008416F091851680E0DF91CF911994CF922D
:104F9000DF92EF92FF920F931F93CF93DF93CDB7E2
:104FA000DEB72C970FB6F894DEBF0FBECDBFF090E2
:104FB0008A16E0908B162091FB0421111DC047EB4F
:104FC00056E16E2D8F2D0F943C3E90E080E0F80E60
:104FD000F0928A16E0928B1699272C960FB6F894C9
:104FE000DEBF0FBECDBFDF91CF911F910F91FF901C
:104FF000EF90DF90CF900895C0905716D09058163C
:1050000023E536E13A8329832F2D30E03C832B833F
:105010002E2D30E03E832D8318861F827A87698784
:105020001C861B860EEE11E29E012F5F3F4F46E469
:1050300051E2BC01C6010F943D26B60183E596E11D
:105040000F94783D8F819885C2CF6FEF7FEF0C94DE
:10505000C727CF92DF92EF92FF920F931F93CF93C8
:10506000DF93CDB7DEB72C970FB6F894DEBF0FBE37
:10507000CDBFF0908A16E0908B162091FB04211191
:105080001DC047E956E16E2D8F2D0F943C3E90E0F8
:1050900080E0F80EF0928A16E0928B1699272C96F3
:1050A0000FB6F894DEBF0FBECDBFDF91CF911F9139
:1050B0000F91FF90EF90DF90CF900895C09057161A
:1050C000D090581623E536E13A8329832F2D30E01E
:1050D0003C832B832E2D30E03E832D8318861F8248
:1050E0007A8769871C861B860EEE11E29E012F5F70
:1050F0003F4F49E451E2BC01C6010F943D26B60181
:1051000083E596E10F94783D8F819885C2CFBF9259
:10511000CF92DF92EF92FF920F931F93CF93DF9383
:105120008B01F42EE90141FB662760F90E944226BB
:10513000882309F45AC0B12C0115110521F0C801CA
:105140000E94FAB9B82EE12C209721F0CE010E94DE
:10515000E5BBE82E80E8C82ED12CF0FE1EC085E10C
:1051600090E08B199109B7FC93958E199109E7FC92
:10517000939597FD019695958795F82E30E8C32E67
:10518000D12CFA94F7FC09C060E270E080E090E076
:105190000E942427C81AD90AF4CFBB2099F0C6016F
:1051A00066E070E00F944E59262F409131085091DF
:1051B000320860913008C8010E943AB996E0899F90
:1051C00060011124EE2031F0B601CE010E942928A1
:1051D000C81AD90A87E0C816D10438F060E270E036
:1051E00080E090E00E942427F3CFDF91CF911F91C0
:1051F0000F91FF90EF90DF90CF90BF9008956FEFE9
:105200007FEF0C942928AF92BF92CF92DF92EF925A
:10521000FF920F931F93CF93DF935C016B010E946A
:10522000FAB9E82EC6010E94E5BBF12C03E110E0BB
:10523000081B1109C5E20E151F050CF4CFE18C2FD8
:1052400090E09C012E5F3F4F409187164217130656
:1052500009F0CCF5099720918916281719069CF1B9
:1052600040913108509132086091300810928A16AE
:10527000C0938B1625E1C5010E943AB9D1E0C11453
:10528000D104B1F06AE370E080E090E00E9424274E
:105290000E151F05D4F4C45F80918716C81740F01F
:1052A000209189164C2F4950550B241715067CF474
:1052B000DF91CF911F910F91FF90EF90DF90CF90F2
:1052C000BF90AF900895D0E0DACFDD2389F3802F2F
:1052D000880F080F000F00938A16C0938B1660E2A8
:1052E00070E080E090E00E942427C601DF91CF911A
:1052F0001F910F91FF90EF90DF90CF90BF90AF90F4
:105300000C94FF288F929F92AF92BF92CF92DF9220
:10531000EF92FF920F931F93CF93DF93CDB7DEB73A
:105320002C970FB6F894DEBF0FBECDBF982F862FF7
:105330005A017901D02E692F0E944226882309F450
:1053400089C0C701002391F10E94FAB9C82E80904C
:105350005716909058168091FB04811145C01FEF9D
:1053600023E12C19409131085091320860913008A6
:10537000C5010E943AB9CC2009F46CC0B6E08B9FFD
:10538000500111246AE370E080E090E00E9424273D
:1053900057E0A516B10408F444C060E270E080E074
:1053A00090E00E942427A81AB90AF2CF0E94E5BB18
:1053B000C82E80905716909058168091FB04882331
:1053C00071F2FE0133968AE0DF011D928A95E9F7BA
:1053D00083E596E19A83898305EC11E29E012F5FB4
:1053E0003F4F49E451E212C0FE0133968AE0DF01EB
:1053F0001D928A95E9F783E596E19A83898305EC06
:1054000011E29E012F5F3F4F46E451E2B701C40114
:105410000F943D26B40183E596E10F94783D1F81FA
:105420009FCF40912F08212F30E0A6E0CA9EC001F7
:1054300011242E5F3F4F281739070CF49C0180E898
:10544000821B80938A1640938B16C701DD20A9F03A
:105450000E9425282C960FB6F894DEBF0FBECDBF54
:10546000DF91CF911F910F91FF90EF90DF90CF9040
:10547000BF90AF909F908F9008950E94FF28EACF31
:10548000EFE4F6E183AF64AFCA010C94FF282F92DA
:105490003F924F925F926F927F928F929F92AF92C4
:1054A000BF92CF92DF92EF92FF920F931F93CF9311
:1054B000DF93D62FC72FFC0180809180A280B3801C
:1054C000C501B40120E831E541E050E00F94D15826
:1054D000C9016DE671E00F944E596B017C01C50165
:1054E000B40120E13EE040E050E00F94D158CA0101
:1054F000B90128E130E040E050E00F94D158362E59
:10550000272E062F172F8CE3482E512C612C712C3F
:10551000C501B401A30192010F94D158B62EA72E54
:10552000CA01B901A30192010F94D158CB01C11452
:10553000D10479F1AF92BF927F936F932F923F92F4
:10554000FF92EF92DF92CF9285EF94E19F938F933A
:10555000CF93DF930F9424528DB79EB70E960FB65C
:10556000F8949EBF0FBE8DBF8D2F9C2FDF91CF91E2
:105570001F910F91FF90EF90DF90CF90BF90AF9071
:105580009F908F907F906F905F904F903F902F9063
:105590000895E114F104C9F0AF92BF927F936F9325
:1055A0002F923F92FF92EF9285EE94E19F938F931B
:1055B000CF93DF930F942452EDB7FEB73C960FB60E
:1055C000F894FEBF0FBEEDBFCFCF012BB9F0AF9265
:1055D000BF927F936F932F923F9289ED94E19F93B7
:1055E0008F93CF93DF930F9424528DB79EB70A9673
:1055F0000FB6F8949EBF0FBE8DBFB6CF892BA9F012
:10560000AF92BF927F936F9381ED94E19F938F93BD
:10561000CF93DF930F942452EDB7FEB738960FB6B1
:10562000F894FEBF0FBEEDBF9FCFAF92BF928DEC3F
:1056300094E19F938F93CF93DF930F9424520F9015
:105640000F900F900F900F900F908ECF8F929F9290
:10565000AF92BF92CF92DF92EF92FF920F931F9380
:10566000CF93DF931092F8041092F7042FE3209366
:10567000F6041092F5041092F4041092F3041092C0
:10568000EF041092F0041092F1041092F2049C01C5
:10569000F90190812F5F3F4F9032D1F39E34C9F4CE
:1056A000818190ED980F9A3020F08D3211F08B327D
:1056B00081F432969F012F5F3F4F808180538A3063
:1056C00008F47BC09F012F5F3F4F8081803209F437
:1056D00076C0F0935308E09352088F010F5F1F4F7D
:1056E000C0816AE270E0C8010F94CD5C009731F090
:1056F000FC01319780818032E1F31182CD3429F0B1
:10570000C43519F0C73409F04BC0F80180810F5F30
:105710001F4F8032D1F380538A3008F041C0C093CC
:10572000F60430E020E04AE0DF011196429FC0011C
:10573000439F900D11249C01205331098081280F33
:10574000311D87FD3A95818190ED980F9A30C8F10F
:105750003093F5042093F4048E3261F4329690E095
:105760004AE0DF0131968C9150ED580F5A3058F1D4
:105770009093F304CD01DC0101964C914032D9F3B2
:10578000CD3489F52E31310539F018F52731310541
:1057900019F02C31310539F5B093F804A093F704D2
:1057A000DF91CF911F910F91FF90EF90DF90CF90FD
:1057B000BF90AF909F908F900895F9017BCFF90132
:1057C00081CFFD01B1CF949F800D112490ED980FF2
:1057D000C8CF2537310538F027373105E8F2203AB0
:1057E00083E03807C9F2D091520840E050E0BA0196
:1057F00010E000E0C12CD12C7601C394FD0131965C
:105800008C91882309F47FC08132E1F4CD34D1F446
:1058100020323105B9F44093EF045093F0046093C3
:10582000F1047093F204F093F804E093F70463E258
:1058300070E0CF010F94CD5C009709F4B1CFFC016B
:105840001082AECF81548A3108F058C0DF019D919B
:10585000903291F0A0EDA90FAA30E8F09E3271F4D9
:10586000918190539A30B8F00115110519F48F0108
:105870000150110990E013C0FD01E8CF9D3211F0F5
:105880009B3291F79181A0EDA90FAA3020F09E32B2
:1058900059F79281E6CF9E2F9D1B309759F3A82F81
:1058A000B0E04601570104C0880C991CAA1CBB1C1F
:1058B0008A95D2F7482959296A297B29AB52BB4FCF
:1058C0009C9380818154DF018A3108F497CFDF01F6
:1058D0008191882309F492CF90ED980F9A30B8F314
:1058E00093ED980F923098F38B3289F3CD010196A6
:1058F000EC91E03209F082CFDC01F8CF01151105FF
:1059000001F78D01DECF1093F8040093F704409364
:10591000EF045093F0046093F1047093F20440CFCD
:105920009B01AC01485F5F4FBC016C5F7F4F0C94E3
:105930003B240F931F93CF93DF9300D000D01F928F
:105940001F92CDB7DEB7FC018B0183A5811112C078
:1059500081E083A784819581A681B781B05889832E
:105960009A83AB83BC83BE016F5F7F4F85E398E072
:105970000E94902C1D821E821F82188620E030E03B
:1059800040E05FE36091A5107091A6108091A71090
:105990009091A8100F947F5969837A838B839C839D
:1059A0009E012B5F3F4FAE014F5F5F4F61EA70E199
:1059B0008DE990E10E943B241D821E821F82188681
:1059C00020E030E040E05FE3F8016085718582858A
:1059D00093850F947F5969837A838B839C83B80165
:1059E0006C5F7F4F9E012B5F3F4FAE014F5F5F4F5C
:1059F000C8010E943B2428960FB6F894DEBF0FBE64
:105A0000CDBFDF91CF911F910F9108952F923F92BB
:105A10004F925F926F927F928F929F92AF92BF92BE
:105A2000CF92DF92EF92FF920F931F93CF93DF936A
:105A3000CDB7DEB7A2970FB6F894DEBF0FBECDBFCD
:105A40008C011B015E834D8340909D1050909E10F1
:105A500060909F107090A0108090A1109090A21064
:105A6000A090A310B090A410DB018D919D910D909A
:105A7000BC91A02D8F87988BA98BBA8B9C01AD010F
:105A8000C301B2010F947E596B017C01D1011496C0
:105A90008D919D910D90BC91A02D8B8B9C8BAD8B8E
:105AA000BE8B9C01AD01C501B4010F947E596F8B73
:105AB000788F898F9A8FAD81BE818D919D910D9048
:105AC000BC91A02D8F839887A987BA879C01AD01CF
:105AD000C301B2010F947E596B8F7C8F8D8F9E8F87
:105AE000AD81BE8114968D919D910D90BC91A02D9C
:105AF0008B879C87AD87BE879C01AD01C501B40132
:105B00000F947E596F8F78A389A39AA3A70196015A
:105B1000C701B6010F94F3526B017C012F89388DB8
:105B2000498D5A8DCA01B9010F94F3529B01AC0102
:105B3000C701B6010F947F594B015C012F8538894D
:105B400049895A896F81788589859A850F947E590C
:105B50002B013C012B893C894D895E896B857C85B5
:105B60008D859E850F947E596B017C01A301920166
:105B7000C301B2010F94F3522B013C01A70196011E
:105B8000C701B6010F94F3529B01AC01C301B201EE
:105B90000F947F590F942D5C6B017C012B8D3C8DF4
:105BA0004D8D5E8DCA01B9010F94F3522B013C015A
:105BB0002F8D38A149A15AA1CA01B9010F94F352FE
:105BC0009B01AC01C301B2010F947F599B01AC0151
:105BD000C501B4010F94DF5B1816B4F520E030E086
:105BE000A901C701B6010F94DF5B87FF2AC0C70177
:105BF000B601905820E030E040EA50E40F94DF5BBB
:105C0000181614F5A1016D817E81C8010E94062D30
:105C1000A2960FB6F894DEBF0FBECDBFDF91CF9135
:105C20001F910F91FF90EF90DF90CF90BF90AF90BA
:105C30009F908F907F906F905F904F903F902F90AC
:105C40000895C701B601D6CF20E030E040E050E42F
:105C5000C501B4010F94DF5B181624F4B101C8012B
:105C60000E94992C19821A821B821C82BE016F5FCE
:105C70007F4FC1010E94902C2DEC3CEC4CEC5CE37E
:105C8000C701B6010F94F3529B01AC01F80160818A
:105C90007181828193810F94F35269837A838B831C
:105CA0009C83C8010F946F2EBE016F5F7F4F8D8163
:105CB0009E810E94902CACCF4F925F926F927F9208
:105CC0009F92AF92BF92CF92DF92EF92FF920F938B
:105CD0001F93CF93DF93CDB7DEB768970FB6F894D5
:105CE000DEBF0FBECDBFFB019080342F390D3530A4
:105CF00008F026C1E180022F0E0D053008F020C10A
:105D0000EE2DF0E0EA54FB4F4080512C712C612CB9
:105D1000092C04C076946794579447940A94D2F758
:105D200040FE0EC110E0F801EA54FB4F4080512CB8
:105D3000712C612CC32ED12C04C076946794579497
:105D400047943A95D2F740FEFBC0F22E642F5C01D7
:105D5000660F770B072E000C880B990B0F9494524B
:105D60002B013C01892D94E08902F0011124EE55AC
:105D7000F94EA301920160817181828193810F9418
:105D80007F596D877E878F87988BF601EE0FFF1FF7
:105D9000EE0FFF1FEE55F94EA30192016081718154
:105DA000828193810F947E5969837A838B839C834C
:105DB0006F2D660F770B072E000C880B990B0F9435
:105DC00094522B013C018E2D94E08902F0011124A4
:105DD000E257F94EA3019201608171818281938122
:105DE0000F947F59698B7A8B8B8B9C8B000F111FC3
:105DF000000F111FF801E257F94EA30192016081D3
:105E00007181828193810F947E596D837E838F830C
:105E10009887F50180859185A285B38589879A87C2
:105E2000AB87BC878D8B9E8BAF8BB88F4FEE50E0CE
:105E300061E070E0CE0141960E94FCD54FEE50E04B
:105E400061E070E0CE0105960E94FCD54FEE50E077
:105E500061E070E0CE010D960E94FCD54FEE50E05F
:105E600061E070E0CE0101960E94FCD5C988DA8815
:105E7000EB88FC8827E137EB41ED58EBC701B60111
:105E80000F94DF5B87FD5CC027E030E040E753E420
:105E9000C701B6010F948D5218160CF451C0CD8471
:105EA000DE84EF84F88827E137EB41ED58EBC7013A
:105EB000B6010F94DF5B87FD43C027E030E040E789
:105EC00053E4C701B6010F948D521816CCF1CD8062
:105ED000DE80EF80F88427E137EB41ED58EBC70116
:105EE000B6010F94DF5B87FD2BC027E030E040E771
:105EF00053E4C701B6010F948D5218160CF1C980F6
:105F0000DA80EB80FC8027E137EB41ED58EBC701ED
:105F1000B6010F94DF5B87FD13C027E030E040E758
:105F200053E4C701B6010F948D5218164CF0AE0120
:105F30004F5F5F4FBE01635F7F4FC5010E94062D1B
:105F400068960FB6F894DEBF0FBECDBFDF91CF913C
:105F50001F910F91FF90EF90DF90CF90BF90AF9087
:105F60009F907F906F905F904F9008958C3891052F
:105F700014F08CE890E090937208809371080C9470
:105F800051C60E94812597FD0CC00E9481256F3F5C
:105F900071058105910509F034F40E948125862F51
:105FA000089580E008958FEF08958091BF04909147
:105FB000C004892B41F00E94C12F91E0811101C0E2
:105FC00090E0892F089591E0FCCF0E948125CB01BC
:105FD00008950F931F93CF938091BF049091C004B5
:105FE0000097E9F0FC018F01C1912C2F2F7D81F0EA
:105FF000C53411F0C536B9F7F801108270E060E0E1
:106000000F941C4EF801C083CF911F910F910895FA
:1060100070E060E0CF911F910F910D941C4E60E0F5
:1060200070E0CB01F1CF2FEB280F2A3108F047C0E9
:10603000E22FF0E08091EF049091F004A091F10440
:10604000B091F20404C0B695A795979587952A95C7
:10605000D2F780FD02C081700895EB52FB4FE081C2
:10606000EE2341F18091520890915308E80FF92FE7
:10607000F11D808190ED980F9A3030F08E3251F4FE
:10608000818180538A3098F4F093C004E093BF0478
:1060900081E008958D3211F08B3249F4818190EDC9
:1060A000980F9A3088F38E3211F48281EACFF0E0B3
:1060B000E0E0EACF1092C0041092BF04E9CF80E084
:1060C00008950E941330882341F081E02091BF049D
:1060D0003091C004232B09F480E00895CF93DF931F
:1060E000EB010E946130882319F00E948125EB01A9
:1060F000CE01DF91CF910895CF92DF92EF92FF9280
:106100006A017B010E946130882331F0FF90EF909B
:10611000DF90CF900C94E92FC701B601FF90EF906C
:10612000DF90CF9008954F925F926F927F928F92FF
:106130009F92AF92BF92CF92DF92EF92FF921F9306
:10614000CF93DF9300D01F92CDB7DEB719821A82AA
:106150001B821C82CE0101964C018DE9C82E80E184
:10616000D82E95E3E92E98E0F92E2FE4A22E29E00F
:10617000B22E10E088E5810F0E946130F401819316
:106180004F01882341F00E94E92F2B013C018091AF
:106190005210882359F0F60180819181A281B38148
:1061A000F70180839183A283B38314C0812F0E945F
:1061B000A621882309F4D0C0F601208131814281D3
:1061C0005381C301B2010F947F59F701608371833A
:1061D000828393831F5FF4E0CF0ED11C84E0E80E2E
:1061E000F11C94E0A90EB11C133021F685E40E9445
:1061F00061308C83882309F4B9C00E94E92F6B01B8
:106200007C0183E00E94A621882371F02091A910CF
:106210003091AA104091AB105091AC10C701B6015B
:106220000F947F596B017C01C0924108D0924208C3
:10623000E0924308F09244088091CE05882359F1FA
:106240008091C11682FF27C08C81882321F189812A
:10625000811103C08A818823F1F02DEC3CEC4CE4E1
:106260005DE36091A6087091A7088091A8089091BD
:10627000A9080F947F599B01AC016091A510709102
:10628000A6108091A7109091A8100F94DF5B1816AC
:1062900014F40F94D23F40E050E0BA0186E40E942B
:1062A0007C3020E030E0A9010F94DF5B181684F405
:1062B0000E94E92F20E030E040E752E40F94795A41
:1062C0006093790270937A0280937B0290937C02B0
:1062D0008091531083FD2CC080915210811128C0F1
:1062E0008091AF07882321F12091A9103091AA1045
:1062F0004091AB105091AC106091410870914208F0
:1063000080914308909144080F947E592091BC07D6
:106310003091BD074091BE075091BF070F947F5940
:106320006093BC077093BD078093BE079093BF072F
:106330000F900F900F900F90DF91CF911F91FF90D2
:10634000EF90DF90CF90BF90AF909F908F907F9015
:106350006F905F904F900895F501208131814281C7
:106360005381C301B2010F947E592FCF8091A910A0
:106370009091AA10A091AB10B091AC1080934108FD
:1063800090934208A0934308B093440855CFCF930D
:10639000DF93EB010E946130882321F0DF91CF91E0
:1063A0000C94E52FCE01DF91CF910895CF93DF9329
:1063B000C82FD62F0E946130882321F0DF91CF9122
:1063C0000C94D52F8C2F0E941330811101C08D2F7A
:1063D000DF91CF910895EDE9F8E082EBDF011D92A6
:1063E0008A95E9F708958091CE05811104C00E9435
:1063F000EB310D9497418091C11682FD0D94D23FEF
:10640000089580919D08882361F090914E09891329
:1064100008C08091C11683FF04C08BED98E00D94F5
:10642000A24180E00895FC01238121110C9416D231
:106430000895CF92DF92EF92FF920F931F93CF9325
:1064400090912402913009F461C0662351F01092BA
:10645000A20410929E0410929F041092A004109225
:10646000A104C82F0F945335C0909E04D0909F0470
:10647000E090A004F090A1049B01AC012C193D090F
:106480004E095F0969017A01F7FC40C02091A2041E
:10649000C7FD15C04C2F0C2E000C550B4C5F5F4FE9
:1064A000E22F022E000CFF0B4E175F077CF144EF2A
:1064B000C42EDD24D394E12CF12C2C1734F438EEC7
:1064C000C32E33E0D32EE12CF12CC60ED71EE81ECE
:1064D000F91EC0929E04D0929F04E092A004F09214
:1064E000A104022F017010E084E2809FB001819F1F
:1064F000700D701B112460597C4F82E390E00E9464
:106500002E7D8091A2048F5F8093A204CF911F9172
:106510000F91FF90EF90DF90CF9008950F931F930E
:1065200001E010E020E030E0082E04C0000F111F51
:10653000221F331F0A94D2F740910305509104059E
:106540006091050570910605402B512B622B732B32
:106550004093030550930405609305057093060569
:1065600090912302891303C081E0809352101F9100
:106570000F9108951092330610923406109235064A
:1065800010923606EFECF5E084E6DF011D928A9565
:10659000E9F7089590919C109817B1F00E94D6DC0D
:1065A00080919C10882341F08DE990E10E94F9DCF4
:1065B00010929C100C9471F281E080939C108DE9F4
:1065C00090E10E942BDCF6CF08954F925F926F927C
:1065D0007F928F929F92AF92BF92CF92DF92EF9273
:1065E000FF921F93CF93DF93EC01162F2091670842
:1065F000309168084091690850916A0868817981F2
:106600008A819B810F948D52882309F4AEC0B0908B
:106610009C1080E00E94CA32C880D980EA80FB804A
:1066200020E030E0A901C701B6010F94DF5B181626
:106630001CF0C12CD12C7601C0926708D09268085A
:10664000E0926908F0926A082DEB37E346E855EBD3
:10665000C701B6010F94DF5B87FD0BC02DEB37E35D
:1066600046E855E3C701B6010F948D5218160CF099
:1066700078C0A701960160E070E080E89FE30F9486
:10668000795A6093B2057093B3058093B4059093E3
:10669000B50580EF9FEFA9E7B4EC8093B605909322
:1066A000B705A093B805B093B905BB2009F45DC048
:1066B00040909D1050909E1060909F107090A01080
:1066C0008090A1109090A210A090A310B090A41060
:1066D000C090A510D090A610E090A710F090A81040
:1066E00081E00E94CA32112309F43FC020919D101D
:1066F00030919E1040919F105091A010C301B201A3
:106700000F948D5281111CC02091A1103091A210C4
:106710004091A3105091A410C501B4010F948D5263
:1067200081110EC02091A5103091A6104091A710A4
:106730005091A810C701B6010F948D528823A9F07B
:10674000DF91CF911F91FF90EF90DF90CF90BF909E
:10675000AF909F908F907F906F905F904F900C9430
:1067600019FB60E070E0CB018CCFDF91CF911F91DE
:10677000FF90EF90DF90CF90BF90AF909F908F9061
:106780007F906F905F904F900895EF92FF920F93DC
:106790001F93CF93DF930FEC15E0C5E07801D5E0B0
:1067A000F70161917191819191917F0120E030E039
:1067B000A9010F948D5281110EC0D15089F7C1509B
:1067C0000C5E1F4FC111EACFDF91CF911F910F9146
:1067D000FF90EF90089581E0F7CFEFE6F0E0808141
:1067E0008260808308958091490890914A08892B9E
:1067F00079F48091490890914A08892B49F42091B5
:10680000490830914A0881E0232B19F480E008956B
:1068100081E00895CF92DF92EF92FF926B017C01AD
:1068200083E3C816D104E104F10470F082E3C81ACE
:10683000D108E108F10862E370E080E090E00F9495
:1068400020350E9473F2ECCFC701B6010F942035BA
:10685000FF90EF90DF90CF900C9473F280914E06F2
:1068600081110AC080916508813041F08091C11684
:1068700082FB882780F9089580E0089581E00895DB
:106880005F9A8091C3078E7F8093C3078A9A809115
:10689000C3078D7F8093C307809108018095817025
:1068A000809306018091C3078B7F8093C3070C946C
:1068B000C0219091C11693FB882780F993FF06C0F1
:1068C00081E090912918911101C080E00895809194
:1068D0004E06811110C080916508823061F00E94DF
:1068E0005934882349F08091C11682FB882780F9AA
:1068F00091E08927089581E008950E94673481110D
:106900000DC0109203051092040510920505109217
:106910000605109207058FEF0E94C2230C9456FEC5
:10692000EDE8F9E010821182089581E008958F92D8
:106930009F92AF92BF92CF92DF92EF92FF920F930E
:10694000CF93DF931F92CDB7DEB75C017B01490186
:106950006B01C40ED51EF501808191810F94AB5857
:106960008983002311F0F7018083BE016F5F7F4FA1
:10697000C4010F946325F501808191810196918373
:106980008083FFEFEF1AFF0AEC14FD0421F780E08B
:106990000F90DF91CF910F91FF90EF90DF90CF900C
:1069A000BF90AF909F908F9008959091C00095FFF9
:1069B000FCCF8093C6000895CF93DF93EC018991BB
:1069C000882319F00E94D534FACF8DE00E94D53487
:1069D0008AE0DF91CF910C94D534CF92DF92EF9281
:1069E000FF92CF936B017C01C42F4A3069F4F7FE0C
:1069F0000BC0F094E094D094C094C11CD11CE11C55
:106A0000F11C8DE20E94D5344C2FC701B601CF9105
:106A1000FF90EF90DF90CF900D94343FCF93DF93B2
:106A2000EC01FE0184912196882319F00E94D5344F
:106A3000F8CFDF91CF9108950F931F93CF938C01DF
:106A4000C62F85E392E10E940E35C8010E940E35E3
:106A50008AE30E94D53480E38C0F0E94D5348AE00B
:106A6000CF911F910F910C94D53488EB93E10E9444
:106A70000E3560E088EA93E10E941C3560E083E90E
:106A800093E10E941C3561E08CE893E10E941C3583
:106A900061E081E893E10E941C3561E081E793E1C8
:106AA0000E941C3560E088E693E10E941C3561E09D
:106AB0008EE593E10E941C3560E084E593E10E943D
:106AC0001C3560E08DE493E10E941C3560E085E4B4
:106AD00093E10E941C3561E087E393E10E941C353D
:106AE00061E089E293E10E941C3560E08AE193E174
:106AF0000E941C3560E08CE093E10E941C3560E050
:106B000086EF92E10E941C3561E085EE92E10E94E1
:106B10001C3561E086ED92E10E941C3561E08FEC4E
:106B200092E10E941C3560E088EC92E10E941C35E5
:106B300061E08FEB92E10E941C3561E08AEA92E10C
:106B40000E941C3561E08CE992E10E941C3561E0F5
:106B500089E892E10E941C3560E08CE792E10E9496
:106B60001C3561E087E792E10E941C3561E08AE60E
:106B700092E10E941C3560E086E592E10E941C359E
:106B800060E083E492E10E941C3560E085EC96E1D0
:106B90000E94A321682F61708AE392E10C941C3556
:106BA0000E94D53485EF9CE00C940E350F931F9313
:106BB000CF938C01C62F84E799E00E940E35C8015F
:106BC0000E940E35CC2331F08AE0CF911F910F91B6
:106BD0000C94D534CF911F910F91089560E083E418
:106BE00090E40E94D63584E899E00E940E358AE050
:106BF0000C94D534EF92FF920F931F93CF937C01A7
:106C00008B01C42F60E083E490E40E94D635C70175
:106C10000E940E3580E20E94D534C8010E940E35D4
:106C2000CC2319F08C2F0E94D5348AE0CF911F918C
:106C30000F91FF90EF900C94D534DF92EF92FF927A
:106C40000F931F93CF93DF93D82E7B018A01E90125
:106C50000E94EE35D0924D0840E0B70187E590E400
:106C60000E94FA350115110531F040E0B80180E5C8
:106C700090E40E94FA35209731F040E0BE0180E5B3
:106C800090E40E94FA3560E083E490E40E94D635F7
:106C90008BE490E40E940E358AE0DF91CF911F9142
:106CA0000F91FF90EF90DF900C94D53461E08EE768
:106CB00099E00C94D635AF92BF92CF92DF92EF92CB
:106CC000FF920F931F93CF93DF9389E499E00E9483
:106CD0000E3560913306709134068091350690919F
:106CE000360645E00F949C0786E399E00E940E3536
:106CF000C0E0D9E0D15021F080E20E94D534FACF33
:106D00008C2F0F949B3FCF5FC53099F78AE00E948C
:106D1000D5340FEC15E0C0E080E20E94D5348C2F12
:106D20000F949B3F5801D5E080E20E94D534F501D5
:106D3000C080D180E280F380A7019601C701B6012F
:106D40000F94715C81112CC020E030E0A901C701D3
:106D5000B6010F94DF5B87FD03C08BE20E94D53440
:106D600045E0C701B6010F949C07D15084E1A80EFD
:106D7000B11CD111D9CF8AE00E94D534CF5F0C5F0E
:106D80001F4FC53049F68AE0DF91CF911F910F91D7
:106D9000FF90EF90DF90CF90BF90AF900C94D534E0
:106DA000F12C80E20E94D534F3948DE3F8E0FF12D9
:106DB000F9CFDBCF811107C083E39EE00E940E353F
:106DC0008AE00C94D53487E39EE0F8CFCF93DF932D
:106DD000EB010E940E35CE01DF91CF910D94A23FC1
:106DE000CF93C62F0E940E358C2FCF910D949B3FD1
:106DF000CF92DF92EF92FF926A017B010E940E35E3
:106E000042E0C701B601FF90EF90DF90CF900D9464
:106E10009C07CF92DF92EF92FF926A017B010E9462
:106E20000E354AE0C701B601FF90EF90DF90CF909A
:106E30000C94ED342F923F924F925F926F927F921B
:106E40008F929F92AF92BF92CF92DF92EF92FF927A
:106E50000F931F93CF93DF93CDB7DEB7C654D109FD
:106E60000FB6F894DEBF0FBECDBF70E060E085E4E2
:106E70000E94C731182F8F3F09F483C08823E9F09F
:106E800083E796E1CA5BDF4F0FB6F894DEBF0FBE13
:106E9000CDBFDF91CF911F910F91FF90EF90DF90C9
:106EA000CF90BF90AF909F908F907F906F905F90AA
:106EB0004F903F902F900C940E3524EB30E03A83A6
:106EC000298383E50E946130882321F00E94E52F09
:106ED0009A83898365E070E083E40E94C7318AA7C2
:106EE00060E085E50E94D63125968FAF259760E05A
:106EF00086E696E10E9464B2A981BA81BD01BB0F0A
:106F0000880B990B0F9494526D837E838F83279601
:106F10009FAF27970F945335688B798B8A8B9B8B08
:106F20001F3F09F045C420E030E04CE053E46D81A0
:106F30007E818F8127969FAD27970F94DF5B181670
:106F40000CF0AAC18BE396E10E940E35CA5BDF4FBD
:106F50000FB6F894DEBF0FBECDBFDF91CF911F916A
:106F60000F91FF90EF90DF90CF90BF90AF909F90E8
:106F70008F907F906F905F904F903F902F900D94E7
:106F8000924246E450E05A8349839BCF1FAEAFC183
:106F90002496EEADFFAD2497808383C2FBEE4F2E87
:106FA000512C612C712C04C384E190E0A0E0B0E08E
:106FB0008C8B9D8BAE8BBF8BE4E14E2E512C612CC4
:106FC000712C04C34C8A5D8A6E8A7F8AFFC2249624
:106FD000EEADFFAD24978083D4C389819A81AB81C4
:106FE000BC8129A93AA94BA95CA9821B930BA40BCC
:106FF000B50BB7FD59C08FAD0F9440088AE00E94D1
:10700000D53489819A81AB81BC818053984FAF4F31
:10701000BF4F89AB9AABABABBCAB9DA9911177C00D
:107020002EA93FA948AD59ADB101802F26969FAD3D
:1070300026970F94DF5B18160CF053C020E030E069
:1070400040E050E4B101802F26969FAD26970F9423
:107050007F596EAB7FAB88AF99AF2CA53DA54EA5F0
:107060005FA589819A81AB81BC81280F391F4A1F96
:107070005B1F2AAF3BAF4CAF5DAF20E030E040EC90
:1070800050E46D817E818F8127969FAD27970F9465
:107090007E599101402F26965FAD26970F948D5211
:1070A000881F8827881F8DAB88899989AA89BB8901
:1070B000C816D906EA06FB0610F4D701C6012981D5
:1070C0003A814B815C81281B390B4A0B5B0BDA013F
:1070D000C90181389F44A241B105A8F187E895E133
:1070E0000EC289819A81AB81BC812AAD3BAD4CAD8A
:1070F0005DAD821B930BA40BB50B48E156E367E231
:1071000076E3B7FDD1CF812F0E943ED6CDCF20E0D0
:1071100030E040EF51E46D817E818F8127969FADF5
:1071200027970F947E599B01AC01B101802F2696C1
:107130009FAD26970F948D5287FFB6CF44EC56E350
:1071400064ED76E3E0CF4AA55BA5888D998D48175D
:1071500059070CF09EC003970CF49BC08AE295E19E
:107160000E940E351F3F09F076C0AAE1B5E1BA834F
:10717000A98389E095E10E940E3589819A810E9458
:107180000E35488559856A857B8586E295E10E94A2
:10719000F8368AE00E94D53489E095E10E940E35E8
:1071A00089819A810E940E3549A15AA16BA17CA1C7
:1071B00082E295E10E94F8368AE00E94D53489E0A7
:1071C00095E10E940E3589819A810E940E35B501A4
:1071D000A4018EE195E10E94F8368AE00E94D53440
:1071E0002596FFAD2597FF2391F12CEA35EC47E278
:1071F0005EE369A17AA18BA19CA10F94F3526B016C
:107200007C012CEA35EC47E25EE3C501B4010F9442
:10721000795A288539854A855B851F3F09F5209372
:107220007408309375084093760850937708C0929D
:107230007808D0927908E0927A08F0927B086093FF
:107240007C0870937D0880937E0890937F0881E08E
:10725000809362027BCEEDE8FFE3FA83E98389CF76
:107260002093D8153093D9154093DA155093DB1538
:10727000C092DC15D092DD15E092DE15F092DF159C
:107280006093E0157093E1158093E2159093E315F8
:10729000DECF0E946EB680C087E296E10E940E3576
:1072A0000E9431D58FE78093730824EB30E0A8EE7D
:1072B000B3E00F9425596CA77DA78EA79FA72889B7
:1072C00039894A895B89260F371F481F591F2AAF02
:1072D0003BAF4CAF5DAF1092620281E080937102D0
:1072E00032E0310F3EAF323008F450CE1FAFC888C5
:1072F000D988EA88FB88C9AADAAAEBAAFCAA812C59
:10730000912C540189A29AA2ABA2BCA2888699862C
:10731000AA86BB868FE790E0A0E0B0E08C8B9D8BC7
:10732000AE8BBF8B1C8690E49A8FACE1AB8FB6E43A
:10733000BC8F1D8E1E8E1F8E18A23FE7432E512C30
:10734000612C712C1DAA8EAA9FAAA8AEB9AE1EA24E
:107350001FA218A619A6E1E0EDA3198E188E212C04
:10736000312C00E026961FAE2697F5E11F02C001E2
:1073700011249C0121533A4E22963FAF2EAF229703
:10738000285F3F4F24963FAF2EAF24974AA5042E87
:10739000000C550B5BA74AA780917102882309F462
:1073A000B0C00F94533569837A838B839C8350914B
:1073B0004C0658AB552309F48BC00E94E4D560916C
:1073C0006F08709170081F3F39F02296AEADBFADC7
:1073D000229714966D917C91072E000C880B990BC7
:1073E0000F9494521B01082F26969FAF26972D8D40
:1073F0003E8D4F8D58A126969FAD26970F94DF5B4B
:1074000018163CF42D8E3E8E0F8F2696BFAD269714
:10741000B8A32C853A8D4B8D5C8DB101802F2696BB
:107420009FAD26970F948D5287FF07C02C863A8E0A
:107430000B8F2696EFAD2697EC8FFDA19101402F83
:1074400026965FAD26976D817E818F8127969FADB1
:107450002797FF2309F45AC00F948D5287FF38C035
:1074600049815A816B817C814C195D096E097F09C4
:10747000DB01CA0188589341A109B109B7FD28C0B1
:107480008C899D89AE89BF8984199509A609B70998
:10749000B595A795979587951F3F09F079CD80936E
:1074A00073084EA35FA368A779A7FD81FD8F2E8186
:1074B0002E8F3F813F8F27964FAD279748A3898115
:1074C0009A81AB81BC81888B998BAA8BBB8B1DA2C7
:1074D00020E030E040EF51E46D817E818F8127967E
:1074E0009FAD27970F947F599101402F26965FAD4E
:1074F00026970F948D5287FF70CD85EA95E10E9403
:107500000E35109271020E9431D5A1CE0F94DF5B2F
:107510001816F4F689819A81AB81BC812889398952
:107520004A895B89821B930BA40BB50BAC01BD018F
:10753000485853416109710977FDCACF488D598D6B
:10754000452B09F40DC1CEA0DFA0E8A4F9A4C80E14
:10755000D91EEA1EFB1E2EA13FA148A559A5281B36
:10756000390B4A0B5B0BC301B2010F94C158A70141
:1075700096010F94F3584C885D886E887F88420E80
:10758000531E641E751E54E14516510461047104B6
:107590000CF40ACD8CEE48165104610471040CF011
:1075A000FDCC90E849165104610471040CF40ACD35
:1075B0004C8A5D8A6E8A7F8A2EEF30E040E050E090
:1075C000241935094609570929013A014C895D8971
:1075D0006E897F898FE196E10E940937B301A2018C
:1075E0008AE196E10E9409374C855A8D6B8D7C8D1E
:1075F00083E196E10E94F8364D8D5E8D6F8D78A106
:107600008CE096E10E94F836A88DB98D13970CF4A2
:10761000A7C0C301B2010F94945220E030E040E8CB
:1076200050E40F94F3524B015C012C853A8D4B8D45
:107630005C8D6D8D7E8D8F8D98A10F947E592BED75
:107640003FE049E450E40F94F35220E030E040E0A2
:107650005FE30F94F3529B01AC01C501B4010F9499
:10766000795A6C877D878E879F87C701B6010F94F3
:1076700094522FE632E143E85AE30F94F3526B0140
:107680007C011E3F59F02AE939E949E15FE3812C89
:10769000912CA12C6EE3B62E1F3F59F42DEC3CEC3F
:1076A0004CE45EE37BEA872E7AEA972EA92C7EE3F0
:1076B000B72E6C857D858E859F850F94F3526887E4
:1076C00079878A879B879B01AC010F947F59A7011B
:1076D00096010F94795A69A37AA38BA39CA328855A
:1076E00039854A855B85C701B6010F94F352A50120
:1076F00094010F94F3524B015C014C855D856E85BE
:107700007F8586E096E10E94F836B701A60180E009
:1077100096E10E94F8368AE00E94D534BEAD81EF32
:1077200095E1B23010F082EE95E10E940E35488569
:1077300059856A857B858CED95E10E94F83649A1D3
:107740005AA16BA17CA186ED95E10E94F836B501A6
:10775000A40180ED95E10E94F8368AE00E94D534BC
:107760008C899D89AE89BF89840D951DA61DB71D85
:10777000B595A795979587951F3F09F028CC8093DD
:107780007308288D398D2F5F3F4F398F288F3D81AA
:107790003C874E814A8F5F815B8F27968FAD2797FD
:1077A0008C8FC980DA80EB80FC8098A99DA390CE55
:1077B000E12E012E000CFF08F70183E0EE0FFF1F02
:1077C0008A95E1F7E759FD4F668177816F5071091E
:1077D000072E000C880B990B0F9494529B01AC015F
:1077E0006D817E818F8127969FAD27970F94DF5BF8
:1077F00018160CF4A7CB87E296E10E940E350E9482
:1078000031D585E18E9DF0018F9DF00D1124E1535E
:10781000FA4E8FE7808722E330E049CDCF93DF93A4
:10782000EB010E940E35CE01DF91CF910D941A2706
:107830002F923F924F925F926F927F928F929F9280
:10784000AF92BF92CF92DF92EF92FF920F931F936E
:10785000CF93DF93CDB7DEB7C058D1090FB6F894F8
:10786000DEBF0FBECDBF80E89CE00E940E350F94B6
:10787000B44281118FC084E50E946130882329F0D1
:107880000E94E52F81110E94E7D480E090E0A0E8FB
:10789000BFE389839A83AB83BC838D839E83AF834D
:1078A000B8878DEC9CECACE4BEE389879A87AB8704
:1078B000BC8780E090E0A0E2B1E48D879E87AF872F
:1078C000B88B8CE390E09A8B898B8DEC90E09C8B4D
:1078D0008B8B8DEC9CECACECBEE38D8B9E8BAF8BDD
:1078E000B88F80E090E0A0EEBFE3898F9A8FAB8FD6
:1078F000BC8F1BA61CA64AE959E969E97EE38FE41F
:107900000E947C306D8F7E8F8F8F98A360E083E420
:107910000E94D63189A360E08BE40E94D6318AA30D
:1079200089E40E94613010E0F12CE12C8823C1F041
:107930000E94C12F90E01816190614F481E090E01F
:1079400011E0180F212F2150330BC90126E0289F89
:10795000F001299FF00D1124E75FF74FE280F380DB
:1079600082E40E946130882319F00E94E52F7C0197
:10797000E114F10459F1C70188978536910520F18A
:107980006CE870E082E59CE00E940E3C8DE49CE097
:107990000E940E35C058DF4F0FB6F894DEBF0FBE01
:1079A000CDBFDF91CF911F910F91FF90EF90DF90AE
:1079B000CF90BF90AF909F908F907F906F905F908F
:1079C0004F903F902F900895FA8AE98A8CE40E94A4
:1079D00061308823E1F00E94E92F6B017C01C986A8
:1079E000DA86EB86FC8620E030E0A9010F94DF5BAD
:1079F00087FD0AC020E030E040E050E4C701B60156
:107A00000F948D5218161CF485E29CE0C1CF81E5DD
:107A10000E941330882331F18091BF049091C004FB
:107A2000892BE9F00E94E92F6B017C01CD82DE8277
:107A3000EF82F8862DEC3CEC4CE45DE30F94DF5BC9
:107A400087FD0AC020E030E040E751E4C701B601FD
:107A50000F948D52181634F484EF9BE099CF89EC83
:107A60009BE096CF83E50E9461308823E9F00E9475
:107A7000E92F6B017C01CD8ADE8AEF8AF88E2DEC2E
:107A80003CEC4CEC5DE30F94DF5B87FD0AC020E02B
:107A900030E040E050E4C701B6010F948D52181653
:107AA0001CF482EA9BE074CF80E50E9413308823A7
:107AB00041F08091BF049091C004892B29F58FEF8C
:107AC0008BA786E40E946130882309F43DC00E94A0
:107AD000E92F6B017C01C98EDA8EEB8EFC8E20E0E3
:107AE00030E040E85FE30F94DF5B87FD0AC020E0F1
:107AF00030E040E850E4C701B6010F948D521816EB
:107B00001CF581E59BE044CF8BA58F5F8BA70E947E
:107B1000E92F6B017C01CD86DE86EF86F88A20E0B6
:107B200030E0A9010F94DF5B87FD0BC020E030E05F
:107B300048EC51E4C701B6010F948D5218160CF0B1
:107B4000C0CF8AE79BE024CFC98CDA8CEB8CFC8C0D
:107B50008D889E88AF88B88CA7019601C701B601B1
:107B60000F94F3529B01AC0160E070E084E490E478
:107B70000F94795A29813A814B815C810F94F35299
:107B80002B013C01A5019401C501B4010F94F352EE
:107B9000A70196010F94F3522CEE31E548EB5DE31B
:107BA0000F94795A9B01AC01C301B2010F94F352B7
:107BB00069837A838B839C83112309F1412F415080
:107BC000550B26E0249FF001259FF00D1124E75F5F
:107BD000F74F0081118188E40E946130882319F0F9
:107BE0000E94E52F8C010115110571F0C801855A1D
:107BF00091098838910530F083E29BE0C9CE10E00E
:107C000000E0E9CF1C8B0B8B85E50E9413308823A5
:107C1000C9F00F945335611571058105910511F077
:107C20000F94134E8091BF049091C004892BC9F02A
:107C30000E94E92F6093BB047093BC048093BD0441
:107C40009093BE046AE170E082E50E94C731E59638
:107C50009FAF8EAFE5971816190644F08FEE9AE0A5
:107C600097CE60E070E088E492E4E4CF89E50E947A
:107C70006130882309F40AC10E94E92F2091530939
:107C80003091540940915509509156090F947E59ED
:107C90004B015C0188E50E946130882309F4FFC034
:107CA0000E94E92F20914F093091500940915109CC
:107CB000509152090F947E596B017C01CBA2DCA23A
:107CC000EDA2FEA28FA298A6A9A6BAA627E137EB3D
:107CD00041ED58EBC501B4010F94DF5B87FDE8C0AF
:107CE00027E030E040E753E4C501B4010F948D5222
:107CF00018160CF4DDC027E137EB41ED58EBC70156
:107D0000B6010F94DF5B87FDD3C027E030E040E78A
:107D100053E4C701B6010F948D5218160CF4C8C075
:107D200084E40E94133011E081270E94CA3280E06F
:107D300090E0A0EAB0E48DA79EA7AFA7B8ABCE01B4
:107D40008D960F94142E50918408EC965FAFEC97AB
:107D5000109284080E94D1C382E79AE00E940E35F7
:107D600089899A894A970CF0A6C063E68FE49AE065
:107D70000E9464B20F948C358B899C890E9458DCD8
:107D800041E061E080E00F94380A882309F4A6C03E
:107D90000F9492420F948C351092A9101092AA1051
:107DA0001092AB101092AC1089EA90E10E9470EE34
:107DB0001BA5112309F4F5C020E030E040E751E4B1
:107DC0006091841070918510809186109091871039
:107DD0000F94795A21966CAF7DAF8EAF9FAF2197EC
:107DE0001F3F09F0F9C481E08093000563E687EA4C
:107DF0009AE00E9464B268E873E182E090E00E9439
:107E00002E7D80E1EDE9F0E1A5E3B8E001900D926F
:107E10008A95E1F7CE0101960F946F2EC12CD12CDB
:107E2000760180915F0982FDB1C068E873E182E06C
:107E300090E00E942E7D20E030E040E85EE360911B
:107E400041087091420880914308909144080F9432
:107E50007F59609341087093420880934308909340
:107E6000440820E030E040E85EE3C701B6010F942B
:107E70007F596B017C0120E030E84BE354E40F9420
:107E8000DF5B87FD73C01092000528C08090A110B1
:107E90009090A210A090A310B090A410FBCEC09020
:107EA0009D10D0909E10E0909F10F090A01006CFF3
:107EB00085EC9AE06DCD63E682E69AE00E9464B2BA
:107EC0000F948C351093000589899A890E94B62FEA
:107ED00061E081E00F94B308811147CF6FEF89EB28
:107EE0009AE00E9464B28CA5811112C081E08CA737
:107EF0008D819E81AF81B885B0588DA79EA7AFA711
:107F0000B8ABBE01635D7F4F85E398E00E94902C83
:107F100080E090E0A0EAB0E480933D0890933E08B2
:107F2000A0933F08B09340081DA61EA61FA618AA3E
:107F3000BE01635D7F4F85E398E00E94902CEC9634
:107F40005FADEC97509384080E94D1C31092000556
:107F50008AA181111FCD10927208109271080E949F
:107F600051C690E080E00E9458DC14CDCE01CD9641
:107F70000E9461F980E1EDE9F0E1A5E3B8E001904C
:107F80000D928A95E1F70E94D6DC4BCF0E9429B969
:107F900063E68AE99AE00E9464B20F948C351092ED
:107FA0000005E6EBF4E085E0DF011D928A95E9F734
:107FB00080E1EDE9F0E1A5E3B8E001900D928A954A
:107FC000E1F789859A85AB85BC8580933D089093C0
:107FD0003E08A0933F08B09340081DA61EA61FA60A
:107FE00018AABE01635D7F4F85E398E00E94902C44
:107FF000BE01635E7F4F85E398E00E94902C81E094
:108000008093000589A1882309F43CC420919D1028
:1080100030919E1040919F105091A010AC962CAFC3
:108020003DAF4EAF5FAFAC978091A1109091A21081
:10803000A091A310B091A410E0968CAF9DAFAEAF0D
:10804000BFAFE097A2EAB6E1A196BFAFAEAFA197EE
:10805000312C212CBFEF6C96BFAF6C97EFEFA4963D
:10806000EFAFA497FFEFE396FFAFE3972FE4EA9615
:108070002FAFEA9733ECEB963FAFEB9707E481E045
:1080800090E0A0E0B0E0022C04C0880F991FAA1F66
:10809000BB1F0A94D2F7C458DF4F88839983AA8301
:1080A000BB83CC57D040A6EBB4E0E296BFAFAEAFF7
:1080B000E297EEE8F6E1A396FFAFEEAFA39710E0EC
:1080C000C058DF4F2882C058D040E296AEADBFAD59
:1080D000E2978D91E296BFAFAEAFE29790E0B0E04D
:1080E000A0E0C458DF4F288139814A815B81CC5799
:1080F000D04082239323A423B523892B8A2B8B2B57
:1081000009F0E5C0A196AEADBFADA197CD90DD90D1
:10811000ED90FC90A396AEADBFADA3972D913D9190
:108120004D915C91A8962CAF3DAF4EAF5FAFA89735
:10813000A7019601AC966CAD7DAD8EAD9FADAC97B1
:108140000F947E592B013C01A8962CAD3DAD4EAD50
:108150005FADA897E0966CAD7DAD8EAD9FADE0971D
:108160000F947E594B015C01A3019201C301B2013E
:108170000F94F3522B013C01A5019401C501B401F8
:108180000F94F3529B01AC01C301B2010F947F59CC
:108190000F942D5C4B015C01A70196016BA17CA1A2
:1081A0008DA19EA10F947E596B017C01A8962CADE8
:1081B0003DAD4EAD5FADA8976FA178A589A59AA5F5
:1081C0000F947E592B013C01A7019601C701B6010E
:1081D0000F94F3526B017C01A3019201C301B20120
:1081E0000F94F3529B01AC01C701B6010F947F5964
:1081F0000F942D5C20E030E040E751E40F94795A71
:10820000A50194010F947F596B017C018090BB0400
:108210009090BC04A090BD04B090BE0420E030E07B
:1082200040E85FE3C501B4010F94DF5B1816F4F476
:10823000C501B4010F94EB5A4B015C0160E070E0A2
:10824000CB01181419041A041B0434F40F94C44D00
:10825000A50194010F94F3580F9494529B01AC0123
:10826000B601C7010F947F596B017C01E3962FADD6
:10827000E397EA963FADEA97EB964FADEB97502F19
:10828000B601C7010F948D5287FF21C06C961FAFB6
:108290006C97C058DF4FB881C058D040A496BFAF8C
:1082A000A497E696CFAEE697E796DFAEE797E89617
:1082B000EFAEE897E996FFAEE997E396CFAEE39786
:1082C000EA96DFAEEA97EB96EFAEEB970F2D1F5FC6
:1082D000A396EEADFFADA3973496A396FFAFEEAF96
:1082E000A397153009F0F1CEFFEF2F1A3F0AA196A0
:1082F0002EAD3FADA1972C5F3F4FA1963FAF2EAF64
:10830000A19735E02316310409F0B9CE6C964FAD34
:108310006C97E42FF0E0EA54FB4F208181E090E07D
:10832000A0E0B0E0A4960FACA49704C0880F991FFA
:10833000AA1FBB1F0A94D2F7822B8083A4965FAD3D
:10834000A49762965FAF629763964FAF6397E69686
:108350008FADE697E7969FADE797E896AFADE897C4
:10836000E996BFADE99767968CAF9DAFAEAFBFAF53
:1083700067975F3F09F414C24F3F09F411C284E0CC
:108380004802F0011124E257F94E10810181328038
:10839000238027E137EB41ED58EB612F702F832DC0
:1083A000922D0F94DF5B87FDFFC127E030E040E7AF
:1083B00053E4612F702F832D922D0F948D52181638
:1083C0000CF4F2C1A4969FADA497A4E09A02F00128
:1083D0001124EE55F94EC080D180E280F38027E170
:1083E00037EB41ED58EBB601C7010F94DF5B87FD1A
:1083F000DBC127E030E040E753E4B601C7010F944A
:108400008D5218160CF4D0C120E030E040EA50E460
:10841000B601C7010F947F59A0966FAFA097A2969F
:108420007FAFA297A5968FAFA597A9969FAFA99763
:10843000CB01A596AFADA597A996BFADA9972196FB
:108440008CAF9DAFAEAFBFAF2197812F902FA32DE3
:10845000B22D25968CAF9DAFAEAFBFAF2597A4963A
:10846000BFADA497B11150C26C96EFAD6C97E111FE
:1084700018C220E030E040EA50E4612F702F832DD5
:10848000922D0F947F59A4966FAFA497AD967FAFAE
:10849000AD97E1968FAFE197E3969FAFE3976C9628
:1084A000FFAD6C97FF2309F4F1C26C963FAD6C975A
:1084B000A096CFAEA097A296DFAEA297A596EFAEFC
:1084C000A597A996FFAEA99734300CF014C222EDFF
:1084D000822E23E5922E2BE7A22E21E4B22E2196A6
:1084E0004CAC5DAC6EAC7FAC219725962CAD3DAD10
:1084F0004EAD5FAD25976F962CAF3DAF4EAF5FAFE2
:108500006F97A3019201B601C7010F947E592D9672
:108510006CAF7DAF8EAF9FAF2D976F962CAD3DADFD
:108520004EAD5FAD6F97612F702F832D922D0F94FD
:108530007E5961966CAF7DAF8EAF9FAF6197A301FF
:10854000920160919D1070919E1080919F1090916A
:10855000A0100F947E592B013C016F962CAD3DADC0
:108560004EAD5FAD6F976091A1107091A210809198
:10857000A3109091A4100F947E596F966CAF7DAFAD
:108580008EAF9FAF6F97A0968FADA097A2969FAD2D
:10859000A297A596AFADA597A996BFADA9978DA7B0
:1085A0009EA7AFA7B8ABA4968FADA497AD969FAD8D
:1085B000AD97E196AFADE197E396BFADE39789AB99
:1085C0009AABABABBCABC984DA84EB84FC84CDAA98
:1085D000DEAAEFAAF8AE2DEC3CEC4CEC5CE3C50156
:1085E000B4010F94F35229813A814B815C810F943D
:1085F000F3522091A9103091AA104091AB105091E4
:10860000AC100F947F5969AF7AAF8BAF9CAFA301C9
:108610009201C301B2010F94F3522B013C016F96FA
:108620002CAD3DAD4EAD5FAD6F97CA01B9010F9452
:10863000F3529B01AC01C301B2010F947F5920E0BA
:1086400030E040E050E40F94DF5B1816ACF420E01B
:1086500030E040E05FE3C701B6010F947F592996EF
:108660006CAF7DAF8EAF9FAF2997BE01635C7F4F2C
:10867000CE0101960E94992C89859A85AB85BC858F
:1086800029968CAF9DAFAEAFBFAF29976B961CAE4E
:108690001DAE1EAE1FAE6B97BE01695A7F4FCE0155
:1086A000CD960E94902CCE0101960F946F2EA09033
:1086B0007C10B0907D10C0907E10D0907F10E09024
:1086C0007810F090791000917A1010917B1097013A
:1086D000A801B501C6010F94DF5B181614F07501EF
:1086E00086018090790290907A02A0907B02B090EF
:1086F0007C022DEC3CEC4CEC5DE3B701C8010F941F
:10870000F3526093790270937A0280937B02909384
:108710007C0240E0BE01675B7F4FCE018D960F94D7
:108720004D3680E1EDE9F0E1A5E3B8E001900D926E
:108730008A95E1F78092790290927A02A0927B0268
:10874000B0927C020E9470258111C8CB20E04FEFCF
:10875000BE016F5A7F4FCE0101960E945C2E20E031
:1087600041E0BE016F5A7F4FCE0101960E945C2E00
:108770002FEF40E0BE016F5A7F4FCE0101960E945D
:108780005C2E21E040E0BE016F5A7F4FCE01019682
:108790000E945C2E0E94D6DC0E94702581119ECB27
:1087A0008091AD108093AE10E5964EAD5FADE5972C
:1087B00041505109E5965FAF4EAFE597452B09F45F
:1087C0008DCB62968FAD629787FD88CB63968FAD18
:1087D000639787FF17CC82CB63E687E89AE00E9415
:1087E00064B20F948C3580E1EDE9F0E1A5E3B8E0E7
:1087F00001900D928A95E1F72D853E854F85588928
:10880000609141087091420880914308909144081A
:108810000F947F59609341087093420880934308F6
:1088200090934408CE01CD960E9461F92D853E8536
:108830004F855889609141087091420880914308A2
:10884000909144080F947E596093410870934208B8
:1088500080934308909344088CA58111A2CB81E0BA
:108860008CA78D819E81AF81B885B0588DA79EA7BA
:10887000AFA7B8ABBE01635D7F4F85E398E00E9470
:10888000902C8FCB2BA13CA14DA15EA1AC962CAF1F
:108890003DAF4EAF5FAFAC978FA198A5A9A5BAA584
:1088A000CBCBC601D70121968CAF9DAFAEAFBFAF8A
:1088B000219720E030E040EA50E4612F702F832DB3
:1088C000922D0F947E5925966CAF7DAF8EAF9FAFE2
:1088D00025976C962FAD6C9724300CF4CACDA496D6
:1088E0001FAFA497AD960FAFAD97E1963FAEE1975E
:1088F000E3962FAEE39792ED892E93E5992E9BEFA9
:10890000A92E90E4B92EEBCDA4964FADA497443098
:108910000CF46EC06C965FAD6C975430BCF120E0E7
:1089200030E040EA50E4B601C7010F947E59219629
:108930006CAF7DAF8EAF9FAF219720E030E040EA73
:1089400050E4612F702F832D922D0F947E59A496A1
:108950006FAFA497AD967FAFAD97E1968FAFE197DC
:10896000E3969FAFE3976C969FAD6C97A096CFAEC2
:10897000A097A296DFAEA297A596EFAEA597A9966F
:10898000FFAEA99794300CF0B6CFA1CDC601D701A8
:1089900021968CAF9DAFAEAFBFAF219720E030E006
:1089A00040EA50E4612F702F832D922D0F947F5950
:1089B00025966CAF7DAF8EAF9FAF25976C968FAD30
:1089C0006C978111BACF20E030E040EA50E4B60164
:1089D000C7010F947E59A0966FAFA097A2967FAF64
:1089E000A297A5968FAFA597A9969FAFA99777CF86
:1089F0006C96AFAD6C97A1112BC020E030E040E247
:108A000051E4A0966FADA097A2967FADA297A596D0
:108A10008FADA597A9969FADA9970F947E59A09663
:108A20006FAFA097A2967FAFA297A5968FAFA5979D
:108A3000A9969FAFA997A4961FAFA497AD960FAF25
:108A4000AD97E1963FAEE197E3962FAEE3973FCD2A
:108A50006C96BFAD6C97B43034F120E030E040E26A
:108A600051E4A0966FADA097A2967FADA297A59670
:108A70008FADA597A9969FADA9970F947E59219682
:108A80006CAF7DAF8EAF9FAF2197D5CFA096CFAE05
:108A9000A097A296DFAEA297A596EFAEA597A9964E
:108AA000FFAEA99728CFA4961FAFA497AD960FAF9E
:108AB000AD97E1963FAEE197E3962FAEE39782ED57
:108AC000882E83E5982E8BEFA82E81E4B82E07CD53
:108AD0008FE299E00C940E35CF92DF92EF92FF92E5
:108AE0000F931F93CF93DF9388E50E941330D82E06
:108AF00089E40E941330C82E8823D1F10E94E52F0B
:108B0000D82F89E50E941330182F8AE40E94133071
:108B1000082F882309F455C00E94E52FC82F8AE545
:108B20000E941330E82EF12C811104C081E50E94CF
:108B30001330F82EC11001C000E0802F90E0D1105A
:108B400001C010E0810F911D019721F4E11062C076
:108B5000F11060C00E94684583E19EE0DF91CF91F3
:108B60001F910F91FF90EF90DF90CF900C940E35F6
:108B7000D11002C0DFEFC5CF0E94E92F20914F092D
:108B80003091500940915109509152090F947E59EA
:108B900020E030E040EA51E40F947E5920E030E0DC
:108BA0004EEB51E40F947F5922E936E74CEA5CE33F
:108BB0000F94F3520F94EB5AD62F653008F4A1CFDF
:108BC000D9CF111102C0CFEFAACF0E94E92F209177
:108BD00053093091540940915509509156090F9409
:108BE0007E5920E030E040EA51E40F947E5920E0C5
:108BF00030E04EEB51E40F947F5922E936E74CEA1E
:108C00005CE30F94F3520F94EB5AC62F653008F4CF
:108C100086CFD9CFD7FD02C0C7FF05C00E946845E7
:108C20008AEF9DE09BCF0E94E92F9B01AC010D2FA5
:108C3000DD0F110BAC2FCC0FBB0B60E070E0CB0154
:108C4000FF2091F065E0609FF001619FF00D11241D
:108C5000EA0FFB1FEE0FFF1FEE0FFF1FE153FA4F4E
:108C60006081718182819381E5E0E09FE001E19F75
:108C7000D00D1124CA0FDB1FCC0FDD1FCC0FDD1F61
:108C8000C153DA4F0F947F59688379838A839B831A
:108C9000DF91CF911F910F91FF90EF90DF90CF90D8
:108CA000089589E299E00C940E35CF9384E50E94F3
:108CB0006130C0E08823D9F00E94C12FC82F181658
:108CC000B4F40E9451468DE40E94D5348091F4049E
:108CD0009091F5040F94A23F6C2FCC0F770B8BEF84
:108CE0009EE00E940E3C8AE00E94D534CFEF8C2F8C
:108CF000CF9108954F925F926F927F928F929F9241
:108D0000AF92BF92CF92DF92EF92FF92CF93DF9319
:108D1000CDB7DEB72C970FB6F894DEBF0FBECDBF30
:108D200040904F095090500960905109709052093D
:108D30002091390230913A0240913B0250913C021D
:108D4000C301B2010F947F5969837A838B839C831B
:108D50008090530990905409A0905509B0905609FD
:108D600020913D0230913E0240913F0250914002DD
:108D7000C501B4010F947F596D837E838F839887DB
:108D8000C0905709D0905809E0905909F0905A09BD
:108D9000209141023091420240914302509144029D
:108DA000C701B6010F947F5969877A878B879C87A3
:108DB000209145023091460240914702509148026D
:108DC000C301B2010F947F592B013C01209149024C
:108DD00030914A0240914B0250914C02C501B401BE
:108DE0000F947F594B015C0120914D0230914E024E
:108DF00040914F0250915002C701B6010F947F5924
:108E00006B017C010E9451468CE49EE00E940E356D
:108E100083E50E941330882321F00E94D52F809390
:108E2000370280913702811151C083E39EE00E9496
:108E30000E3584E49EE00E940E3549815A816B8193
:108E40007C818AEE9BE20E94F8364D815E816F81C3
:108E5000788587EF90E40E94F83649855A856B85BE
:108E60007C8584EF90E40E94F83682E49EE00E94C4
:108E70000E358AE39EE00E940E35B301A2018AEE10
:108E80009BE20E94F836B501A40187EF90E40E94AE
:108E9000F836B701A60184EF90E40E94F8368AE024
:108EA0002C960FB6F894DEBF0FBECDBFDF91CF91E9
:108EB000FF90EF90DF90CF90BF90AF909F908F90FA
:108EC0007F906F905F904F900C94D53487E39EE035
:108ED000AECF2F923F924F925F926F927F928F927E
:108EE0009F92AF92BF92CF92DF92EF92FF920F9339
:108EF0001F93CF93DF93CDB7DEB76A970FB6F89481
:108F0000DEBF0FBECDBF83E50E941330182F309017
:108F10009C10882319F00E94D52F382E40909D1068
:108F200050909E1060909F107090A0108091A110A2
:108F30009091A210A091A310B091A4108B8B9C8B48
:108F4000AD8BBE8B8091A5109091A610A091A7101B
:108F5000B091A8108F8B988FA98FBA8F112329F009
:108F6000311003C080E00E94CA3286E50E941330AF
:108F7000888B0E94C533882309F4BFC083E40E9414
:108F80001330882309F498C00E94E92F6B017C01FB
:108F9000AFECB5E0BF83AE83B987A887F5E0FD836A
:108FA0001D861E8628EC2F8702EC1A86212C88EC61
:108FB0008B8792E49C87A885B985BA8BA98B15E02D
:108FC000E989FA8981909190A190B190FA8BE98B0F
:108FD0002A85322D4B855C85C501B4010F948D52D5
:108FE00087FF04C08A86292CAB86BC862D853E85EA
:108FF0004F85502FC501B4010F94DF5B181624F480
:109000008D869E86AF860B2D1150D1F6FD81F150D5
:10901000FD8388859985449699878887F111CBCF00
:109020002D853E854F85502F6A85722D8B859C85B9
:109030000F947F5920E030E040E05FE30F94F3525B
:10904000A70196010F947F596B017C012DEB37E34B
:1090500046E855EB0F94DF5B87FD0AC02DEB37E345
:1090600046E855E3C701B6010F948D52181624F552
:1090700080E00E94CA3215E0AE80BF8005E0D501D5
:109080006D917D918D919D915D014D01B4E08B1AA3
:109090009108A70196010F947E59F40160837183B2
:1090A00082839383015059F711508E819F8144969A
:1090B0009F838E831111E0CFA889AA2351F00E94CB
:1090C000C533882331F080ED9CE00E940E350E946C
:1090D0005B368AE50E941330882359F00E94E92FFD
:1090E00069837A838B839C8360E0CE0101960E9422
:1090F000E532832D0E94CA320BC0311003C098891B
:10910000992339F30E94514686EE9CE00E940E3569
:10911000332051F080919C10811106C00E94684557
:1091200081EB9CE00E940E350E94514683EA9CE050
:109130000E940E3580919C100E94DA360E945146A2
:1091400086E99CE00E940E35C0906708D0906808C0
:10915000E0906908F0906A0820E030E0A901C701BA
:10916000B6010F94DF5B18160CF053C042E0C70144
:10917000B6010F949C078DE00E94D5348AE00E94CE
:10918000D534A301920160919D1070919E10809141
:109190009F109091A0100F948D5281111FC02B89A8
:1091A0003C894D895E896091A1107091A2108091D7
:1091B000A3109091A4100F948D5281110FC02F898C
:1091C000388D498D5A8D6091A5107091A6108091AF
:1091D000A7109091A8100F948D5281110E9419FB35
:1091E0006A960FB6F894DEBF0FBECDBFDF91CF9168
:1091F0001F910F91FF90EF90DF90CF90BF90AF90B5
:109200009F908F907F906F905F904F903F902F90A6
:10921000089581E99CE00E940E35B3CFCF93C82F0B
:1092200082E0C11184E040E060E00E94D3840E94AB
:10923000514689E999E0CC2311F08EEA99E0CF916B
:109240000C940E35FF920F931F93CF93DF93EC0195
:109250008B01F42E0E9431D50E94684589E099E087
:109260000E940E350115110511F40DE81FE320973A
:1092700011F4C0E0D9E00E941CB91F930F93DF9353
:10928000CF9380EF98E09F938F9381E08F930E941C
:1092900049B20E94EA83C0915416C695C6958FE4E0
:1092A00096E10E949527DC2FDD0F1D2F1C0FEDB7D7
:1092B000FEB737960FB6F894FEBF0FBEEDBF83E042
:1092C0000E94792644E653E16C2F80E00E94402AF8
:1092D00010928A16D0938B1681EE98E00E94252872
:1092E00010928A1610938B1684ED98E00E94252820
:1092F00083E596E10F94463D8111E1CF61E087EF70
:1093000098E00E94D63589EE93E030E6019729F087
:10931000232F2A950000E9F7F9CFF89489EE93E01E
:1093200038EE019729F0232F2A950000E9F7F9CFAD
:109330000E9431D5FF2041F00E9440340E94C2219A
:10934000909905C0A895FCCF0E94C021F7CF909BB3
:1093500002C0A895FCCFF0E0E0E0DF91CF911F9133
:109360000F91FF9019945F926F927F928F929F92CC
:10937000AF92BF92CF92DF92EF92FF920F931F9323
:10938000CF93DF931F92CDB7DEB77C0139018B01FC
:109390005B01A40EB51ED12CC12CA016B10609F498
:1093A00050C0F70180809180F80151908F0159825F
:1093B000C4010F94AB585816B9F1652DC4010F9430
:1093C000B358FFEFCF1ADF0AC6018F779927892B91
:1093D00021F162E070E080E090E00F942035C4015C
:1093E0000F94AB5899818917F9F00E94514683E791
:1093F00096E00E940E3581E00F90DF91CF911F9192
:109400000F91FF90EF90DF90CF90BF90AF909F9023
:109410008F907F906F905F90089562E070E080E0A1
:1094200090E00E940A34DBCFBE016F5F7F4FC30123
:109430000F946325F7018081918101969183808348
:10944000ACCF80E0D9CF8091AD109091AE102FEFCE
:109450003FEF981751F0E92FF0E0E355FF4E2281DE
:1094600030E09F5F9F779093AE10C90108951F92DF
:109470000F920FB60F9211240F900FBE0F901F90F6
:1094800018951F920F920FB60F9211240BB60F92E0
:109490002F933F934F935F936F937F938F939F93FC
:1094A000EF93FF939091C6005091AE103091AD10A4
:1094B00041E0430F4F7720917D04213108F099C09E
:1094C000E22FF0E08827E859F54B8F4F0D9476593D
:1094D000794AA24AB14AC04AC74AF94ACB4AF94A2C
:1094E000CF4AD34AF94AD74ADB4ADF4AE64AF94A21
:1094F000F14A903229F0F8F49A3011F09D3001F5DC
:10950000541731F0E32FF0E0E355FF4E9283342FF0
:109510003093AD10FF91EF919F918F917F916F915B
:109520005F914F913F912F910F900BBE0F900FBE07
:109530000F901F9018959D3481F081E09E3471F05A
:1095400080E10CC09A3338F49033D0F69032C1F2F7
:109550009D32B1F7D5CF9D3499F782E080937D0499
:10956000CFCF913359F018F4903251F2E9CF88E01F
:109570009433A1F38BE0983389F3E2CF83E0EECF0D
:1095800084E0903359F386E0913341F3D9CF85E0FD
:109590009833B1F6E3CF87E0923391F6DFCF89E0DD
:1095A000913371F6DBCF8AE0903351F6D7CF8CE060
:1095B000973331F6D3CF8DE0963311F6CFCF90327B
:1095C00009F49ECF8EE0933549F2BACF80ED890F32
:1095D0008A3008F095CF2FE020937D0480937C049F
:1095E0008FCF9A3019F09D3009F08ACF10927D0408
:1095F00087CF9A3019F09D3009F082CF80918D1677
:109600008823A1F3273001F138F4253079F710923F
:10961000710210924F08EACF2A30D1F02F3031F783
:1096200020917C0480914D0810924D08823089F37E
:10963000843091F08130D1F6222319F02130B1F637
:1096400082E080934E08D2CF81E080934106CECF56
:1096500081E080934006CACF65E27EE17093C60741
:109660006093C507C3CF8EBD0DB407FEFDCF08952F
:109670008FEF8EBD0DB407FEFDCF8EB5089590918E
:1096800064009B7F90936400982F906A96959CBD90
:1096900080FD03C091E0863009F490E09DBD0895FF
:1096A000CF93DF93EB010E940E35CE01DF91CF9176
:1096B0000C94AECEAF92BF92CF92DF92EF92FF9218
:1096C0000F931F93CF93DF93CDB7DEB7E6970FB617
:1096D000F894DEBF0FBECDBF0091F7041091F804DF
:1096E000F80101900020E9F731976F01C01AD10A03
:1096F000F801CF01801B910B8C159D053CF48191E5
:109700008F32B9F7DF0111971C92F3CF8BE1E2EEB4
:10971000F6E1DE015C9601900D928A95E1F7F12C5D
:10972000E12CEC14FD040CF05DC0F801EE0DFF1D02
:109730008081811103C08FEFE81AF80A5801AE0C3E
:10974000BF1CF5018081882309F44CC0FFEFEF1A9C
:10975000FF0AF801EE0DFF1D7F01E01AF10A819169
:109760008111FACFCE014C960E9414D38BE1FE01F9
:109770007C96DE01119601900D928A95E1F7B50174
:10978000CE0101960E9420CBCE0101960E94133299
:109790008FE20E94D5348091211381113BC08CE56A
:1097A00093E00E94AECE8091C11684FF1BC0198247
:1097B0001C8221E0A501BE01645E7F4FCE010196AF
:1097C0000F94BD05811129C08AE00E94D5340E9402
:1097D0005146B50189EB94E10E94504BCE010196B0
:1097E0000E9413328AE00E94D534CE014C960E942A
:1097F0001332E6960FB6F894DEBF0FBECDBFDF91F1
:10980000CF911F910F91FF90EF90DF90CF90BF907D
:10981000AF90089581E293E1C4CFCE014C960E94AF
:1098200016D28BE1FE013196DE015C9601900D921D
:109830008A95E1F7CE0101960E94133272CF2F92E2
:109840003F924F925F926F927F928F929F92AF92D0
:10985000BF92CF92DF92EF92FF920F931F93CF931D
:10986000DF9300D000D000D01F921F92CDB7DEB79B
:10987000B82E80919A11843008F0D1C10F945335DD
:109880006B017C0180919A11811108C08091AD100B
:109890009091AE10891B8F7709F463C681E6A82EDC
:1098A00013C08A3019F08D3009F0F6C0109295116E
:1098B0008091331190913411FC01E15DFE4E1682CE
:1098C000892BF1F40E9473F280919A11843008F090
:1098D000ECC08091AD109091AE10891B8F7709F488
:1098E000E4C00E94234A97FFDCCF0E94684589EBC1
:1098F00097E00E940E358091AD108093AE10E4CFBA
:10990000109234111092331105E311E1F8018191A5
:10991000803209F446C08E3409F0A9C064EB77E0C8
:10992000C8010F940A524C01892B41F06EE470E09B
:10993000C80104960F94CD5C009709F4C8014AE071
:1099400050E070E060E001960F947A4F2B013C01EB
:1099500080912F1190913011A0913111B09132115D
:109960000196A11DB11D481659066A067B0629F00D
:1099700060E081E897E0892851F16AE270E0C8016F
:109980000F94FC5C9C01009729F1982F901B912C5F
:10999000992349F09150F801E90FF11D8081982633
:1099A000F7CF8F01B3CF4AE050E070E060E0C9012B
:1099B00001960F947A4F292D30E050E040E0621775
:1099C00073078407950751F060E082E697E00F94F3
:1099D000302A7ACF60E088E397E0F9CF40922F11E8
:1099E00050923011609231117092321180910808BA
:1099F0008130E1F067E470E0C8010F94CD5C00971E
:109A0000A9F04AE050E070E060E001960F947A4FD0
:109A1000643071058105910548F487E996E00E945C
:109A20000E3560E08DE896E00E9464B2C092540862
:109A3000D0925508E0925608F0925708809135115F
:109A40008B3309F441CF80919A11843008F03CCFD8
:109A500080919C118A9DC001112465E371E18356B8
:109A60009E4E0F94D85C80E00F94EA292DCF809110
:109A7000C11680FFBBCF60E17FE3C8010F940A529B
:109A8000009731F0FC01838180538A3008F0AECF1B
:109A900060E08EE097E09BCF23E331E145E351E1C5
:109AA00065E971E10E944F210FCF8091C11682FFBD
:109AB000B6C01A82198271E6F72EE0E1EE2EF9E6C1
:109AC000DF2E80919A11843008F0A9C00E9487216E
:109AD0008111A5C041E050E0BE016B5F7F4F86E27F
:109AE00098E10E944ECF0D8110E0019711F00FEF29
:109AF0001FEF80912E1890912F18A0913018B091DF
:109B000031188093BD169093BE16A093BF16B093E4
:109B1000C0160E9487210F3F100749F4811107C02A
:109B20000E94684587ED97E00E940E35CACF4091AC
:109B30009C11242F30E00A3061F00D3051F0882361
:109B400009F45FC089819A81009719F001969A8380
:109B5000898310927E0489819A81F29EF001F39E9E
:109B6000F00D1124E656FE4EE80FF91F1382892BE3
:109B700069F50E9473F20E948721882309F4A1CF1E
:109B80000E94D6DC86E298E10E9416D28091B81637
:109B9000882391F181508093B8168D9DC0011124C6
:109BA00062E08C5C984F0F945243E091B81624E029
:109BB000E29FF0011124E05DF84F608171818281A4
:109BC00093810E94B4230E9489CA7BCF1A82198292
:109BD00081E00F94EA298091BD169091BE16A09164
:109BE000BF16B091C0168093961190939711A093D1
:109BF0009811B0939911BFCF0E941FD2E09208082C
:109C000060CF4F9DA001112443565E4E9E012F5FF1
:109C10003F4F6EE774E0802F0E944F2152CF0F9488
:109C200053356B017C01B11004C080914E0688232E
:109C300051F0C0924508D0924608E0924708F09251
:109C40004808BB24B3948091D1049091D204A09190
:109C5000D304B091D4040097A105B10551F140910E
:109C60004508509146086091470870914808840F54
:109C7000951FA61FB71FA7019601281B390B4A0B7A
:109C80005B0BDA01C901B7FD14C00E946845609101
:109C900052087091530882E398E00E94504B8AE08A
:109CA0000E94D53440E070E060E090E080E00E94E7
:109CB00022498091100290911102A0911202B0915C
:109CC0001302892B8A2B8B2B79F090911716809198
:109CD0001816981709F4ACC1C0924508D0924608EE
:109CE000E0924708F092480880918F049091900488
:109CF0009099E0C101969093900480938F04809195
:109D00008F04909190048E3E92406CF00E946845C2
:109D10008FE098E00E940E3540E070E060E090E057
:109D200080E00E9422490F9453354B015C018091E1
:109D30004F08811108C0209117169091181681E0E4
:109D4000291301C080E02091D3153091D41591E002
:109D500089272A3A31050CF480E091E04091830490
:109D6000509184046091850470918604452B462BA4
:109D7000472B09F490E0981789F0882309F4A0C1D3
:109D8000D501C40180569444A24FBF4F80938304F1
:109D900090938404A0938504B09386044090A91006
:109DA0005090AA106090AB107090AC1020917F047E
:109DB000309180044091810450918204C301B2012A
:109DC0000F948D52882319F180918304909184041B
:109DD000A0918504B091860440927F045092800443
:109DE0006092810470928204892B8A2B8B2B09F458
:109DF00049C0D501C40180569444A24FBF4F8093FF
:109E0000830490938404A0938504B0938604809186
:109E1000830490918404A0918504B09186040097F6
:109E2000A105B10579F1881A990AAA0ABB0AB7FCFB
:109E300029C0109283041092840410928504109219
:109E400086048AEF97E00E940E3560E086EE97E088
:109E50000E9464B28091D5159091D61518161906F6
:109E600024F490E080E00E9458DC80917108909189
:109E700072081816190634F41092720810927108BC
:109E80000E9451C680918B0490918C04A0918D0406
:109E9000B0918E0446015701881A990AAA0ABB0A92
:109EA000D501C401B7FD9CC12091171690911816D9
:109EB0008091600240916102291306C190918D0941
:109EC000899FC0011124880F892F881F990B9195B4
:109ED0008D8380918E09489FC0011124880F892F9E
:109EE000881F990B91958E830F94533569837A83DC
:109EF0008B839C8340E0BE016F5F7F4FCE01059650
:109F00000E942ADD6D8170E089E00F944A3441E0BF
:109F1000BE016F5F7F4FCE0105960E942ADD6E81E4
:109F200070E087E00F944A3480914D06882309F44D
:109F30004AC10091330210913402C8010297209166
:109F4000D5153091D615281739070CF43CC18090EF
:109F500018168F82188619861A861B868091171606
:109F60009F80891509F4CAC0892D90E03BE6A32E95
:109F7000A89EF001A99EF00D1124EE55F64F4589DB
:109F800056896789708D452B462B472B81F4418D6F
:109F9000528D638D748D452B462B472B41F4458D97
:109FA000568D678D70A1452B462B472BE1F12BE693
:109FB000B22EB89E9001B99E300D1124A9014E55C4
:109FC000564F1A01FA0161817281838194810F9445
:109FD0002D5C4B015C01F10161A172A183A194A1EF
:109FE0000F9492522B013C01F10165A176A187A14A
:109FF00090A50F9492529B01AC01C301B2010F9442
:10A00000795AA50194010F94F3524B015C01288504
:10A0100039854A855B850F94DF5B181624F48886A2
:10A020009986AA86BB868F818F5F8F708F8396CF2C
:10A03000BB2019F01092910457CE0F945335009124
:10A0400045081091460820914708309148088090B3
:10A05000100290901102A0901202B0901302080D0D
:10A06000191D2A1D3B1D601B710B820B930B97FD65
:10A07000E1CF80919104811137CE81E080939104EA
:10A080005F9A8091C3078E7F8093C3078A9A8091DD
:10A09000C3078D7F8093C3078091080180958170ED
:10A0A000809306018091C3078B7F8093C3070E9432
:10A0B000C0211ACE181619060CF021CE01971BCE1E
:10A0C00080E090E0DC0162CE209118165BE6259FCF
:10A0D000900111242E55364FF901EF59FF4F908111
:10A0E000899FC0011124880F892F881F990B919592
:10A0F0008D832E593F4FF9018081EDCE20912D02A5
:10A1000030912E0240912F0250913002688579855E
:10A110008A859B850F94F3524B015C01B801012E97
:10A12000000C880B990B0F9494529B01AC01C50154
:10A13000B4010F947F5969837A838B839C83409108
:10A14000310250913202B801CE0101960E94FCD535
:10A1500089809A80AB80BC804090870450908804AE
:10A160006090890470908A04A3019201C501B40132
:10A170000F948D5287FF16C028E431EE4AE75FE363
:10A18000C301B2010F94F35220E037ED43EA5CE3E0
:10A190000F947F59A50194010F94F35269837A8338
:10A1A0008B839C8369817A818B819C8160938704F6
:10A1B000709388048093890490938A040F94EB5AD7
:10A1C000CB010E9458DCF4E6CF0ED11CE11CF11C3F
:10A1D000C0928B04D0928C04E0928D04F0928E0495
:10A1E0000E9473F280910808882309F47AC1909143
:10A1F0000901892F8095817010910802181709F4C0
:10A200005AC02091C11620622093C1168093080283
:10A2100090FD10C064EF71E080E090E00E940A348D
:10A220000E9441D28091C11683FDBEC1112309F461
:10A2300042C002C00E9430D2123008F46BC100E06C
:10A240000E94BB2683E080937D020F9453356C59A6
:10A250007F4F8F4F9F4F6093FC047093FD0480935A
:10A26000FE049093FF04002331F1123021F5809118
:10A27000C11683FF20C00F948C40882379F081E0C1
:10A280000F94A83F42EB50E06DE978E087EC96E14F
:10A290000E944ECF87EC96E10E9416D20E940132B6
:10A2A000811144C10E94EB310F94974181E080936A
:10A2B000B7160F94D9410F9453356B017C0110915F
:10A2C0000F021123F1F0809150088823D1F04091C2
:10A2D0009204509193046091940470919504460106
:10A2E0005701841A950AA60AB70AB501A40177FD99
:10A2F0001AC0833009F430C10CF01FC181300CF05A
:10A3000024C1212F30E0A8EEB3E00F942559C60EEA
:10A31000D71EE81EF91EC0929204D0929304E092D8
:10A320009404F092950480916508813009F073C01F
:10A330000F9453356B017C0180919A0490919B049A
:10A34000A0919C04B0919D04A7019601281B390B94
:10A350004A0B5B0BDA01C901B7FD3AC0D701C60150
:10A36000805F984DAF4FBF4F80939A0490939B04AA
:10A37000A0939C04B0939D048090C2059090C30567
:10A38000A090C405B090C5050E9494FDAB01BC012E
:10A390004093C2055093C3056093C4057093C505EF
:10A3A0008091B4079091B507A091B607B091B70717
:10A3B00088199909AA09BB09840F951FA61FB71F01
:10A3C0008093B4079093B507A093B607B093B707EF
:10A3D0008091960490919704A0919804B09199046B
:10A3E00046015701881A990AAA0ABB0AD501C40175
:10A3F000B7FD11C020E8C20E2EEED21E26E3E21EEB
:10A40000F11CC0929604D0929704E0929804F092C6
:10A4100099040E94DADB0F9425020E946EB68091A7
:10A42000D004882379F10F9453356B017C0180911E
:10A43000CC049091CD04A091CE04B091CF044601FC
:10A440005701881A990AAA0ABB0AD501C401B7FDA7
:10A4500019C02091D00430E0A8EEB3E00F94255944
:10A46000C60ED71EE81EF91EC092CC04D092CD04B1
:10A47000E092CE04F092CF0480E00F9440088AE08E
:10A480000E94D5348091CB04882359F10F94533521
:10A490006B017C018091C7049091C804A091C9040C
:10A4A000B091CA04A7019601281B390B4A0B5B0B1C
:10A4B000DA01C901B7FD15C02091CB0430E0A8EE48
:10A4C000B3E00F942559C60ED71EE81EF91EC092A0
:10A4D000C704D092C804E092C904F092CA040F9451
:10A4E000AF402B960FB6F894DEBF0FBECDBFDF9105
:10A4F000CF911F910F91FF90EF90DF90CF90BF9081
:10A50000AF909F908F907F906F905F904F903F9013
:10A510002F90089560E08FE698E00E9464B28091E9
:10A520000A0581118CCE0E94EA8389CE8CE898E0DE
:10A530009093C6078093C507BECE843009F0E1CE64
:10A540000E94514683E998E004C00E94514682EC83
:10A5500098E00E940E35D5CE0E9451468BEA98E0D5
:10A56000F8CF8091540890915508A0915608B09169
:10A570005708A7019601281B390B4A0B5B0BDA0120
:10A58000C901885E9340A109B109B7FD87C981ED72
:10A5900097E00E940E35C0925408D0925508E09280
:10A5A0005608F09257087AC9123028F460E08DE717
:10A5B00098E00E9464B201E043CECF93DF93C82FAE
:10A5C000D62F8091531083FD14C080919F09811173
:10A5D00010C08091820290918302AC0141505109D8
:10A5E0002091D5153091D6152417350714F40E9403
:10A5F00058DC40E06D2F8BE00E94D384CC2339F0EF
:10A6000040E061E080E0DF91CF910D94380A8091C5
:10A610009F0991E0892780937102809171028823BC
:10A6200089F08091D3159091D4152091D515309152
:10A63000D615821B930B97FF03C0919581959109C5
:10A64000029744F4109271028091531083FF06C068
:10A65000C1E01AC080E00E941F4CDFCFC0919F096B
:10A66000C11112C0809182029091830201972091C2
:10A67000D5153091D6152817390754F70E94514641
:10A6800088E899E00E940E358C2FDF91CF910895D4
:10A69000AF92BF92CF92DF92EF92FF920F931F93F0
:10A6A000CF93DF93CDB7DEB764970FB6F894DEBFD4
:10A6B0000FBECDBF0E945546D82E87FDB5C08AE596
:10A6C0000E946130882309F4C0C040E050E0BA0124
:10A6D0008AE50E947C307B018C014D2D63E085E092
:10A6E0000E94D3842091A5103091A6104091A7100C
:10A6F0005091A81060E070E08AE793E40F947E59CF
:10A700005B016C019701A8010F94DF5B181614F030
:10A710007501860120E030E0A901B701C8010F945E
:10A72000DF5B181624F4E12CF12C00E010E0B701F7
:10A73000C8010F94EB5A072E000C880B990B0F944D
:10A7400094526D837E838F83988720E030E0A90147
:10A750000F948D52882321F0CE0105960E94022489
:10A7600080E090E0A0EAB1E489879A87AB87BC8754
:10A770001D861E861F86188A8CE40E94133088234B
:10A7800009F468C00E94E92F6B017C0120E030E0F1
:10A79000A901C701B6010F94DF5B87FF04C0F7FA78
:10A7A000F094F7F8F094C98ADA8AEB8AFC8A20914F
:10A7B000D5153091D6152430310574F08091D3151C
:10A7C0009091D415821B930B97FF03C091958195AF
:10A7D000910901E004970CF400E063E080E00E943E
:10A7E000DD52811140C083E080932402109209055C
:10A7F0000E94EA836D817E818F8198858B019C0107
:10A80000305809831A832B833C8320E030E0A90170
:10A810000F948D52882321F0CE0101960E940224CC
:10A82000109209050E94EA8364960FB6F894DEBF81
:10A830000FBECDBFDF91CF911F910F91FF90EF9091
:10A84000DF90CF90BF90AF900895E12CF12C00E203
:10A8500011E443CFC090CA05D090CB05E090CC0561
:10A86000F090CD0593CF83E0E82E22E0AE01475F64
:10A870005F4FBE016F5E7F4FCE010D960F94342C5B
:10A88000B9CF6F927F928F929F92AF92BF92CF92E9
:10A89000DF92EF92FF920F931F93CF93DF9300D03D
:10A8A00000D01F921F92CDB7DEB75C014B013A0179
:10A8B000F22E68010091460610924206109243065D
:10A8C0001092440610924506109246060F945F358A
:10A8D0008091D5159091D6158C159D051CF4C60157
:10A8E0000E9458DC60E080E00E94DD5281112DC1A1
:10A8F000109209050E94EA831C141D0444F4C60149
:10A900000E9458DC40E060E080E00F94380A40E0AC
:10A9100060E088E00E94D38460E081E00E94DD5224
:10A9200080E090E0A0E7B2E489839A83AB83BC83A4
:10A9300080E090E0A0E8B0EC8D839E83AF83B88781
:10A94000BE016F5F7F4FCE0105960E9448F287E0FF
:10A950000E9488F0811158C08091A5109091A61096
:10A96000A091A710B091A8104091AA045091AB04F7
:10A970006091AC047091AD04C090A604D090A7047F
:10A98000E090A804F090A904C0923508D09236084F
:10A99000E0923708F09238084093390850933A080B
:10A9A00060933B0870933C0880933D0890933E0869
:10A9B000A0933F08B093400880E090E0A8E4B2E4A0
:10A9C00089839A83AB83BC83CE0101960E9461F98F
:10A9D0008091AE049091AF04A091B004B091B10405
:10A9E00080933D0890933E08A0933F08B0934008A1
:10A9F00080E090E0A0EAB0E489839A83AB83BC83D3
:10AA0000CE0101960E9461F9C12CD12C80E7E82E7D
:10AA100082E4F82EC982DA82EB82FC8280E090E048
:10AA2000A0E8B0E48D839E83AF83B887BE016F5FDB
:10AA30007F4FCE0105960E9448F220E030E0A90148
:10AA40006091B2047091B3048091B4049091B50404
:10AA50000F948D5287FF0BC0C982DA82EB82FC8291
:10AA6000BE016F5F7F4F82EB94E00E9448F28091BD
:10AA7000B2049091B304A091B404B091B504809352
:10AA8000A9109093AA10A093AB10B093AC10809330
:10AA9000410890934208A0934308B093440881E48E
:10AAA00098E00E9470EE8091CE0581110F94D23F04
:10AAB000109209050E94EA8361E081E39AE00E9416
:10AAC000D63580914E06815080934E0646EE5DE16C
:10AAD00069E37AE085E00F943F2D80914E0688234C
:10AAE00039F00E9489CA80914E06815080934E06AB
:10AAF0008091A504882351F01092A5048091A304AD
:10AB000080938D098091A40480938E0980916508BB
:10AB1000823011F40E9456FE0F9492420E94EA8302
:10AB200028960FB6F894DEBF0FBECDBFDF91CF9150
:10AB30001F910F91FF90EF90DF90CF90BF90AF905B
:10AB40009F908F907F906F900895E12C2F2DA301FF
:10AB5000B401C5010F94342CCFCE4F925F926F9207
:10AB60007F92AF92BF92CF92DF92EF92FF921F93AC
:10AB7000CF93DF9300D000D01F921F92CDB7DEB7E6
:10AB80005C01E62EF42E642F80E00E94DD52182F27
:10AB900081111BC0EE2021F0109209050E94EA836A
:10ABA000812F28960FB6F894DEBF0FBECDBFDF9180
:10ABB000CF911F91FF90EF90DF90CF90BF90AF901B
:10ABC0007F906F905F904F900895EE2029F040E0C5
:10ABD0006F2D83E00E94D38480E090E0A0E7B2E490
:10ABE0008D839E83AF83B88780E090E0A0E8B0ECCF
:10ABF00089839A83AB83BC83BE016B5F7F4FCE0199
:10AC000001960E9448F268E873E180E090E00E94BB
:10AC10000A34C12CD12C88ECE82E81E4F82ECD82A8
:10AC2000DE82EF82F88680E090E0A0E8B0E48983DD
:10AC30009A83AB83BC83BE016B5F7F4FCE010196CD
:10AC40000E9448F240908C1050908D1060908E10B1
:10AC500070908F10C0928C10D0928D10E0928E1058
:10AC6000F0928F1080E090E0A0E2B2E48D839E83AA
:10AC7000AF83B887F50180819181A281B3818983F7
:10AC80009A83AB83BC83BE016B5F7F4FCE0101967D
:10AC90000E9448F240928C1050928D1060928E105B
:10ACA00070928F10129A64E670E080E090E00E944B
:10ACB0000A3476CFBF92CF92DF92EF92FF920F933A
:10ACC0001F93CF93DF9300D01F92CDB7DEB77C01E7
:10ACD0006B018A01B22E61E084E29AE00E94D635CF
:10ACE00046EE5DE16BE27AE085E00F943F2D9091B6
:10ACF0004E0681E0890F80934E068091C11682FF37
:10AD000006C08B7F8093C1169E5F90934E060E9473
:10AD10008EFE80E1EDE9F0E1A6EAB4E001900D924B
:10AD20008A95E1F70E94D6DC8091A50481110FC0BD
:10AD300081E08093A50480918D098093A3041092F3
:10AD40008D0980918E098093A40410928E0920E0D1
:10AD500030E0A901F70160817181828193810F94B4
:10AD60008D528823F1F080919F0981110CC0809150
:10AD700082029091830201972091D3153091D415CE
:10AD80002817390774F080E090E0A0E7B2E48983E7
:10AD90009A83AB83BC83BE016F5F7F4FC7010E9464
:10ADA00048F287E00E9488F0811103C0B6010F9439
:10ADB0006A0120E030E0A901F8016081718182819F
:10ADC00093810F948D52882329F042E06B2DC801A6
:10ADD0000E94AD55129A64E670E080E090E00E9417
:10ADE0000A3481E00F900F900F900F90DF91CF9178
:10ADF0001F910F91FF90EF90DF90CF90BF9008953B
:10AE0000CF92DF92EF92FF92CF93DF936B017C01A1
:10AE1000D42FC091500883E08093500881E0809344
:10AE20004F08C114D104E104F10431F00F945335FB
:10AE3000C60ED71EE81EF91E80914F08882389F0A0
:10AE4000C114D104E104F10421F48D2F0E941F4CA0
:10AE5000F3CF0F9453356C197D098E099F0997FD27
:10AE6000F4CF10924F08C0935008DF91CF91FF901C
:10AE7000EF90DF90CF9008951F93CF93DF93D82F5B
:10AE8000C62F0E940E4961E08C2F0E9419320F9448
:10AE90005335685370458F4F9F4F609342067093B0
:10AEA00043068093440690934506109246061091FF
:10AEB000500883E08093500830E020E04EE650E4F4
:10AEC00066E17AE082E00E941D3681E080934F08BF
:10AED00080914F08882309F463C060E08C2F0E94A2
:10AEE000193280914606882309F456C040E060E09C
:10AEF0008AE00E94D3840E9451468CEF99E00E9420
:10AF00000E3530E020E046EE59E06DEE79E082E06B
:10AF10000E941D3641E060E070E0CB010E940057C6
:10AF200030E020E050E040E069ED79E085E00E940B
:10AF30001D3610924206109243061092440610925B
:10AF40004506109246060F945F3560E080E00E944F
:10AF5000DD528D2F0E940E490F9453356853704572
:10AF60008F4F9F4F60934206709343068093440631
:10AF7000909345061092460630E020E04EE650E4FD
:10AF80006DEC79E082E00E941D3681E080934F08ED
:10AF900061E08C2F0E94193281E00E941F4C98CFF3
:10AFA00010935008DF91CF911F910895CF92DF92B7
:10AFB000EF92FF920F931F93CF93DF93CDB7DEB73E
:10AFC000A0970FB6F894DEBF0FBECDBF0E945546C6
:10AFD00087FDD1C0482F61E081E00E94D38485E4E1
:10AFE0000E941330882309F4D5C00E94E92F6B0119
:10AFF0007C0120E030E0A9010F94DF5B87FF04C0F3
:10B00000F7FAF094F7F8F094F7FAF094F7F8F09470
:10B01000C98ADA8AEB8AFC8A8CE0E8E8F2E0DE0191
:10B02000119601900D928A95E1F78AE50E946130B0
:10B03000882351F040E050E0BA018AE50E947C305C
:10B0400069877A878B879C8788E50E94613088238F
:10B0500051F040E050E0BA0188E50E947C306983FD
:10B060007A838B839C8389E50E946130882351F029
:10B0700040E050E0BA0189E50E947C306D837E8318
:10B080008F83988785E50E941330882309F489C04F
:10B090000E94E92F6B017C0120E030E0A901C7018B
:10B0A000B6010F94DF5B87FF04C0F7FAF094F7F85E
:10B0B000F094F7FAF094F7F8F094CD8ADE8AEF8AEC
:10B0C000F88E198E1A8E1B8E1C8E8CE40E94133003
:10B0D000882309F46FC00E94E92F6B017C0120E0F6
:10B0E00030E0A901C701B6010F94DF5B87FF04C000
:10B0F000F7FAF094F7F8F094CD8EDE8EEF8EF8A28A
:10B1000062E070E082E40E94C731F82E80914E0622
:10B11000811131C021E0AE014B5E5F4FBE016F5F18
:10B120007F4FCE0141960E945A56882321F16F2D00
:10B1300081E00E943C5782E50E946130882309F437
:10B1400042C00E94E52F40E050E060EA71E44D8784
:10B150005E876F87788B20914E06222361F08C01E9
:10B160002F2DAE01435F5F4FBE01635E7F4FCE0167
:10B1700049960E944154A0960FB6F894DEBF0FBEC8
:10B18000CDBFDF91CF911F910F91FF90EF90DF9096
:10B19000CF900895C12CD12C80E8E82E80E4F82EC1
:10B1A00033CFC090C605D090C705E090C805F09099
:10B1B000C90572CFC090CA05D090CB05E090CC05F0
:10B1C000F090CD058CCF90E080E0BDCFCF92DF92A4
:10B1D000EF92FF920F931F93CF93DF93CDB7DEB71C
:10B1E0006C970FB6F894DEBF0FBECDBF8CE40E9403
:10B1F0001330882309F4C3C00E94E92F6B017C013E
:10B2000020E030E0A9010F94DF5B87FF04C0F7FA6C
:10B21000F094F7F8F094F7FAF094F7F8F094C98EF8
:10B22000DA8EEB8EFC8E8CE0E8E8F2E0DE0111961F
:10B2300001900D928A95E1F788E50E94613088239C
:10B24000A1F040E050E0BA0188E50E947C302091F6
:10B250004F093091500940915109509152090F9472
:10B260007E5969837A838B839C8389E50E94613050
:10B270008823A1F040E050E0BA0189E50E947C30CB
:10B2800020914F0930915009409151095091520934
:10B290000F947E596D837E838F8398878AE50E9401
:10B2A0006130882351F040E050E0BA018AE50E9405
:10B2B0007C3069877A878B879C87F090C116F2FA79
:10B2C000FF24F0F840E061E080E00E94D38460E079
:10B2D00080E50E94D631E82E1D861E861F86188ABC
:10B2E00080914E0681113CC02E2DAE01435F5F4F11
:10B2F000BE016F5F7F4FCE0149960E945A56882348
:10B3000079F18091CE0581110F94D23FFF2011F089
:10B31000EE2031F160E080E00E943C57898D9A8DEB
:10B32000AB8DBC8DB0588D8B9E8BAF8BB88F198A2F
:10B330001A8A1B8A1C8A1D861E861F86188A80917F
:10B340004E06882369F010E000E020E0AE014B5E7D
:10B350005F4FBE016F5E7F4FCE010D960E9441543C
:10B360006C960FB6F894DEBF0FBECDBFDF91CF91C4
:10B370001F910F91FF90EF90DF90CF900895C12C17
:10B38000D12C80E8E82E80E4F82E45CF2F923F9212
:10B390004F925F926F927F928F929F92AF92BF92E5
:10B3A000CF92DF92EF92FF920F931F93CF93DF9391
:10B3B000CDB7DEB7E1970FB6F894DEBF0FBECDBFB5
:10B3C00089AB2091500828AB21E020935008809150
:10B3D000F6048D3409F463C4843511F40C94A96E19
:10B3E000873409F044C18091F4049091F5048A31C6
:10B3F000910509F4D7C108F03DC18430910508F0EA
:10B4000030C1209108088230910508F451C12130E3
:10B4100009F054C111E0029709F010E00E94933046
:10B4200019821A821B821C821D821E821F8218862C
:10B4300082E50E946130882309F453C10E94E92FFC
:10B440006B017C0120E030E0A9010F948D5288232C
:10B4500009F4EAC040909D1050909E1060909F109B
:10B460007090A0108091A1109091A210A091A310B3
:10B47000B091A41088A799A7AAA7BBA78090350868
:10B4800090903608A0903708B0903808809139081D
:10B4900090913A08A0913B08B0913C088CA79DA7D9
:10B4A000AEA7BFA7A5019401C301B2010F948D52AD
:10B4B00081110DC02CA53DA54EA55FA568A579A558
:10B4C0008AA59BA50F948D52882309F4ADC0A301D2
:10B4D0009201C501B4010F947E5920E030E040E0B4
:10B4E0005FE30F94F3526CA37DA38EA39FA328A5C3
:10B4F00039A54AA55BA56CA57DA58EA59FA50F9432
:10B500007E5920E030E040E05FE30F94F3522B01DE
:10B510003C0120E030E0A901C701B6010F948D5233
:10B52000881F8827881F181709F4D2C080E090E090
:10B53000A0E8BFEB88A799A7AAA7BBA72CA13DA10C
:10B540004EA15FA1CA01B9010F94F3524B015C01F6
:10B55000A3019201C301B2010F94F3529B01AC010C
:10B56000C501B4010F947F590F942D5C4B015C0110
:10B57000AC019B01C701B6010F947E596CA77DA752
:10B580008EA79FA7A5019401C701B6010F947F590B
:10B590009B01AC016CA57DA58EA59FA50F94F352D0
:10B5A0006B017C0120E030E0A9010F94DF5B87FD97
:10B5B00094C0C701B6010F942D5C6B017C01C301DF
:10B5C000B2019058A50194010F94795A28A539A584
:10B5D0004AA55BA50F94F352A70196010F94F3526D
:10B5E0002CA13DA14EA15FA10F947F5969837A835D
:10B5F0008B839C83A50194016CA17DA18EA19FA149
:10B600000F94795A28A539A54AA55BA50F94F35242
:10B61000A70196010F94F352A30192010F947F5951
:10B620006D837E838F83988720E030E0A901698154
:10B630007A818B819C810F948D52811166C020E0AC
:10B6400030E0A9016D817E818F8198850F948D52A4
:10B6500081115BC00E9468458EE09FE00E940E351C
:10B660002DC08430910509F463C0459739F10F94DA
:10B67000262C24C08A32910509F4ECC158F48C318F
:10B68000910509F4AAC008F490C04D9781F70E9473
:10B69000BD7114C08B35910509F459C28C359105E3
:10B6A00009F459C28A35910511F71092660806C04F
:10B6B000213021F40E9493300E94AEF639A9311155
:10B6C00002C00F94B43588A9809350080C94DE66AC
:10B6D00080E090E0A0E8BFE32DCFC12CD12C760113
:10B6E0006ECF89E40E946130882331F00E94E92FF7
:10B6F00069837A838B839C838AE40E9461308823E8
:10B7000009F492CF0E94E92F8BCF412FBE016F5FCA
:10B710007F4F85E398E00F944D360F945335609337
:10B720004508709346088093470890934808C6CF11
:10B7300080E50E946130C12CD12C7601882321F054
:10B740000E9460256B017C0183E50E9461308823A3
:10B7500061F00E94E92F20E030E04AE754E40F94C2
:10B76000F3520F94F25A6B017C010E94D6DC809157
:10B770006413811105C060E084E29FE00E9464B21E
:10B780000F945335C60ED71EE81EF91E0F9453357D
:10B790006C197D098E099F0997FF90CF80E00E9468
:10B7A0001F4CF4CF0E94183C89CF0F94B4428111F2
:10B7B00085CF8CE0E4E9F2E0DE01119601900D9274
:10B7C0008A95E1F770E060E080E50E946E30BE018E
:10B7D0006F5F7F4F0F946A0171CF87E00E9488F0FE
:10B7E000811106C060E08FE40E94D631811166CFDE
:10B7F0000E94D6DC1092380260919C108CE40E946A
:10B80000D631982E80E00E94CA320F94533560934F
:10B8100045087093460880934708909348088091A4
:10B82000790290917A02A0917B02B0917C02809380
:10B83000C3049093C404A093C504B093C60480913C
:10B840007302909174029093C2048093C10484E6C1
:10B8500090E0909374028093730281E08093C1071B
:10B860000E941BFC8AE50E941330A82E88E50E94E6
:10B870001330182F89E50E941330B82E181308C012
:10B88000B12EA11205C011E0BB24B394AA24A39445
:10B8900082E50E946130882309F4D2C00E94E92F1A
:10B8A0006C8F7D8F8E8F9F8F20E030E0A9010F94E9
:10B8B0008D52882349F0111103C0BB2009F494C0B4
:10B8C000CE014C960F94142E112309F488C0BB208E
:10B8D00009F482C010929D1010929E1010929F1039
:10B8E0001092A0101092A1101092A2101092A3100A
:10B8F0001092A4100E9471F2ECEBF7E2C590D59083
:10B90000E590F490E0ECF7E24590559065907490E6
:10B91000A7019601C301B2010F948D5287FF95C014
:10B92000A7019601C301B2010F94795A9B01AC01A2
:10B930000F94F35220E030E040E85FE30F947F592A
:10B940000F942D5C20E030E048E452E40F94F35271
:10B9500069837A838B839C838091A5109091A61034
:10B96000A091A710B091A8108CA39DA3AEA3BFA3D4
:10B9700020E030E040EC5FE3C301B2010F94F352EA
:10B980002B013C0177FA709477F8709420E030E056
:10B9900040EC5FE3C701B6010F94F3529058DE010B
:10B9A00011966D01ECA0FDA00EA11FA1A3019201B3
:10B9B0000E9471F10E9486FD10929D1010929E10BF
:10B9C00010929F101092A0101092A1101092A2102D
:10B9D0001092A3101092A41080E00E94C8F9BB201E
:10B9E00019F081E00E94C8F9AA2019F082E00E94B3
:10B9F000C8F90E9471F28091C0078093C107892D18
:10BA00000E94CA328091C3049091C404A091C504DD
:10BA1000B091C6048093790290937A02A0937B023E
:10BA2000B0937C028091C1049091C20490937402FF
:10BA30008093730283E080937D020E9419FB3ECEC7
:10BA400060E070E080E890E42BCFA3019201C70191
:10BA5000B6016ACF80910808813009F02FCE89E4C1
:10BA60000E946130082F10E0882319F00E94E52F12
:10BA7000182F8AE40E946130F82E882339F00E9442
:10BA8000E52F011106C0853068F005C080E0002375
:10BA900049F0153028F08DE29FE00E940E350ECE61
:10BAA000F110F1CF90E1EDE9F0E1A5E3B8E001900C
:10BAB0000D929A95E1F7002391F0B4E01B02F0019A
:10BAC0001124EE55F94E408151816281738140937A
:10BAD0003508509336086093370870933808FF2074
:10BAE00091F024E08202F0011124E257F94E8081A6
:10BAF0009181A281B3818093390890933A08A093F1
:10BB00003B08B0933C0840E050E0BA0186E40E9454
:10BB10007C306B017C0120E030E0A9010F94DF5BF9
:10BB200018168CF420E030E040E752E4C701B6017B
:10BB30000F94795A69837A838B839C83CE01019613
:10BB40000E9461F9BBCD60E070E0CB01F3CF8FE0E4
:10BB500080936608B3CD8091F304882381F1893006
:10BB600009F0ACCD60EAA62E62E0B62E7DE9C72EC4
:10BB700070E1D72EE12C00E010E0D5018D915D0140
:10BB80000E946130F82E882361F0133011F4082FE1
:10BB9000FE2C0E94E92FF6016083718382839383D8
:10BBA000EF2C1F5FF4E0CF0ED11C143031F7EE20E4
:10BBB00009F457C00E9471F20E9419FB7FCD50EA30
:10BBC000C52E52E0D52EF12CE12C00E010E0D6017C
:10BBD0008D916D010E946130382E8823D9F10E9429
:10BBE000E92F4B015C01133059F0F701E15BF64F8F
:10BBF00020813181428153810F947E594B015C0138
:10BC0000F701E356FF4E2081318142815381C50106
:10BC1000B4010F947E592B013C012DEB37E346E82C
:10BC200055EB0F94DF5B87FD0AC02DEB37E346E849
:10BC300055E3C301B2010F948D5218165CF4133012
:10BC4000C1F48092A9109092AA10A092AB10B09269
:10BC5000AC10032D1F5FB4E0EB0EF11C143009F0A3
:10BC6000B6CF002309F4A8CF89EA90E10E9470EED4
:10BC7000A3CFF701EB57F74F5F01A301920160815A
:10BC80007181828193810F947F59D5016D937D934A
:10BC90008D939C931397812F0E9468F0DBCF809146
:10BCA000F4049091F5048837910511F40C94EC6834
:10BCB00008F077C28D34910509F4ADC708F0D3C000
:10BCC0008A31910509F4CFC608F094C084319105FA
:10BCD00009F415C608F071C08131910509F4D6C583
:10BCE00008F044C0029708F0C2CC80E50E946130A1
:10BCF000C12CD12C7601882321F00E9460256B0194
:10BD00007C0183E50E946130882361F00E94E92F65
:10BD100020E030E04AE754E40F94F3520F94F25AD3
:10BD20006B017C010E94D6DC8091F7049091F804AD
:10BD3000009709F4A5C50F9460428091F404909196
:10BD4000F5046EE47FE0892B11F466E47FE030E0D7
:10BD500020E04EE650E482E00E941D3640E0C7013C
:10BD6000B6010E9400570F949242A8CC429709F066
:10BD70007ECC83E50E946130882311F40C94236803
:10BD80000F94533560934508709346088093470895
:10BD9000909348080E94E92F20E030E04AE754E4FD
:10BDA0000F94F3520F94F25A6093100270931102A1
:10BDB000809312029093130281CC8731910509F48C
:10BDC000D3C570F48531910509F4CAC5469709F0C9
:10BDD0004ECC8091C11682FD71CC0E9430D26ECCC7
:10BDE0008831910509F4D5C5499709F040CC0E94E6
:10BDF000E65864CC8F31910509F4DAC6D0F48C3161
:10BE0000910509F49DC608F441C68D31910509F4E8
:10BE10009FC64E9709F02BCC8091C11683FF4ECC64
:10BE20000F940C2C8091F7049091F8040F942F41FB
:10BE300045CC8934910509F4DAC650F48032910575
:10BE400009F48DC6819709F012CC0E945A4B36CC6A
:10BE50008B34910509F4DBC68C34910509F007CCCD
:10BE60000E948EFE2BCC8B36910509F4C0C708F0DA
:10BE70000FC18435910509F47CCF40F581359105DA
:10BE800011F40C94036890F48E34910509F0EFCB13
:10BE900070E060E083E50E94C7318E34910509F0BF
:10BEA000BFC60E94FCDB0F94924208CC82359105FC
:10BEB00011F40C941B688335910509F0D8CB80915F
:10BEC00066088F7E806280936608F8CB883691057D
:10BED00009F42AC708F09CC08535910511F40C942B
:10BEE00066688C35910509F0C2CB0E94554687FDE6
:10BEF000E5CB8091EF0484FD0AC08091F10487FDB9
:10BF000006C08091F204837011F40C94946820EAC6
:10BF1000C22E22E0D22E34E5E32E30E1F32E10E0E3
:10BF2000D6018D916D010E946130882309F466C0AD
:10BF3000133011F00C948B680E94E92F4B015C01C7
:10BF400020E030E040EA51E40F948D5287FF4EC06C
:10BF5000A501940160917410709175108091761014
:10BF6000909177100F94795A2B013C01AC019B0101
:10BF7000609181097091820980918309909184096F
:10BF80000F94F3526093810970938209809383091F
:10BF900090938409A301920160918410709185109F
:10BFA00080918610909187100F94F35260938410C3
:10BFB00070938510809386109093871060916D091F
:10BFC00070916E0980916F09909170090F9492524F
:10BFD000A30192010F94F3520F94F25A60936D09EA
:10BFE00070936E0980936F0990937009809274101A
:10BFF00090927510A0927610B09277101F5FF4E0C7
:10C00000EF0EF11C143009F08BCF0E94B2DC56CB3E
:10C010008936910509F4C0C68A36910509F027CB07
:10C0200080E50F94482DF82E81E08F1508F446CB5B
:10C0300081E40E94133060918D09062F10E0811178
:10C0400002C00FEF10E089E40E946130882311F4F0
:10C050000C94DB6E0E94C12F90E01816190614F4A0
:10C0600081E090E026E0289FF001299FF00D112447
:10C07000E75FF74F04811581EF2DF0E0E357F64FAE
:10C080000F3F110519F010F00FEF10E0008316CBF1
:10C090008137910509F40DC708F068C08E36910507
:10C0A00009F4B3C608F059C08C36910509F406CBE3
:10C0B0008D36910509F0DBCA8091531083FDFECACD
:10C0C0000E945546F82E87FDF9CA89E40E94613026
:10C0D000882311F40C94C96E0E94C12F90E01816A9
:10C0E000190614F481E090E026E0289FF001299FD2
:10C0F000F00D1124E75FF74F8081918110E00E94DD
:10C1000058DC61E081E00F94A1462091D515309173
:10C11000D6158091D3159091D415821793070CF002
:10C1200032C68FE390E19F938F938AE490E19F93CF
:10C130008F931F920E9449B20F900F900F900F9013
:10C140000F9001E00F946A46002309F4B7CA40E05B
:10C15000612F8F2D0F94380AB1CA8F36910509F4DB
:10C1600067C68037910509F4A9CA81CA8537910548
:10C1700009F4E7C758F48237910509F4DAC7833721
:10C18000910509F074CA0E94353598CA8637910521
:10C1900009F4E9C78737910509F069CA0E94FFFBD6
:10C1A0008DCA8039E1E09E0711F40C942B6C08F0E5
:10C1B000ECC18D3C910511F40C94F66908F0A6C011
:10C1C0008B39910509F4F8C640F58D37910509F4CE
:10C1D0000ECE58F48937910509F049CA1092C1076B
:10C1E0001092C0070E941BFC69CA8C38910509F4A3
:10C1F0007FC68139910509F03ACA70E060E083E5B5
:10C200000E94C731823010F40C94F4680E94684593
:10C2100080EA90E10E940E3551CA893C910511F4E3
:10C220000C946169B0F58E3B910509F487C6883C92
:10C23000910509F01CCA0E945546182F87FD3ECA79
:10C240000091840884E40E946130F82E8823C1F0B4
:10C250000E94E92F4B015C0120E030E0A9010F941E
:10C260008D52882311F40C945E6924E01202F001CF
:10C270001124E058F74F80829182A282B3820F2D61
:10C28000602F83E50E94D631809384080E94D1C339
:10C2900015CA8B3C910511F40C948B698C3C91056B
:10C2A00009F0E5C98091F00487FF02C00C94AE69E3
:10C2B0008091F1048E7011F00C94AE694091881059
:10C2C0005091891060918A1070918B1085EC90E1EB
:10C2D0000E94F83640918C1050918D1060918E1014
:10C2E00070918F1082EC90E10E94F836409190108E
:10C2F00050919110609192107091931089E79CE297
:10C300000E94F8368AE00E94D534D8C9823221E0F2
:10C31000920711F40C94676B80F58C3D910511F434
:10C320000C94CD6A60F48E3C910511F40C947D6AF6
:10C33000833D910509F09BC90E947A46BFC98D3D96
:10C34000910511F40C94106B8A3F910509F08FC987
:10C3500083E40E941330882321F00E94E52F0E947D
:10C360008A26609151027091520281E591E10E940A
:10C370000E3C8AE00E94D534A1C98E32A1E09A0712
:10C3800011F40C94E16B08F083C08C32E1E09E075D
:10C3900011F40C94C36B8D32914009F068C985E4A7
:10C3A0000F94482D81110C94D96B80E50E941330B5
:10C3B000882351F00E94E92F6093D8157093D91506
:10C3C0008093DA159093DB1589E40E94133088235B
:10C3D00081F00E94E92F2CEA35EC47E25EE30F94EE
:10C3E000F3526093DC157093DD158093DE15909306
:10C3F000DF1584E40E941330882381F00E94E92F26
:10C400002CEA35EC47E25EE30F94795A6093E0152D
:10C410007093E1158093E2159093E3150E945146C5
:10C420004091D8155091D9156091DA157091DB15AE
:10C430008FE291E10E94F8362CEA35EC47E25EE3A8
:10C440006091DC157091DD158091DE159091DF15FE
:10C450000F94795AAB01BC018BE291E10E94F8364E
:10C460002CEA35EC47E25EE36091E0157091E1154E
:10C470008091E2159091E3150F94F352AB01BC014A
:10C4800087E291E10E94F8368AE00E94D53416C90D
:10C490008F3221E0920711F40C94276C8033914085
:10C4A00009F0E5C880E50E941330882351F00E940E
:10C4B000E92F6093740870937508809376089093C1
:10C4C000770889E40E941330882381F00E94E92FC5
:10C4D0002CEA35EC47E25EE30F94F3526093780860
:10C4E0007093790880937A0890937B0884E40E9483
:10C4F0001330882381F00E94E92F2CEA35EC47E2C3
:10C500005EE30F94795A60937C0870937D08809362
:10C510007E0890937F080E94514640917408509184
:10C52000750860917608709177088DE491E10E941A
:10C53000F8362CEA35EC47E25EE3609178087091BA
:10C54000790880917A0890917B080F94795AAB0111
:10C55000BC0189E491E10E94F8362CEA35EC47E20F
:10C560005EE360917C0870917D0880917E089091D7
:10C570007F080F94F352AB01BC0185E491E10E9466
:10C58000F8368AE00E94D53499C8883FA1E09A071E
:10C5900011F40C945E6D08F047C08C3AE1E09E0700
:10C5A00011F40C94336CC8F48D3921E0920711F426
:10C5B0000C948C6E28F48A39914009F47FC857C8CE
:10C5C000843AB1E09B0711F40C942F6C853A9140AA
:10C5D00009F04DC80E946C4571C8853FF1E09F0786
:10C5E00011F40C94566D68F4863E31E0930711F413
:10C5F0000C94E46C843F914009F039C80E94A8D89B
:10C600005DC8863FB1E09B0711F40C945A6D873FDB
:10C61000914009F02CC861E083E50E94D63191E099
:10C6200089270F94C60B4AC88C36F3E09F0709F49C
:10C6300045C808F0D5C08B3532E0930711F40C944F
:10C64000816D70F48C30B2E09B0711F40C94706D26
:10C650008835924011F00C94375B0E94D6572EC853
:10C660008D3BF2E09F0711F40C94016E8E3B9240DB
:10C6700011F00C94375B0E945546182F87FD1EC899
:10C680008AE50E946130812C912C90E2A92E91E4E0
:10C69000B92E882341F040E050E0BA018AE50E94BB
:10C6A0007C304B015C01412F64E083E00E94D38425
:10C6B00020E030E0A901C501B4010F94DF5B18163A
:10C6C0007CF580E090E0A0EAB0E489839A83AB83B4
:10C6D000BC832091A5103091A6104091A7105091D5
:10C6E000A810C501B4010F947F596B017C0120E0B3
:10C6F00030E04AE753E40F948D5287FD06C0C12C09
:10C70000D12C8AE7E82E83E4F82ECC8EDD8EEE8ED7
:10C71000FF8EBE016F5F7F4FCE014C960E9429F2C3
:10C7200085E50E941330882311F40C94056E0E9455
:10C73000E92F6B017C0120E030E0A901C701B601BF
:10C740000F94DF5B87FF04C0F7FAF094F7F8F094DA
:10C75000F7FAF094F7F8F094C982DA82EB82FC825F
:10C7600044E061E0CE0101960E94AD5520E030E04A
:10C77000A901C501B4010F94DF5B18165CF580E0D8
:10C7800090E0A0EAB0E489839A83AB83BC83A501DF
:10C7900094016091A5107091A6108091A7109091BE
:10C7A000A8100F947E596B017C0120E030E0A901B4
:10C7B0000F94DF5B18161CF0C12CD12C7601CC8EA7
:10C7C000DD8EEE8EFF8EBE016F5F7F4FCE014C96E9
:10C7D0000E9429F2109209050E94EA830C945E5B84
:10C7E000873E33E0930711F40C947C6EC8F48438D0
:10C7F000B3E09B0711F40C94116E803A934011F052
:10C800000C94375B2091F7043091F8049091C11695
:10C8100092609093C116C9010F9409430C945E5B1A
:10C82000883EF3E09F0711F40C94A56E893E934077
:10C8300011F00C94375B0F94D94181110C945E5B1D
:10C840000E94EB310F9497410E9494FD6D33710566
:10C850008105910520F081E392E10E942F6F8DE226
:10C8600092E10E942F6F84EE8093010589E192E1AD
:10C870000E940E3585E192E10E942F6F0C945E5B61
:10C8800060E086E59FE00E9464B257CA8091EF04A1
:10C8900084FD17C08091F10487FD13C08091F204DC
:10C8A000837079F460E089E69FE00E9464B25F984B
:10C8B0008A988091080181708093060112980C94E7
:10C8C0005E5B88E50E94133081115F9889E50E94C4
:10C8D000133081118A988AE50E941330882329F049
:10C8E0008091080181708093060185E40E941330D5
:10C8F000882311F40C945E5B12980C945E5B80911B
:10C90000C11683FF25C081E89FE00E940E3580910B
:10C91000C11683FF17C082EE96E10E9414D38BE10B
:10C92000E2EEF6E1DE01119601900D928A95E1F7B3
:10C9300070E060E0CE0101960F94B506CE0101963D
:10C940000E94133282E79FE00E940E350C945E5BDA
:10C950000E94514682E99FE00E940E350C945E5B76
:10C960000E9441D20C945E5B8091F7049091F80490
:10C97000FC012191222331F02032D9F7DF011197F8
:10C980001C92F7CF60E00F945243109201050C9473
:10C990005E5B83E50E946130882321F00E9481253F
:10C9A0000E94B42384E50E9461308823A9F00E948C
:10C9B00081256B017C010E943BFEC092BE05D09296
:10C9C000BF05E092C005F092C105CD28CE28CF2842
:10C9D00019F081E08093650880914E068823F9F074
:10C9E00080E090E0A0EAB1E489839A83AB83BC83C2
:10C9F0001C8E1D8E1E8E1F8E18A219A21AA21BA29B
:10CA000010E000E020E0AE014F5F5F4FBE01645ECA
:10CA10007F4FCE0180960E9441540C945E5B0E9431
:10CA20005934882381F00E9489CA0E947D348BED9D
:10CA300098E00F94E840109296111092971110927E
:10CA400098111092991161E08EE19EE10E94D63515
:10CA500046EE5DE16CE97FE085E00F943F2D0F9499
:10CA600092420C945E5B8091C11683FD02C00C94CF
:10CA70005E5B83E50E946130882311F40C945E5B59
:10CA80000E9481250E94B4230C945E5B83E40E9483
:10CA90001330882361F182EB9FE00E940E35809174
:10CAA00029188823F9F0BE016F5F7F4F86E298E175
:10CAB0000E94A7D2CE0101960E94AECECE01019671
:10CAC0000F94324280912113882339F080E20E9432
:10CAD000D53481E293E10E94AECE8AE00E94D53443
:10CAE0000C945E5B88EA9FE00E940E35F6CF83E5EA
:10CAF0000E946130882301F10E94C12F182F8C33CE
:10CB000008F08CE38093CB040F9453356B017C01C8
:10CB1000212F30E0A8EEB3E00F942559C60ED71EA2
:10CB2000E81EF91EC092C704D092C804E092C9045E
:10CB3000F092CA040C945E5B0F94AF400C945E5B61
:10CB40008091F7049091F8040F9409430C945E5B74
:10CB50008091C1168E7F8093C1160C945E5B80918C
:10CB6000C11682FD0E94D6DC8091C11683FD02C0F1
:10CB70000C945E5B60E080E50E94D631182F682F30
:10CB80008091F7049091F8040F94524383E50E943A
:10CB90006130882321F00E9481250E94B4230E94E5
:10CBA00089CA11110C945E5B0E947D340C945E5B0B
:10CBB0000E9494FD6C8F7D8F8E8F9F8FBE016F5F63
:10CBC0007F4FCE014C960E94472ACE0101960F94CA
:10CBD00060420E945146BE016F5F7F4F81EC9FE033
:10CBE0000E94504B8AE00E94D5340C945E5B80E535
:10CBF0000E941330882311F40C945E5B0E94C12FB5
:10CC0000853608F084E6809301050C945E5B0E94F3
:10CC10007D340C945E5B81E00E94C6FD0C945E5BEB
:10CC20008CE290E10E940E356091B0077091B107DF
:10CC300083E290E10E94E6366091B2077091B307FB
:10CC400086E190E10E94E6366091B0077091B107ED
:10CC50008091B2079091B307681B790B80916508AA
:10CC6000815021E030E0823010F030E020E0621BA3
:10CC7000730B8BE090E10E94E6368AE00E94D53487
:10CC800083E090E10E940E358091B4079091B50742
:10CC9000A091B607B091B7078C8F9D8FAE8FBF8FD5
:10CCA000BE016F5F7F4FCE014C960E94472ABE01A6
:10CCB0006F5F7F4F86EF9FE00E94504B8091B807D7
:10CCC0009091B907A091BA07B091BB078C8F9D8F47
:10CCD000AE8FBF8FBE016F5F7F4FCE014C960E941B
:10CCE000472ABE016F5F7F4F86EE9FE00E94504B48
:10CCF00020E030E04AE754E46091BC077091BD0742
:10CD00008091BE079091BF070F94795AAB01BC0187
:10CD10008EEC9FE00E94F8368DE60E94D5348AE0C2
:10CD20000E94D5340C945E5B8091531083FF02C047
:10CD30000C945E5B0E94554687FF02C00C945E5BBC
:10CD400089E40E946130882311F40C94BE6E0E9425
:10CD5000C12F90E01816190614F481E090E026E047
:10CD6000289FF001299FF00D1124E75FF74F808184
:10CD700091810E9458DC61E080E00F94A1460F94FD
:10CD80006A460C945E5B84E390E1112309F4CBC9FD
:10CD9000012FD8C9182FD6C90E945546182F87FDD4
:10CDA0000AC08FE490E10E940E35812F0F94400855
:10CDB0008AE00E94D53438A930935008E1960FB626
:10CDC000F894DEBF0FBECDBFDF91CF911F910F91C1
:10CDD000FF90EF90DF90CF90BF90AF909F908F909B
:10CDE0007F906F905F904F903F902F90089580E5D7
:10CDF0000F94482D823010F00C945E5BE82FF0E029
:10CE0000E357F64F10820C945E5B8EE40E94613013
:10CE1000882311F40C945E5B0E94812560932F118E
:10CE20007093301180933111909332110C945E5BAA
:10CE300083E50E941330882329F083E50F94482D61
:10CE4000809353100E94514680E690E10E940E3577
:10CE500080915310882351F110E000E020E0809190
:10CE6000531090E0B0E0A0E0002E04C0B695A79566
:10CE7000979587950A94D2F780FF12C0FF24F39408
:10CE8000F20E222319F08CE20E94D534F801EE0F45
:10CE9000FF1FEA5AFF4E859194910E940E352F2D67
:10CEA0000F5F1F4F05301105D1F617CE82E590E1D7
:10CEB0001BCE83E50E946130882369F00E94C12F58
:10CEC0008D3320F480930F020C945E5B8CE380938F
:10CED0000F020C945E5B0E94514660910F0287E640
:10CEE00090E10E94F0368AE00E94D5340C945E5B9B
:10CEF0008091531083FF02C00C945E5B89E40E9412
:10CF00006130882309F463C70E94C12F90E018168E
:10CF1000190614F481E090E026E0289FF001299F93
:10CF2000F00D1124E75FF74F828193810E94B62FA5
:10CF300061E080E00F94A1460C945E5B80915310F9
:10CF400083FF02C00C945E5B89E40E9461308823F9
:10CF500009F447C70E94C12F90E01816190614F46F
:10CF600081E090E026E0289FF001299FF00D112438
:10CF7000E75FF74F8281938110E00E94B62F60E057
:10CF800081E00F94A1462091710830917208809140
:10CF90006F0890917008821793071CF48DE790E159
:10CFA00002C08EE690E160E00E9464B260E0812FF2
:10CFB0000F94B3080C945E5B83E50E946130882374
:10CFC00011F40C945E5B0E94C12F182F8C3308F073
:10CFD0008CE38093D0040F9453356B017C01212F97
:10CFE00030E0A8EEB3E00F942559C60ED71EE81E18
:10CFF000F91EC092CC04D092CD04E092CE04F092FF
:10D00000CF040C945E5B0E9431D50E94E7DC81E086
:10D010000E94C6FD0E94903468EE73E080E090E0CC
:10D020000E940A340E94C22160E08CE890E10E94D4
:10D0300064B20C945E5B809166088F7D8061809302
:10D0400066080C945E5B8091EF0484FD0CC08091B7
:10D05000F10487FD08C08091F204837021F40E94DE
:10D06000E7DC0C945E5B0E94D6DC88E50E941330FE
:10D07000882331F05F9A8091C3078E7F8093C30726
:10D0800089E50E941330882331F08A9A8091C30782
:10D090008D7F8093C3078AE50E941330882359F05F
:10D0A0008091080180958170809306018091C3076B
:10D0B0008B7F8093C30785E40E941330882311F48B
:10D0C0000C945E5B0E94C0210C945E5B83E50E9421
:10D0D0001330882311F40C945E5B0F9453356093E6
:10D0E00045087093460880934708909348080E942B
:10D0F000E92F20E030E04AE754E40F94F3520F9414
:10D10000F25A6093D1047093D2048093D304909325
:10D11000D4040C945E5B0E94E92FF701648B758B3D
:10D12000868B978B0C94FE5F81E00F94D12B0C942F
:10D130005E5B0F946C2B89E296E10E94FED70C9403
:10D140005E5B8091F7049091F804009741F0DC0158
:10D150002C91222321F00F9460420C945E5B0F947B
:10D1600092420C945E5B0091F7041091F80494E0F5
:10D17000F12C40E09150F9F0F8018081282F2B7FAD
:10D18000213499F421812133B1F4813411F18534B2
:10D1900009F441E098012E5F3F4F89012F5F3F4F17
:10D1A000F80180818032C9F3E5CF803521F4818197
:10D1B00080538A3078F341110E945146FF2021F0BC
:10D1C0008DE990E10E940E35C8010E94DC340C9478
:10D1D0005E5BFF24F394DECF2093C1072093C0074A
:10D1E0000E941BFC0C945E5B8C01112788E40E945A
:10D1F00061308823C1F00E94E52F8A3A91050CF432
:10D200004BC00E94E52F8D3291400CF048C00E9427
:10D21000E52F26E0209FF001219FF00D1124E75F0C
:10D22000F74F9183808382E40E9461308823A9F0C4
:10D230000E94E52F0597B4F10E94E52F8D389105E6
:10D24000A4F50E94E52F26E0209FF001219FF00D1C
:10D250001124E75FF74F9383828386E40E94613055
:10D26000882311F40C945E5B0E94E52F97FD20C08B
:10D270000E94E52F8F3F910509F0ECF40E94E52F05
:10D2800026E0209FF001219FF00D1124E75FF74F6A
:10D29000958384830C945E5B8AEA90E0BACF8CE23B
:10D2A00091E0B7CF85E090E0CECF8CE890E0CBCF97
:10D2B00090E080E0E5CF8FEF90E0E2CF80E00C944B
:10D2C00044610E94554687FF02C00C945E5B00EAF1
:10D2D00012E084E5E82E80E1F82E94EAC92E92E06F
:10D2E000D92ED8018D918D010E941330882359F0D9
:10D2F0000E94E92F0F94F25AF701608371838283B1
:10D3000093830E9464DCF4E0EF0EF11CC016D1069A
:10D3100041F70C945E5B0E94554687FF02C00C9457
:10D320005E5BB0EAEB2EB2E0FB2E10E000E0D7012E
:10D330008D917D010E941330882349F00E94E92FCE
:10D34000F801EC5AFF4E64A375A386A397A30C5F64
:10D350001F4F0031110559F70C945E5B83E50E9465
:10D360006130882391F00E94E92F609388107093B8
:10D37000891080938A1090938B1060939010709313
:10D380009110809392109093931080E50E946130E9
:10D39000882351F00E94E92F6093881070938910C0
:10D3A00080938A1090938B1082E50E9461308823CD
:10D3B00051F00E94E92F60938C1070938D10809330
:10D3C0008E1090938F1084E50E946130882311F4B1
:10D3D0000C945E5B0E94E92F609390107093911003
:10D3E00080939210909393100C945E5B8091EF0465
:10D3F000827151F48091F1048C7831F48091F204BF
:10D40000837011F40C945E5B82E40E9413308823D5
:10D4100051F00E94602560936410709365108093B2
:10D4200066109093671083E50E941330882351F0B3
:10D430000E94E92F6093941070939510809396103A
:10D440009093971084E50E941330882351F00E9436
:10D45000E92F609398107093991080939A1090938D
:10D460009B1088E50E941330882351F00E94E92F19
:10D470006093750970937609809377099093780982
:10D4800089E50E941330882351F00E94E92F6093B0
:10D49000790970937A0980937B0990937C098AE5D6
:10D4A0000E9413308823B1F00E94E92F60937D0918
:10D4B00070937E0980937F09909380092DEC3CEC5A
:10D4C0004CEC5DE30F948D52181624F085ED90E13D
:10D4D0000E940E3585E40E941330882311F40C94C9
:10D4E0005E5B0E94E92F60938109709382098093AB
:10D4F0008309909384090C945E5BA1E9EA2EA8E06D
:10D50000FA2E10E088E5810F0E941330882351F035
:10D510000E94E92FF7016083718382839383812FB7
:10D520000E9468F01F5FF4E0EF0EF11C133051F71A
:10D530008091F10487FF02C00C94DC5D8091F204BD
:10D54000837011F00C94DC5D409191085091920829
:10D55000609193087091940887E091E10E94F836F9
:10D56000409195085091960860919708709198089D
:10D5700087EF90E40E94F8364091990850919A08FC
:10D5800060919B0870919C0884EF90E40E94F836AB
:10D590008AE00E94D5340C945E5B82E40E941330D2
:10D5A000882341F080917302909174029093150248
:10D5B0008093140282E50E941330882341F0809109
:10D5C000140290911502909374028093730283E584
:10D5D0000E946130882331F00E94E52F90937402FD
:10D5E000809373028091EF049091F004A091F10474
:10D5F000B091F204892B8A2B8B2B11F00C945E5B7B
:10D6000060917302709174028EE091E10E940E3C71
:10D6100085E20E94D5348AE00E94D5340C945E5B8A
:10D620000E945546082F87FF02C00C945E5B83E57D
:10D630000E946130002E000C110B7801EE0CFF1CD3
:10D64000882359F10E94E52FF701EB5CFD4F918390
:10D650008083000F111F000F111F980122583D4FAA
:10D660007901BC01990F880B990B0F9494522AE011
:10D6700037ED43E25CE30F94F35206541A4FD8019E
:10D680002D913D914D915C910F94F352F701608380
:10D690007183828393830C945E5B0E94514685E480
:10D6A0000E94D53480E3800F0E94D534F701EB5CF3
:10D6B000FD4F6081718182E191E10E940E3C85E223
:10D6C0000E94D5348AE00E94D5340C945E5B8AE5D2
:10D6D0000E946130882331F10E94E92F20E030E080
:10D6E00040E050EC0F948D5287FD3CC00E94E92F22
:10D6F00020E030E040E050E40F94DF5B1816BCF10E
:10D700000E94E92F20917010309171104091721099
:10D71000509173100F94F3520F94EB5ACB010F9466
:10D72000073605C083E50E9461308111D5CF809115
:10D73000F10487FD21C08091F2048370E9F40E9416
:10D7400051464091330650913406609135067091F0
:10D7500036068AE191E10E94F8368AE00E94D534CB
:10D760000C945E5B60E070E080E090ECCBCF60E01A
:10D7700070E080E090E4C6CF82E50E941330811112
:10D78000DECF0C945E5B64E071E083E50E946E3056
:10D790008C0168EE73E080E50E946E308938F3E119
:10D7A0009F0710F088E893E1B8010E942E7D0C9449
:10D7B0005E5B0E94684583E391E10E940E350C9404
:10D7C0005E5B83E50E941330182F882369F00E9466
:10D7D000E52F9C01909383028093820291E0232B9A
:10D7E00009F090E090939F0980E50E941330882310
:10D7F00061F02091820230918302232B11F00E946C
:10D80000D52F80939F090C945E5B11110C945E5B85
:10D810000E9451468CE791E10E940E3580919F094C
:10D82000882391F084E691E10E940E356091820296
:10D83000709183028BE691E10E940E3C87E691E1B4
:10D840000E940E350C945E5B80E691E1EDCF0E9464
:10D850001A370C945E5B0E94D6DC0C945E5B0E94CF
:10D8600069470C945E5B0F94B44281110C945E5B2B
:10D870007BE8C72E77E2D72E2DE930E13DA32CA31C
:10D88000CE0101961C017C0110E000E0F6016591DB
:10D89000759185919491ACA1BDA18D909D90AD9015
:10D8A000BD90BDA3ACA3A50194010F947E592B019B
:10D8B0003C01F701408251826282738220E030E0B5
:10D8C00040EA51EC0F94DF5B87FD0AC020E030E0B6
:10D8D00040EA51E4C301B2010F948D52181684F44A
:10D8E000F801E25DFF4BE4911E1654F4B7FAB094D0
:10D8F000B7F8B094D7018D929D92AD92BC921397D8
:10D90000F70181909190A190B1907F0120E030E0EB
:10D9100040EA51ECC501B4010F94DF5B87FD3FC0C5
:10D9200020E030E040EA51E4C501B4010F948D528B
:10D930001816ACF10F5F1F4FF4E0CF0ED11C03306F
:10D94000110509F0A3CF61E9E62E68E0F62E10E09C
:10D95000F10181919191A191B1911F01F701819301
:10D960009193A193B1937F01812F0E9468F01F5F73
:10D97000133071F70E9419FB60E08FE891E10E947B
:10D9800064B263E972E084E690E00E942E7D6AEB67
:10D9900072E084E690E00E942E7D0C945E5B0E9413
:10D9A00068458DEA91E10E940E3561E08FE991E1D1
:10D9B0000E9464B20E94EA8368E270E088EC90E022
:10D9C0000E942E7D0C945E5B84E50E9413308823B8
:10D9D000A1F0109203051092040510920505109213
:10D9E0000605109207058FEF0E94C22361E070E0E8
:10D9F00084E50E94C7318093070583E50E941330B8
:10DA0000882321F00E94E52F0E94C22383E40E9414
:10DA10001330882331F080912302803210F40E9469
:10DA20008E3280E50E941330882331F00E94E52F6A
:10DA3000803210F40E948E3285E50E9413308823D4
:10DA400011F40C945E5B0E94E52F803210F00C9470
:10DA50005E5B41E050E060E070E0082E04C0440FDF
:10DA6000551F661F771F0A94D2F740955095609511
:10DA700070950091030510910405209105053091E2
:10DA800006054023512362237323409303055093DB
:10DA90000405609305057093060590912302891390
:10DAA0000C945E5B109252100C945E5B0F94ED121E
:10DAB0000C945E5B0E9426FC0C945E5B2093370600
:10DAC0000F94E11210923706882311F40C945E5BD8
:10DAD0000E9451468BEC91E10E940E350C945E5BE6
:10DAE0008091C11682FF05C080648093C1160C949A
:10DAF0005E5B83FD02C00C945E5B0F940C2C0C9457
:10DB00005E5B0E945546082F87FF02C00C945E5B47
:10DB100085E50E941330882359F10E94E92F4B01BB
:10DB20005C01E02E002E000CFF0820E030E0A9018F
:10DB30000F94DF5B87FF04C0B7FAB094B7F8B094D6
:10DB400020E030E84BE354E4C501B4010F94DF5BFF
:10DB5000970153E0220F331F5A95E1F72A533A4FAA
:10DB60001816D4F1D9018D929D92AD92BC92139763
:10DB70008CE40E941330882311F40C945E5B0E94A5
:10DB8000E92F6B017C01002E000C110B20E030E02E
:10DB9000A9010F94DF5B87FF04C0F7FAF094F7F850
:10DBA000F09420E030E84BE354E4C701B6010F9451
:10DBB000DF5B980143E0220F331F4A95E1F72A53B8
:10DBC0003A4F18169CF0D9011496CD92DD92ED9241
:10DBD000FC9217970C945E5B80E090E8ABE3B4E4B2
:10DBE000F90180839183A283B383C2CF80E090E860
:10DBF000ABE3B4E4F90184839583A683B7830C94E3
:10DC00005E5B0E9448530C945E5B28E01202F001B8
:10DC10001124EA53FA4FC080D180E280F3800C9443
:10DC20009B63A0908509B0908609C0908709D09029
:10DC300088098BE40E946130882339F10E94E92F22
:10DC40007B018C0120E030E0A9010F94DF5B87FDB0
:10DC50000AC020E030E040E251E4B701C8010F946F
:10DC60008D521816A4F48FE30E94D5348BE40E94E1
:10DC7000D53481EE91E10E940E3589ED91E10E944B
:10DC80000E3586ED91E10E940E35750186019701F2
:10DC9000A801B501C6010F948D52882361F00E943E
:10DCA000D6DCC701D8018093850990938609A0939B
:10DCB0008709B09388098091EF049091F004A091B6
:10DCC000F104B091F204892B8A2B8B2B11F00C9468
:10DCD0005E5B0E9451464091850950918609609192
:10DCE00087097091880985EF91E10E94F8368AE0F2
:10DCF0000E94D5340C945E5B81E0809308081092FA
:10DD0000B91360E083E50E94D63181110C945E5B0B
:10DD10000F94132A0C945E5B83E50E9413308823D2
:10DD200041F00E94D52F8093CE050E94F3310C94D0
:10DD30005E5B0E94514680E092E10E940E35809128
:10DD4000CE050E94DA360C945E5B0E94A16F0C94A3
:10DD50005E5B1091F4040F94533560934508709303
:10DD600046088093470890934808112311F40C94B7
:10DD70005E5B812F0E94E7D40C945E5B83E50E947A
:10DD80006130882311F40C94BF660E94E52F0C9437
:10DD9000B96683E50E946130182F811108C082E5C1
:10DDA0000E946130082F882311F40C94CA660E94E7
:10DDB000E52F0C947F6083E50E946130882311F485
:10DDC0000C943C600E9481258B010C943C6083E59F
:10DDD0000E946130882311F40C945E5B0E94E52F51
:10DDE000A5C883E50E946130182F811107C082E524
:10DDF0000E946130882311F40C945E5B0E94E52F31
:10DE0000BCC8DF92EF92FF920F931F93CF93DF93E3
:10DE1000EC01E0905208F09053088AE0D82E6AE0B6
:10DE200070E0CE010F94CD5C8C01009711F0FC01E5
:10DE30001082CE010E94262B81E00E94C659011556
:10DE4000110519F0E801D992EACFC701DF91CF910E
:10DE50001F910F91FF90EF90DF900C94262B4F9223
:10DE60005F926F927F928F929F92AF92BF92CF926A
:10DE7000DF92EF92FF920F931F93CF93DF93CDB773
:10DE8000DEB77C014DB65EB66090520870905308C4
:10DE90008DB69EB66AE070E0C7010F94C8516C0160
:10DEA0008C010E191F09892B21F4C7010F94DA5137
:10DEB0008C01C80101962DB73EB7281B390B0FB650
:10DEC000F8943EBF0FBE2DBF8DB79EB701965C0183
:10DED000A801B7010F94FB51F501E00FF11F10826B
:10DEE000C5010E94262B81E00E94C659C114D104AD
:10DEF00051F076019FEFE91AF90A0FB6F8949EBE29
:10DF00000FBE8DBEC5CF0FB6F8949EBE0FBE8DBEA0
:10DF1000C3010E94262B0FB6F8945EBE0FBE4DBE05
:10DF2000DF91CF911F910F91FF90EF90DF90CF90F5
:10DF3000BF90AF909F908F907F906F905F904F9029
:10DF400008954F925F926F927F928F929F92AF92BD
:10DF5000BF92CF92DF92EF92FF920F931F93CF93D6
:10DF6000DF93CDB7DEB7C059D1090FB6F894DEBF45
:10DF70000FBECDBF0E940132882369F083E50E9465
:10DF80001330882301F120E040E070E060E084E19C
:10DF900094E80E94D67FC057DF4F0FB6F894DEBFDB
:10DFA0000FBECDBFDF91CF911F910F91FF90EF90EA
:10DFB000DF90CF90BF90AF909F908F907F906F90A9
:10DFC0005F904F90089583E40E941330882319F0E6
:10DFD0000E940984E0CF8090440990904509A09068
:10DFE0004609B090470980914D0980FF05C0909186
:10DFF00053109860909353108695817080939F0979
:10E0000080EF9EE00E942F6F8091D3089091D408FA
:10E010009E012F5F3F4F7901009799F09F938F9357
:10E0200087EE9EE09F938F933F932F930F942452FC
:10E03000C7010E94016F0F900F900F900F900F90EB
:10E040000F908091D1089091D208009799F09F93FA
:10E050008F938EED9EE09F938F93FF92EF920F949C
:10E060002452C7010E94016F0F900F900F900F90E4
:10E070000F900F906E0131E8C30ED11C6091B00873
:10E080007091B1088091B2089091B308860123E0A5
:10E0900041E00F945A4D9F938F938CEC9EE09F9399
:10E0A0008F93FF92EF920F942452C7010E94016F49
:10E0B00084EC9EE00E942F6F87E08093C3078093DB
:10E0C000B1050F900F900F900F900F900F908091CF
:10E0D000CC088823F9F06091CD087091CE0880912A
:10E0E000CF089091D00823E041E00F945A4D9F93C0
:10E0F0008F938BEB9EE09F938F93FF92EF920F9401
:10E100002452C7010E94016F0F900F900F900F9043
:10E110000F900F908091D5088823A1F01F928F93C4
:10E120001F921F928EEA9EE09F938F93FF92EF9231
:10E130000F942452C7010E94016F0FB6F894DEBFFE
:10E140000FBECDBF8091D6088823A9F01F928F9370
:10E150001F9281E08F938EEA9EE09F938F93FF92B0
:10E16000EF920F942452C7010E94016F0FB6F894EA
:10E17000DEBF0FBECDBF4090D7085090D80860904A
:10E18000D9087090DA0820E030E0A901C301B2019B
:10E190000F948D52811104C080914D0982FF20C0DF
:10E1A000860121E041E0C301B2010F945A4D9F93D3
:10E1B0008F9380914D0982FB882780F91F928F935E
:10E1C00081EA9EE09F938F93FF92EF920F942452E7
:10E1D000C7010E94016F0FB6F894DEBF0FBECDBF1E
:10E1E0006091A2087091A3088091A4089091A5085D
:10E1F0008E010F581F4F23E041E00F945A4D782EA7
:10E20000692E60919E0870919F088091A00890915E
:10E21000A108860123E041E00F945A4D6F927F924E
:10E220009F938F9380E99EE09F938F93FF92EF924D
:10E230000F942452C7010E94016F6091A60870914B
:10E24000A7088091A8089091A90823E041E00F94C5
:10E250005A4D85E89EE00E942F6FDF92CF928BE7A8
:10E260009EE09F938F93FF92EF920F942452C701E9
:10E270000E94016F8091AF088F938091AE088F93B9
:10E2800084E79EE09F938F93FF92EF920F94245226
:10E29000C7010E94016F6091AA087091AB0880913C
:10E2A000AC089091AD0823E041E00F945A4D9F9344
:10E2B0008F938AE69EE09F938F93FF92EF920F9445
:10E2C0002452C7010E94016F8CE0E4EBF8E0A1E961
:10E2D000B8E001900D928A95E1F78CE0E0ECF8E06F
:10E2E000A5E8B8E001900D928A95E1F780E00E94E0
:10E2F00068F081E00E9468F082E00E9468F08091FE
:10E300004C098093660881E08093CE050E94F3312A
:10E310008BED98E09F938F938BEB97E39F938F9375
:10E32000FF92EF920F9424520FB6F894DEBF0FBE07
:10E33000CDBFC7010E94016F80914B098F938091DF
:10E340004A098F93809149098F93809148098F934F
:10E35000BF92AF929F928F928CE59EE09F938F9396
:10E36000FF92EF920F942452C7010E94016F0FB6E3
:10E37000F894DEBF0FBECDBF0ECE4F925F926F926C
:10E380007F928F929F92AF92BF92CF92DF92EF9245
:10E39000FF920F931F93CF93DF9300D000D01F9273
:10E3A0001F92CDB7DEB783E50F94482D863028F055
:10E3B00083EE9DE00E940E353FC0833009F464C1B6
:10E3C000B0F4813021F1823009F450C080ED9DE03D
:10E3D0000E940E350E94C5338823A1F080919C10C5
:10E3E0000E94DA360E945B360E9419FB25C08430F9
:10E3F00009F490C1853051F780E00E94CA320E9432
:10E40000BA32F2CF82EC9DE00E940E35EDCF0E9431
:10E41000BA3210920E0210920D0280910205811103
:10E4200025C08EE40E94133081111DC080EB9DE059
:10E430009093C6078093C50728960FB6F894DEBF61
:10E440000FBECDBFDF91CF911F910F91FF90EF9045
:10E45000DF90CF90BF90AF909F908F907F906F9004
:10E460005F904F90089586EB9DE0E2CF80910D0282
:10E4700090910E0297FF03C087E89DE09BCF009725
:10E4800009F0A8C01D821E821F8218868DEC9CECAC
:10E49000ACE4BEE389839A83AB83BC83BE016B5F2C
:10E4A0007F4FCE0101960E9429F280910D0290913A
:10E4B0000E02893191050CF0B3C021E0209338029F
:10E4C0009C012F5F3F4F30930E0220930D0265E0B9
:10E4D0000F94405980FF03C024E0291B922F24E0B1
:10E4E0009202F0011124EE55F94E80809180A280B5
:10E4F000B38094E08902F0011124E257F94E408084
:10E500005180628073808DEC9CECACE4BEE38D8323
:10E510009E83AF83B88719821A821B821C82CE0128
:10E5200001966C01E12CF12C00EA10E4A3019201A8
:10E53000C501B4010E9471F119821A821B821C82EA
:10E54000B601CE0105960E9429F280929D1090920C
:10E550009E10A0929F10B092A0104092A1105092D5
:10E56000A2106092A3107092A41010920205009164
:10E570000D0210910E0289E1E82EF12C09311105EE
:10E580000CF47801B70180E29DE00E940E3C69E145
:10E5900070E08BE19DE00E940E3C8AE00E94D53441
:10E5A000101611060CF020CF1F9289E18F93FF9275
:10E5B000EF9284E09DE09F938F9382E19DE09F9393
:10E5C0008F931F920E9449B20FB6F894DEBF0FBE20
:10E5D000CDBF0ACF815065E00F94405980FF03C042
:10E5E00024E0291B922F25E09202F0011124E80F6C
:10E5F000F11D87FDFA95EE0FFF1FEE0FFF1FE15390
:10E60000FA4F8091A5109091A610A091A710B091FB
:10E61000A81080839183A283B3831092380245CFE0
:10E6200080E090E0A0EAB0E48093A5109093A6105B
:10E63000A093A710B093A81089E792E00E9456F12A
:10E640000E94D6DC8FEF9FEF90930E0280930D0215
:10E6500083E79DE00E940E3581E69DE00F946042C5
:10E6600063E972E084E690E00E942E7D6AEB72E03E
:10E6700084E690E00E942E7D8BE59DE00E942F6F46
:10E6800081E00E94CA3271CF89E40E946130882300
:10E6900071F00E94E52F182F853068F064E070E07B
:10E6A00088E49DE00E940E3C85E49DE083CE8AE4F0
:10E6B0000E94D035C1CE8AE40E9461308823B9F32C
:10E6C0000E94E52F082F853048F064E070E082E377
:10E6D0009DE00E940E3C8FE29DE06CCE8AE50E9498
:10E6E00061308823A9F00E94E92F25E01202F00191
:10E6F0001124E00FF11D07FDFA95EE0FFF1FEE0F3D
:10E70000FF1FE153FA4F60837183828393836CCE42
:10E710008AE5CECF8AE50E9461308823C9F30E9442
:10E72000E92F6093330670933406809335069093F7
:10E7300036065ACECF93DF93C0919B11C0936009E8
:10E7400081E6C89FE0011124C356DE4E809153102C
:10E7500080FF05C00E945146CE010E94DC34CE01EC
:10E760000E94262B80E0DF91CF910C94C6598F92A6
:10E770009F92AF92BF92CF92DF92EF92FF92CF9390
:10E780006B017C0120E030E0A9010F948D5287FFDE
:10E79000A3C06DEB77E386E095EBA70196010F949C
:10E7A0007F596B017C0120E030E040E251E40F949E
:10E7B000F35220E030E048EC52E40F94F3524B0166
:10E7C0005C0120E030E040E251ECC701B6010F945B
:10E7D0008D52181654F420E030E048EC52E4C701A2
:10E7E000B6010F94DF5B87FD8BC020E030E0A9010C
:10E7F000C701B6010F948D5287FF73C060E070E0CF
:10E8000080EA90ECA50194010F947F5920E030E05C
:10E8100040E251E40F94795A0F94EB5A6B017C015A
:10E82000F7FC64C020E137E240E050E00F94F35879
:10E83000CA01B9012AE030E040E050E00F94F358FB
:10E84000605D6093AA05C701B60128EE33E040E0A1
:10E8500050E00F94F3589AE0892E912CA12CB12C02
:10E86000CA01B901A50194010F94F358605D60934A
:10E87000AB05C701B60124E630E040E050E00F945C
:10E88000F358CA01B901A50194010F94F358605DD2
:10E890006093AC058EE28093AD05C701B601A5017A
:10E8A00094010F94F358C62FCA01B901A501940130
:10E8B0000F94F358605D6093AE05C05DC093AF05E3
:10E8C0008AEA95E0CF91FF90EF90DF90CF90BF90D4
:10E8D000AF909F908F9008956DEB77E386E095E37E
:10E8E0005CCF60E070E080EA90E48CCFF094E0943C
:10E8F000D094C094C11CD11CE11CF11C6DE2A1CFCD
:10E9000020E030E0A901C701B6010F948D5287FFC6
:10E910006AC060E070E080EA90ECA50194010F9479
:10E920007F5920E030E040E251E40F94795A0F948F
:10E93000EB5A4B015C0120E030E0A901C701B601B0
:10E940000F94DF5B87FD0BC020E030E040E251E434
:10E95000C701B6010F948D5260E287FD13C0B7FC6A
:10E9600047C0C501B40128EE33E040E050E00F9409
:10E97000F358CA01B9012AE030E040E050E00F94BA
:10E98000F358605D6093AB05C501B40124E630E047
:10E9900040E050E00F94F3588AE0C82ED12CE12CCF
:10E9A000F12CCA01B901A70196010F94F358605DDB
:10E9B0006093AC058EE28093AD05C501B401A7015B
:10E9C00096010F94F358C62FCA01B901A701960109
:10E9D0000F94F358605D6093AE05C05DC093AF05C2
:10E9E0008BEA95E06FCF60E070E080EA90E495CF2D
:10E9F000B094A09490948094811C911CA11CB11C93
:10EA00006DE2C0CF6091350270913602072E000C86
:10EA1000880B990B0F9494522AE037ED43E25CE3A4
:10EA20000F94F3522091BA053091BB054091BC057B
:10EA30005091BD050F94F35260937E0270937F0254
:10EA400080938002909381020895E0913008E23033
:10EA500030F4F0E0E357F64F809126088083089564
:10EA60008091B6168823C1F081508093B616E2EEED
:10EA7000F6E1882351F08150990B2BE1289FF0019A
:10EA8000299FF00D1124E85EF84E8BE1ADEFB6E161
:10EA900001900D928A95E1F72091B616211105C0DB
:10EAA0008091C11680628093C11681E090E0A0E061
:10EAB000B0E0211103C080E090E0DC0180931E08EB
:10EAC00090931F08A0932008B09321081092230868
:10EAD00081E080931D0883E080937D020895CF93A9
:10EAE000DF93EC01CB01BA010F94945229EC38EC7E
:10EAF00048EC5EE30F94795A20E030E040E05FE3B9
:10EB00000F947F590F94F25A6883DF91CF91089543
:10EB100080915102909152020C948A26E091300823
:10EB200086E0E802F0011124E75FF74F80912608A4
:10EB300090E0958384830895CF93DF93EC01CB011C
:10EB4000BA010F94945220E030E0A9010F947F594C
:10EB50000F94F25A6883DF91CF9108958F929F921C
:10EB6000AF92BF92CF92DF92EF92FF92CF936B0161
:10EB70007C0120E030E0A9010F948D5287FD9FC0F9
:10EB80006DEB77E386E095E3A70196010F947F593B
:10EB90006B017C0120E030E040E251E40F94F3523D
:10EBA00020E030E048EC52E40F94F3524B015C015A
:10EBB00020E030E0A901C701B6010F948D5220E09A
:10EBC00030E040EA50E487FF04C020E030E040EA53
:10EBD00050ECC501B4010F947F5920E030E040E2D1
:10EBE00051E40F94795A0F94EB5A6B017C018BE23C
:10EBF000F7FE09C0F094E094D094C094C11CD11CDD
:10EC0000E11CF11C8DE28093A905C701B60120E14A
:10EC100037E240E050E00F94F3588AE0882E912CC0
:10EC2000A12CB12CCA01B901A50194010F94F3588C
:10EC3000605D6093AA05C701B60128EE33E040E0AD
:10EC400050E00F94F358CA01B901A50194010F9443
:10EC5000F358605D6093AB05C701B60124E630E070
:10EC600040E050E00F94F358CA01B901A5019401A6
:10EC70000F94F358605D6093AC058EE28093AD0510
:10EC8000C701B601A50194010F94F358C62FCA011C
:10EC9000B901A50194010F94F358605D6093AE052E
:10ECA000C05DC093AF0589EA95E0CF91FF90EF90EA
:10ECB000DF90CF90BF90AF909F908F9008956DEBB5
:10ECC00077E386E095EB60CF8F929F92AF92BF92F1
:10ECD000CF92DF92EF92FF92CF936B017C0120E005
:10ECE00030E0A9010F948D5287FDAAC06DEB77E348
:10ECF00086E095E3A70196010F947F596B017C0193
:10ED000020E030E0A9010F948D5287FF9EC0C7011B
:10ED1000B601905820E030E040E251E40F94F35205
:10ED200020E030E040E251E40F94F35220E030E084
:10ED300040EA50E40F947F5920E030E040E251E493
:10ED40000F94795A0F94EB5A6B017C0180E2809307
:10ED5000A90560E280E1C81687E2D806E104F10463
:10ED60008CF0C701B60120E137E240E050E00F949B
:10ED7000F358CA01B9012AE030E040E050E00F94B6
:10ED8000F358605D6093AA0560E288EEC81683E0E0
:10ED9000D806E104F1048CF0C701B60128EE33E097
:10EDA00040E050E00F94F358CA01B9012AE030E086
:10EDB00040E050E00F94F358605D6093AB0560E273
:10EDC00084E6C816D104E104F1048CF0C701B60151
:10EDD00024E630E040E050E00F94F358CA01B90156
:10EDE0002AE030E040E050E00F94F358605D60931B
:10EDF000AC058AE0882E912CA12CB12CC701B6015C
:10EE0000A50194010F94F358C62FCA01B901A501B9
:10EE100094010F94F358605D6093AD058EE280938A
:10EE2000AE05C05DC093AF0589EA95E0CF91FF9034
:10EE3000EF90DF90CF90BF90AF909F908F9008950C
:10EE40006DEB77E386E095EB55CF20E030E040E2D4
:10EE500051E4C701B60162CFCF93DF93EC01CB0140
:10EE6000BA010F94945220E030E040E251E40F9454
:10EE7000795A20E030E0A9010F947F5968837983A3
:10EE80008A839B83DF91CF910895CF93DF93EC0129
:10EE9000CB01BA010F94945220E030E040E251E4FB
:10EEA0000F94795A20E030E0A9010F947F596883CC
:10EEB00079838A839B83DF91CF9108950F94945235
:10EEC00020E030E040E251E40F94795A20E030E055
:10EED000A9010F947F590C946476CF93DF93EC01D2
:10EEE000CB01BA010F94945220E030E0A9010F94B5
:10EEF0007F59688379838A839B83DF91CF910895BB
:10EF0000CF93DF93EC01CB01BA010F94945220E030
:10EF100030E0A9010F947F59688379838A839B83AA
:10EF2000DF91CF910895CF93DF93EC01CB01BA012C
:10EF30000F9494522AE037ED43E25DE30F94795A3F
:10EF400020E030E0A9010F947F590F94F25A6883B2
:10EF500079838A839B83DF91CF910895CF93DF9349
:10EF6000EC01CB01BA010F9494522AE037ED43E251
:10EF70005DE30F94795A20E030E0A9010F947F59A6
:10EF8000688379838A839B83DF91CF910895CF93A0
:10EF9000DF93EC01CB01BA010F94945220E030E0F2
:10EFA000A9010F947F59688379838A839B83DF91BA
:10EFB000CF910895CF93DF93EC01CB01BA010F9469
:10EFC000945220E030E048EC52E40F94795A20E06B
:10EFD00030E0A9010F947F59688379838A839B83EA
:10EFE000DF91CF910895CF93DF93EC01CB01BA016C
:10EFF0000F94945220E030E048EC52E40F94795A98
:10F0000020E030E0A9010F947F59688379838A83D7
:10F010009B83DF91CF9108950F94945220E030E0CC
:10F0200048EC52E40F94795A20E030E0A9010F94A3
:10F030007F590C94AE75CF93DF93EC01CB01BA01ED
:10F040000F94945220E030E0A9010F947F590F945F
:10F05000EB5A79836883DF91CF910895CF93DF9343
:10F06000EC01CB01BA010F94945220E030E04AE762
:10F0700054E40F94795A20E030E0A9010F947F59AD
:10F08000688379838A839B83DF91CF9108950F945E
:10F09000945220E030E048EC52E40F94795A20E09A
:10F0A00030E0A9010F947F590C94B7732CEA35EC2A
:10F0B00047E25EE36091970570919805809199050C
:10F0C00090919A050F94795A6093E0157093E11529
:10F0D0008093E2159093E31508952CEA35EC47E20E
:10F0E0005EE360919B0570919C0580919D059091D8
:10F0F0009E050F94F3526093DC157093DD15809399
:10F10000DE159093DF1508952CEA35EC47E25EE3B7
:10F1100060919705709198058091990590919A0555
:10F120000F94795A6093E0157093E1158093E2157E
:10F130009093E31508952CEA35EC47E25EE3609185
:10F140009B0570919C0580919D0590919E050F9463
:10F15000F3526093DC157093DD158093DE15909368
:10F16000DF150895E0919005E63010F581E08E0FEF
:10F170008093900540911E0850911F0860912008CF
:10F18000709121089091230880911C0828E0E29F4B
:10F19000F0011124EF5AFA4F20914D1630914E167E
:10F1A000318320834283538364837583968387836B
:10F1B0000895FC01A081B1811C92A281B3818C9140
:10F1C0008F5F8C930280F381E02D90818CE0989F7B
:10F1D000800D1124EFE4F6E113AE84AF0895CF92D1
:10F1E000DF92EF92FF92CF93DF9300D01F92CDB7C3
:10F1F000DEB76B017C0120E030E0A9010F948D5255
:10F2000087FD1CC06DEB77E386E095E3A7019601CF
:10F210000F947F5969837A838B839C8360E2CE014C
:10F2200001960E9426FF0F900F900F900F90DF9194
:10F23000CF91FF90EF90DF90CF9008956DEB77E343
:10F2400086E095EBE3CF0F94945220E030E04AE75C
:10F2500054E40F94795A20E030E0A9010F947F59CB
:10F260000C94EF78CF92DF92EF92FF926B017C01CA
:10F2700020E030E0A9010F948D5287FD26C06DEB90
:10F2800077E386E095E3A70196010F947F596B0120
:10F290007C0120E030E0A9010F948D5220E030E0A5
:10F2A00040E05FE387FF04C020E030E040E05FEB38
:10F2B000C701B6010F947F590F94EB5ACB01FF9011
:10F2C000EF90DF90CF900D94E8006DEB77E386E050
:10F2D00095EBD9CF0F94945220E030E0A9010F9420
:10F2E0007F590C9432790F94945220E030E0A901B8
:10F2F0000F947F590F94EB5ACB010D94E8000F94B3
:10F30000945229EC38EC48EC5EE30F94795A20E0F3
:10F3100030E040E05FE30F947F590F94F25A862F5C
:10F320000D943F010D945F350D945F356FEF809123
:10F3300026080D94F0326CE072EB82E00D944644A6
:10F3400061E172EB81E00D94464466E172EB80E08E
:10F350000D94464467EC7FEA83E00D944644CF92D7
:10F36000DF92EF92FF92CF93DF9300D01F92CDB741
:10F37000DEB76B017C0120E030E0A9010F948D52D3
:10F3800087FD1BC06DEB77E386E095E3A70196014F
:10F390000F947F5969837A838B839C83CE01019676
:10F3A0000E94C2FF0F900F900F900F90DF91CF91AE
:10F3B000FF90EF90DF90CF9008956DEB77E386E0BC
:10F3C00095EBE4CF0F94945220E030E040E251E41A
:10F3D0000F94795A20E030E0A9010F947F590C94E2
:10F3E000AF798091171690911816891B8F7011F4C0
:10F3F0000C942E3481E0089580917D02882351F091
:10F40000609195057091960530E020E041E081E043
:10F410000C948728089584E00D94BF3183E00D9407
:10F42000BF3182E00D94BF310F94945220E030E060
:10F43000A9010F947F590F94F25A862F0D941D0144
:10F4400090919C1081E089270C94CA3261E086E299
:10F4500098E00C94E5320F94542A0C9471F280E0F9
:10F4600090E0A0E8B0E48093A5109093A610A0933C
:10F47000A710B093A8108CED92E00E9456F1E09195
:10F48000A00580E090E0A6EEB2E4E43009F44AC0C2
:10F4900080E090E0A0EBB1E480939D1090939E10EB
:10F4A000A0939F10B093A0108093A1109093A210EE
:10F4B000A093A310B093A410EE0FFF0BE454FD4FE4
:10F4C000808191818330910549F184309105D9F192
:10F4D000029761F480E090E0A0E5B3E480939D1092
:10F4E00090939E10A0939F10B093A01084EC92E094
:10F4F0000E9456F11092A5101092A6101092A7101B
:10F500001092A8108CED92E00E9456F18091A00517
:10F510008F5F8530ECF48093A005089580E090E043
:10F52000A0E5B3E480939D1090939E10A0939F104C
:10F53000B093A0108093A1109093A210A093A31059
:10F54000B093A410D3CF80E090E0A0E5B3E4F2CF75
:10F550001092A0050895CF93DF9300D01F92CDB7EE
:10F56000DEB70F94F25A0F94925269837A838B8399
:10F570009C83CE0101960E94A3FE0F900F900F90E6
:10F580000F90DF91CF9108950F9494522AE037EDB8
:10F5900043E25DE30F94795A20E030E0A9010F9433
:10F5A0007F590C94AB7ACF92DF92EF92FF92CF9378
:10F5B000DF9300D01F92CDB7DEB76B017C0120E056
:10F5C00030E0A9010F948D5287FD1BC06DEB77E3EE
:10F5D00086E095E3A70196010F947F5969837A83AA
:10F5E0008B839C83CE0101960E94A3FE0F900F9007
:10F5F0000F900F90DF91CF91FF90EF90DF90CF9021
:10F6000008956DEB77E386E095EBE4CF0F94945289
:10F610002AE037ED43E25DE30F94795A20E030E0D1
:10F62000A9010F947F590C94D37A0F94945220E03F
:10F6300030E0A9010F947F590C94D37ACF92DF92D6
:10F64000EF92FF926B017C0120E030E0A9010F9462
:10F650008D5287FD26C06DEB77E386E095E3A70129
:10F6600096010F947F596B017C0120E030E0A901E5
:10F670000F948D5220E030E040E05FE387FF04C04C
:10F6800020E030E040E05FEBC701B6010F947F5906
:10F690000F94EB5ACB01FF90EF90DF90CF900D9439
:10F6A0003E006DEB77E386E095EBD9CF0F94945253
:10F6B00020E030E0A9010F947F590C941E7B0C943C
:10F6C000B2DC0C94B2DC0C94B2DC0C94B2DC0C9482
:10F6D00064DC0C9464DC0C9464DC0C9464DCCF92E9
:10F6E000DF92EF92FF92CF93C82F0F9453356B01A7
:10F6F0007C0124EA30E74DE75FE3609125027091D9
:10F70000260280912702909128020F948D5287FD46
:10F7100018C08AEF90E0A0E0B0E08C0D9D1DAE1DFA
:10F72000BF1D80933B0590933C05A0933D05B0938E
:10F730003E05C0931E02CF91FF90EF90DF90CF90D7
:10F74000089580E090E0DC01E8CFCF92DF92EF9265
:10F75000FF920F931F930F94533500910C05109156
:10F760000D0520910E0530910F056B017C01C01A2B
:10F77000D10AE20AF30A9701860137FD11C02091F0
:10F780000B05209520930B056A547C4F8F4F9F4F9C
:10F7900060930C0570930D0580930E0590930F05F3
:10F7A00081E090910B05911101C080E01F910F91B4
:10F7B000FF90EF90DF90CF9008950F9492421092B7
:10F7C0004F08109271020E945934882351F08091A1
:10F7D000C11682FD06C085E29EE19093C607809324
:10F7E000C50761E08EE19EE10E94D6350C9456FE7D
:10F7F0004F925F926F927F928F929F92BF92CF9221
:10F80000DF92EF92FF920F931F93CF93DF9300D07D
:10F8100000D01F921F92CDB7DEB77C016A0149016B
:10F82000FB0190818CE0989F800D1124982FF701A7
:10F830002081822F880F820F880F80938A169093E1
:10F840008B164115510571F1FA82E9827C836B8335
:10F85000011121C0AE014B5F5F4FB401C6010E9490
:10F8600091256C016D817E818F819885611571056F
:10F8700081059105B9F00E942427F70180818F5FEF
:10F880008083853138F3CE0101960E94D978E2CF8A
:10F89000B12C860129C08A01B12C26C045284628F2
:10F8A0004728B1F728960FB6F894DEBF0FBECDBF3C
:10F8B000DF91CF911F910F91FF90EF90DF90CF904C
:10F8C000BF909F908F907F906F905F904F90089522
:10F8D000B39407C0B1102EC001151105C9F20F5F16
:10F8E0001F4F01151105A9F2AE014B5F5F4FB40127
:10F8F000C6010E9491256C014D805E806F807884E6
:10F900004114510461047104A9F0F0E24F1651044E
:10F9100061047104F9F2D301C2018D97A109B10903
:10F920000297A105B10530F04BE244165104610481
:10F93000710471F6F7018081482F4B0D5527551F33
:10F940004631510534F0853020F0CE0101960E94F9
:10F95000D97881E0411451046104710409F480E014
:10F96000B80EF70180818B0D8083BB2009F496CF00
:10F97000BA94AE014B5F5F4FB401C8010E9491255C
:10F980008C016D817E818F8198850E942427EDCF27
:10F99000EF92FF920F931F93CF93DF9300D000D08D
:10F9A00000D01F921F92CDB7DEB77C0120912408B2
:10F9B000422F022E000C550B80912508833099F1BF
:10F9C000843051F18EEA91E25F932F939F938F934E
:10F9D0008E010F5F1F4F1F930F930F942452C70187
:10F9E0000E9458DC4FE350E0B80187EC97E00F9499
:10F9F000ED5C0F900F900F900F900F900F902B9643
:10FA00000FB6F894DEBF0FBECDBFDF91CF911F912F
:10FA10000F91FF90EF9008958AEB91E227FDD4CFEC
:10FA200085EA91E2D1CF83EC91E2CECFE09130082C
:10FA300085E1E802F0011124E153FA4E86819781B5
:10FA40000C94C87CE091300886E0E802F0011124B3
:10FA5000E75FF74F808191810C94C87C0F931F93CF
:10FA6000CF93DF938C01EB0190913B1620913C16D4
:10FA7000921305C00F9425020E9473F2F5CF809176
:10FA80003A1634E0839FF0011124E35CF94E1183B0
:10FA90000083D383C2839F5F90933B168F5F2817A9
:10FAA00039F080933A16DF91CF911F910F9108950D
:10FAB00010923A16F8CF63E972E084E690E00E9473
:10FAC0002E7D6AEB72E084E690E00C942E7D81112D
:10FAD0000C945B7D68EB71E084E190E00C942E7DEA
:10FAE0000E94A8D80C94677D0F94ED120C94677D4A
:10FAF0000E9426FC0C945B7DCF93DF93CDB7DEB7DD
:10FB000020E2488559856F818E810F94FC2EDF910C
:10FB1000CF910895282F10922E0880911E08909161
:10FB20001F08A0912008B0912108B7FF08C01092CB
:10FB30001E0810921F081092200810922108809130
:10FB4000A805882331F080911E0880932208109226
:10FB50001D0880911C081816FCF4082E000C990B47
:10FB6000821B910920912208022E000C330B2817CA
:10FB7000390794F097FF02C090E080E0809322085C
:10FB8000092E000CAA0BBB0B80931E0890931F0834
:10FB9000A0932008B0932108809122086623A9F041
:10FBA00090912308891714F4809323082091230847
:10FBB000022E000C330B2C5F3F4F482F082E000CF9
:10FBC000550B241735071CF484508093230808959F
:10FBD000AF92BF92CF92DF92EF92FF920F931F935B
:10FBE000CF93DF9361E081E00E948A7DC09123087A
:10FBF00005E00C0FD1E08EEEE82E81E2F82E12E047
:10FC00001C1B93EEC92E91E2D92EBD2EBC1AAC2E30
:10FC1000A194C11130C0DD23D9F0809122081816BB
:10FC2000BCF040911E0850911F086091200870910F
:10FC300021084F5F5F4F6F4F7F4F40931E085093D7
:10FC40001F0860932008709321088F5F809322081B
:10FC500080917D02882341F030E020E041E067EFB1
:10FC600071E28A2D0E948728CF5F0C13D2CF83E0E8
:10FC700080931C081FC0C13041F59091220891303B
:10FC800069F080917D028823C9F11F92DF92CF92A3
:10FC9000BF9281E0913051F180E028C080911B0833
:10FCA00010921B08882369F3C0934E0880911D08A9
:10FCB000882339F3DF91CF911F910F91FF90EF903F
:10FCC000DF90CF90BF90AF900895C23069F69091C9
:10FCD00022089230A9F080917D02882379F01F924A
:10FCE000FF92EF921F9381E09230B1F68F930E94C2
:10FCF0007C7D0F900F900F900F900F90D0E0B4CFBD
:10FD000080911B0810921B08882329F3C0934E088A
:10FD100080911D088823F9F2CDCF2F923F924F9208
:10FD20005F926F927F928F929F92AF92BF92CF928B
:10FD3000DF92EF92FF920F931F93CF93DF934C01CB
:10FD40000F94DA5101968401080F191FC8010F940E
:10FD5000DA5101966801C80ED91EF8016080C1E031
:10FD6000611001C0C0E0F6013080D1E0311001C067
:10FD7000D0E0AA24A3946110A12C60E085E00E9449
:10FD80008A7D50902308752C9EE0E92EF12C252CBD
:10FD900021948A2D90E001965C01AC0EB11CAD0E51
:10FDA000B11C71101DC080917D028823A1F0E091EB
:10FDB0002402E25067E072E2E33038F4F0E0EE0F44
:10FDC000FF1FEC51FD4F6081718130E020E043E086
:10FDD000822D0E948728D1E0611013C0D2E011C0AB
:10FDE000D2E06110D1E0D7110CC080917D02882350
:10FDF00041F030E020E041E0B4018D2F85190E94F0
:10FE00008728C1E0CD0F472C4518662079F0C7112F
:10FE10000BC080917D02882339F030E020E041E082
:10FE2000B801842D0E948728C2E0CD0F332071F0E5
:10FE3000C7110BC080917D02882339F030E020E0AB
:10FE400041E0B601842D0E948728CF5FF3E0AF1612
:10FE5000B1040CF4CF5FC71162C080917D0288238A
:10FE600009F45AC030E020E042E064E172E2842DFF
:10FE70000E948728D091090593EF9E0D9093080565
:10FE80008EEF8E0D80932F08209187162E151F045C
:10FE900011F00CF041C0209189169217E8F59EE30D
:10FEA00090938A1680938B1665E470E080E090E072
:10FEB0000E94242761E36D0F062E000C770B880B40
:10FEC000990B0E94242760E270E080E090E00E949D
:10FED00024278091D3159091D4150F94E8000E94A7
:10FEE000FF286FE270E080E090E00E9424270E94EB
:10FEF000A57B811109C085E08D9FF0011124EE5B87
:10FF0000F94F8481811108C08091D5159091D61543
:10FF10000F94E8000E94FF2892E090937D02ECE0AD
:10FF2000EE0EF11C7394FAE4EF16F10409F039CFE8
:10FF3000CF5FC0931C08DF91CF911F910F91FF906D
:10FF4000EF90DF90CF90BF90AF909F908F907F9079
:10FF50006F905F904F903F902F9008958FE192E2C5
:10FF60000C948D7E8CE292E20C948D7E8EE492E273
:10FF70000C948D7E89EE92E20C948D7E84EA92E25E
:10FF80000C948D7E81ED92E20C948D7E84E293E25E
:10FF90000C948D7E87E093E20C948D7E87E892E24C
:10FFA0000C948D7E88E692E20C948D7E8F929F92C7
:10FFB000AF92BF92EF92FF920F931F93CF93DF9375
:10FFC000EC018B01E42EF22E80914D1690914E168D
:10FFD0008C179D0709F43EC02091010527FD109262
:10FFE000010522EBC23ED20709F03FC0805F9B4B68
:10FFF00071F40F9453356E517B4F8F4F9F4F609329
:020000021000EC
:100000009105709392058093930590939405D093F6
:100010004E16C0934D1630E020E000931E0810935A
:100020001F082093200830932108E0922308F092C3
:100030001C08C05FDB4B21F410920A05109290055A
:1000400082E080937D0281E080931D081092A505D7
:1000500010929F05DF91CF911F910F91FF90EF902C
:10006000BF90AF909F908F9008952BEBC03FD20729
:1000700071F6825E924B19F0C0EFDBEBC8CF0F94A4
:1000800053358090910590909205A0909305B09083
:100090009405681979098A099B0997FFEDCF80912A
:1000A000C3078770873041F7C5E6D0E8B0CFCF935C
:1000B000DF93EC010E94B27820E040E070E060E065
:1000C000CE01DF91CF910C94D67F20E040E070E02C
:1000D00060E080ED9EEA0E94D67F81E080930A0571
:1000E00010924C0810924B08089520E040E070E018
:1000F00060E08AEA99E70C94D67F80919F0981118C
:1001000014C0809182029091830201972091D315AF
:100110003091D4152817390744F420E040E070E00E
:1001200060E085ED9AEB0C94D67F0C94758021E00D
:1001300020930A05FC0180819181A281B381809383
:10014000250290932602A0932702B093280220E074
:1001500040E070E060E08091190890911A080C94DA
:10016000D67FCF93DF9300D01F92CDB7DEB78DEC53
:100170009CECACECBCE389839A83AB83BC83CE015B
:1001800001960E9497800F900F900F900F90DF9133
:10019000CF910895CF93DF9300D01F92CDB7DEB7F4
:1001A0008DEC9CECACECBDE389839A83AB83BC8380
:1001B000CE0101960E9497800F900F900F900F90A4
:1001C000DF91CF910895CF93DF9300D01F92CDB7E9
:1001D000DEB780E090E0A0E8BFE389839A83AB8339
:1001E000BC83CE0101960E9497800F900F900F90D4
:1001F0000F90DF91CF910895CF93DF9300D01F929E
:10020000CDB7DEB780E090E0A0E2B1E489839A83C5
:10021000AB83BC83CE0101960E9497800F900F9014
:100220000F900F90DF91CF9108958FEF8093260864
:1002300020E040E070E060E08BE596E90C94D67F2A
:1002400081E080930A051092C3071092B10520E067
:1002500040E070E060E087E591E80E94D67F83E6A9
:1002600096E29093C6078093C507089581E0809336
:100270000A058091C3078770873051F01092C30739
:100280001092B10583E696E29093C6078093C50766
:1002900080919C108093A10580E00E94CA3220E0EA
:1002A00040E070E060E088EA92E80C94D67F8091AC
:1002B0007D02882341F030E020E041E062E570E219
:1002C00082E00E9487288091B1058770873041F4D1
:1002D00020E040E070E060E08AE891E80C94D67F8E
:1002E000089520E040E070E060E081EA91E80E943B
:1002F000D67F81E0809302058091A205811107C01D
:1003000087E390E29093C6078093C50708958DE335
:1003100090E2F8CF80917D02882341F030E020E028
:1003200041E063E470E281E00E94872880911B082D
:1003300010921B08882321F01092A2050C94718161
:1003400008950F931F93CF93DF9300D000D000D078
:100350001F92CDB7DEB780917D028823F1F01F9206
:1003600089E18F938091A20590E001969F938F93EE
:100370008FE290E29F938F938E010F5F1F4F1F9329
:100380000F930F942452B80184E290E20E94032953
:100390000FB6F894DEBF0FBECDBF84E080937D0220
:1003A00080910205811108C020E040E070E060E02B
:1003B00087EE91E80E94D67F2A960FB6F894DEBFAA
:1003C0000FBECDBFDF91CF911F910F910895CF92B6
:1003D000DF92EF92FF92CF93DF9300D01F92CDB7C1
:1003E000DEB780911B0810921B08882331F18091A1
:1003F000A2058F5F8093A2058931E0F081E08093B0
:10040000020520E040E070E060E08BE192EB0E94AA
:10041000D67F8EE190E29093C6078093C5070F9038
:100420000F900F900F90DF91CF91FF90EF90DF90A2
:10043000CF9008950E947181F2CF60911E08709153
:100440001F08809120089091210861157105810590
:10045000910509F43EC00F9494522DEC3CEC4CEC09
:100460005CE30F94F3522091A5103091A6104091B7
:10047000A7105091A8100F947F596B017C0120E0C8
:1004800030E040E850EC0F948D5287FD53C020E0DF
:1004900030E040E850E4C701B6010F94DF5B181666
:1004A0000CF44FC0C092A510D092A610E092A710F5
:1004B000F092A8108CED92E00E9456F182E08093B9
:1004C0007D0210921E0810921F08109220081092B0
:1004D000210880917D02882309F4A1CFC090A51046
:1004E000D090A610E090A710F090A81020E030E087
:1004F000A901C701B6010F948D5227E137EB41EDF9
:1005000058E387FF04C027E137EB41ED58EBC70103
:10051000B6010F947F5969837A838B839C836BE246
:10052000CE0101960E9426FFBC0187E190E20E9465
:10053000032975CFC12CD12C90E8E92E90ECF92E2F
:10054000B1CFC12CD12C80E8E82E80E4F82EAACFC0
:1005500080917D02882341F030E020E041E062E5B7
:1005600070E282E00E9487288091B1058770873011
:1005700079F41092A00520E040E070E060E087EAA6
:100580009BEB0E94D67F81E080939F050C942F7A8D
:1005900008952F923F924F925F926F927F928F9227
:1005A0009F92AF92BF92CF92DF92EF92FF920F9302
:1005B0001F93CF93DF9300D000D0CDB7DEB71C01DF
:1005C0007A8369832B833C834D835E8327013801C3
:1005D00081E080931D080E94B27883E080937D02C1
:1005E00030928F0520928E0589819A8190938D0596
:1005F00080938C058B819C81AD81BE818093880521
:1006000090938905A0938A05B0938B054092840549
:10061000509285056092860570928705F12CE12C39
:10062000C0921E08D0921F08E0922008F092210884
:10063000B0924E16A0924D1690928305809282053C
:100640008C8D8093810526960FB6F894DEBF0FBE81
:10065000CDBFDF91CF911F910F91FF90EF90DF9071
:10066000CF90BF90AF909F908F907F906F905F9052
:100670004F903F902F9008952F923F924F925F920C
:100680006F927F928F929F92AF92BF92CF92DF92A2
:10069000EF92FF920F931F93CF93DF9300D000D080
:1006A00000D0CDB7DEB71C017987688769011A834E
:1006B0000983EB82BA01550F880B990B0F94945262
:1006C00020E030E0A9010F947F594B015C0120E04C
:1006D00030E040E05FEC0F94DF5B18162CF0812CCB
:1006E000912CA12C2FECB22EC501B4010F94EB5A22
:1006F0002B013C01B601DD0C880B990B0F94945231
:1007000020E030E0A9010F947F594B015C0120E00B
:1007100030E040E05FE40F948D5287FD05C0812CEE
:10072000912CA12C9FE4B92EE885F9856081718117
:10073000072E000C880B990B0F94945220E030E0A8
:10074000A9010F947F596B017C01C301B2010F9481
:1007500094529B01AC01C701B6010F947E590F94CE
:10076000F25A6C837D838E839F83C501B4010F94FD
:10077000EB5A7B018C01E418F50806091709FB8187
:10078000FF9389809A808AEBA82E8EEAB82ECC80BF
:10079000DD80A301920168857985C1010E94C9822B
:1007A0000F9029960FB6F894DEBF0FBECDBFDF9134
:1007B000CF911F910F91FF90EF90DF90CF90BF905E
:1007C000AF909F908F907F906F905F904F903F90F1
:1007D0002F90089520E040E070E060E080EF9BEB18
:1007E0000C94D67F0E9490340E9431D50C94EA83F9
:1007F00088E598E00E9491CA0E94EA830D94924293
:100800000E94EA838FEA94E29093C6078093C5071B
:1008100008950E94EB310F94974181E08093B716C1
:100820000F94D9410C94EA836F927F928F929F929A
:10083000AF92BF92CF92DF92EF92FF920F931F93EE
:10084000CF93DF9381E080930A0561E00E948A7D67
:10085000C091230885E0882E8C0ED1E009E014E8D1
:1008600095EBE92E94E2F92E82E0982E9C1A20E076
:10087000C22E24E8D22E30ECA32E34E2B32E7D2EED
:100880007C1A6C2E6194C11130C0DD23D9F08091A7
:1008900022081816BCF040911E0850911F08609164
:1008A0002008709121084F5F5F4F6F4F7F4F40933B
:1008B0001E0850931F0860932008709321088F5FD3
:1008C0008093220880917D02882341F030E020E06F
:1008D00041E06DEC74E2862D0E948728CF5F8C1278
:1008E000D2CF83E080931C0823C0C13081F5809172
:1008F0002208813089F080917D02882309F444C068
:10090000DF92CF92BF92AF927F9281E090912208C6
:10091000913089F180E02FC080911B0810921B0854
:10092000882349F30E94008480911D08882319F3CD
:10093000DF91CF911F910F91FF90EF90DF90CF90BB
:10094000BF90AF909F908F907F906F900895C2302E
:1009500029F6809122088230C9F080917D02882397
:1009600099F01F930F93FF92EF929F9281E09091E5
:100970002208923079F68F930E947C7D0F900F9021
:100980000F900F900F900F90D0E0A8CF80911B0890
:1009900010921B08882309F30E94098480911D0886
:1009A0008823D9F2C5CF61116093240240930905D1
:1009B0008C3008F03AC0E82F880FFF0B8827EC51E5
:1009C000FB478F4F0D9476591785F084FB841A8569
:1009D000FE84018504851085078515850A850D85AA
:1009E00082EB9FE721E020930A0520E040E070E0E1
:1009F00060E00C94D67F8AEB9FE7F4CF8EEB9FE705
:100A0000F1CF82EC9FE7EECF86EC9FE7EBCF8AEC4D
:100A10009FE7E8CF8EEC9FE7E5CF82ED9FE7E2CF3F
:100A200010924E0888EE9DE7DDCF0C94EA838EEAA3
:100A30009FE7D8CF86EB9FE7D5CFCF930E9426FCC8
:100A40000E94A8D8C82F882319F080E00F94C60B05
:100A50008C2F0E94677DCF910C94EA830F931F9394
:100A6000CF93DF93CDB7DEB76E970FB6F894DEBFA6
:100A70000FBECDBF282F082E000C330B90911F0204
:100A8000409120028F3F39F0F901EE0FFF1FEF5D1B
:100A9000FD4F908141814F939F933F938F9389E5C1
:100AA0009EE19F938F938E010F5F1F4F1F930F93B4
:100AB0000F9424524FE350E0B80187EC97E00F9475
:100AC000ED5C0E94EA830FB6F894DEBF0FBECDBF87
:100AD0006E960FB6F894DEBF0FBECDBFDF91CF91FB
:100AE0001F910F9108958FEF0C942E8580913008FF
:100AF0000C942E85E0919005EE2389F0E150E0936F
:100B0000900588E0E89FF0011124EF5AFA4F6281C6
:100B1000738127814681808191810C94D67F0C94CA
:100B2000EA832F923F924F925F926F927F928F92C1
:100B30009F92AF92BF92CF92DF92EF92FF920F936C
:100B40001F93CF93DF9300D01F92CDB7DEB761E044
:100B500081E00E948A7D209123082B832C83822FA1
:100B60008B5F898389E0821B8A8388E0782E721AE2
:100B700087E0682E621A86E0582E521A85E0482EC9
:100B8000421A84E0382E321A222E21942B81211110
:100B90005BC080912208882399F180917D0288238F
:100BA00059F081E090912208911180E024E040E02A
:100BB00057E2622D0F94FC2E80918D0980932608B8
:100BC0008B81853009F0A2C01092300880912208F4
:100BD000853009F45FC180917D02882309F43AC20F
:100BE00011E080912208853009F010E080912608FC
:100BF0000F943F0100E09C014DED56E2642D83C04F
:100C000080911B0810921B08882339F20E947A8574
:100C100080911D08882309F4C0CF0F900F900F908A
:100C20000F90DF91CF911F910F91FF90EF90DF9088
:100C3000CF90BF90AF909F908F907F906F905F907C
:100C40004F903F902F9008958B818130C1F5809116
:100C500022088130E1F080917D02882309F4ACCF35
:100C600011E080912208813009F010E08091730238
:100C7000909174020F94E80061E02C81621B00E007
:100C80009C014AEF56E2812F0E94822995CF8091E4
:100C90001B0810921B088823F1F2E12C10E000E001
:100CA00027EE33E04AE050E063E772E08AEF96E235
:100CB0000E943C8380911D08882369F2AECF8B810E
:100CC000823009F08AC180912208823009F44EC036
:100CD00080917D028823D1F011E08091220882303A
:100CE00009F010E06091330670913406809135066A
:100CF000909136060E94EF7862E02C81621B00E042
:100D00009C0144EF56E2812F0E94822980918E0936
:100D1000809326089B81963009F0E6C081E080939D
:100D2000300880912208863009F4C9C080917D0284
:100D3000882391F011E080912208863009F010E0BC
:100D4000809126080F943F0100E09C014DED56E292
:100D5000652D812F0E9482299B819F5F9B83298122
:100D6000291314CF8AE080931C0857CF80911B0869
:100D700010921B08882309F4ABCF20E030E04AE74B
:100D800054E4609133067091340680913506909159
:100D900036060F94F35220E030E0A9010F947F59FA
:100DA00020E030E04AE754E40F947F590F94F25A60
:100DB0001F92912C812C8EE7A82E8EEAB82E6B0103
:100DC00010EDE12E17E0F12E00E010E028E13CEFFD
:100DD0004FEF5FEF63E376E084EF96E20E94C98213
:100DE0000F9080911D08882309F472CF16CF80914F
:100DF00022088330C9F080917D02882309F486CFD0
:100E000011E080912208833009F010E08091D5151F
:100E10009091D6150F94E80063E02C81621B00E0EE
:100E20009C014DEE56E22FCF80911B0810921B08BB
:100E3000882309F30F94712FE12C04E919E72CE2C0
:100E400031E050E040E065ED75E18DEE96E20E9404
:100E50003C8380911D08882371F2DFCE80911B08AE
:100E600010921B08882309F4C4C00F94712FE12C41
:100E700001E516EC2CE830E050E040E061E778E076
:100E800089EE96E20E943C8380911D08882309F434
:100E9000B0C0C3CE80911B0810921B08882309F4B0
:100EA0009ACE0F94712F65E275E78DED96E20F945F
:100EB0007B3180911D08882309F48DCEAECE8091C0
:100EC0001B0810921B08882309F430CF0F94712F50
:100ED00065E275E78DED96E20F947B3180911D08F8
:100EE000882309F423CF99CE2B81273099F580915F
:100EF00022088730B9F080917D02882309F42CCF35
:100F000011E080912208873009F010E080913502CD
:100F1000909136020F94E80000E09C0148ED56E203
:100F2000662D17CF80911B0810921B08882319F398
:100F3000E12C02E015E727EE33E04AE050E065E3FC
:100F400072E088ED96E20E943C8380911D08882320
:100F500091F263CE8B81883009F062C080912208C3
:100F60008830D9F080917D02882309F4F5CE11E014
:100F700080912208883009F010E060918509709115
:100F8000860980918709909188090E94B77300E0D3
:100F90009C014EEC56E2672DDCCE80911B0810922E
:100FA0001B088823F9F265E879E08EEC96E20F944D
:100FB000353180911D088823A9F22FCE80911B081E
:100FC00010921B088823A1F185E690E80E945780C3
:100FD00080911D08882361F120CE8B81833009F434
:100FE00006CF843009F0E8CD80912208843009F4DE
:100FF00035CF80917D02882309F488CE11E080915D
:101000002208843009F010E08091710890917208F4
:101010000F94E80000E09C0149EE56E2632D33CEC8
:101020009B81993009F098CE80912208893031F265
:1010300080917D02882309F48FCE81E0909122086F
:10104000993009F080E023E043EC56E26A810F9486
:10105000FC2E82CE80918E09809326087DCE5F92F1
:101060006F927F928F929F92AF92BF92CF92DF92B8
:10107000EF92FF920F931F93CF93DF93D1E0809174
:10108000D5159091D615892B09F4D0E061E081E067
:101090000E948A7DC09123088C2E45E0942E9C0EE0
:1010A000AA24A39484E0F82EFC1A83E0D82EDC1A3C
:1010B00082E0C82ECC1A7A2C7C1A6C2E619487E0C0
:1010C000B82EBC1AC111B9C080912208882309F436
:1010D00096C080917D02882359F081E0909122088A
:1010E000911180E024E04EEB56E2662D0F94FC2E29
:1010F00080918E0980932608C430E9F4A0923008CC
:1011000080912208843009F448C180917D028823AF
:1011100091F011E080912208843009F010E0809174
:1011200026080F943F0100E09C0147EA56E26F2D2C
:10113000812F0E94822910E000E035E0E32E5C2E32
:10114000581800932608CE111FC0F801EE0FFF1F9C
:10115000E252F04C8591949190933208809331083B
:10116000809122088C1709F42DC180917D0288237B
:1011700059F081E0909122089E1180E023E04DE932
:1011800056E2652D0F94FC2E8E2D0F5F1F4F96E0BB
:10119000E92E8630B1F68091710890917208892B02
:1011A00019F4DD2309F42EC1C73009F58091220816
:1011B000873009F418C180917D028823C1F082EF45
:1011C00093E89F938F9384E996E29F938F93BF92C6
:1011D00081E090912208973009F080E08F930E947F
:1011E0007C7D0F900F900F900F900F900F9088E0E4
:1011F000D1E0CF5FC91166CF80931C080EC08091EB
:101200001B0810921B08882309F463CF0E947A857B
:1012100080911D08882309F45CCFDF91CF911F9145
:101220000F91FF90EF90DF90CF90BF90AF909F9085
:101230008F907F906F905F900895C13009F060C0EB
:1012400080912208813009F43FC080917D0288237B
:1012500009F44ECF11E080912208813009F010E0AE
:101260008091D5159091D6150F94E80000E09C016F
:1012700047EB56E2672D812F0E94822980918D09CC
:1012800080932608C33009F033CF10923008809144
:101290002208833009F46CC080917D02882309F410
:1012A0004ACF11E080912208833009F010E080914C
:1012B00026080F943F0100E09C0147EA56E26D2D9D
:1012C000812F0E94822914CF80911B0810921B0845
:1012D000882309F4BACF0F94712FE12C02E919E7A2
:1012E0002CE231E050E040E065ED75E187EB96E2FD
:1012F0000E943C8380911D08882309F4A6CF8DCFDE
:10130000C23009F0BBCF809122088230B9F08091C1
:101310007D02882309F4ECCE11E08091220882300E
:1013200009F010E080917108909172080F94E80024
:1013300000E09C0143EB56E26C2D9DCF80911B0891
:1013400010921B08882319F30F94712FE12C01E5EB
:1013500016EC2CE830E050E040E061E778E083EB09
:1013600096E20E943C8380911D08882381F255CF2C
:1013700080911B0810921B08882309F48DCF0F94CD
:10138000712F65E275E787EA96E20F947B318091D1
:101390001D08882309F480CF40CF80911B0810924C
:1013A0001B08882309F4B1CE0F94712F65E275E70D
:1013B00087EA96E20F947B3180911D08882309F417
:1013C000A4CE2BCF80911B0810921B08882309F410
:1013D000CCCE84E09AE80E94578080911D08882333
:1013E00009F4C3CE1ACF80911B0810921B088823E2
:1013F00009F4E1CE0E94F28380911D08882309F44C
:10140000DACE0BCF87E0F5CE4F925F926F927F924C
:101410008F929F92AF92BF92CF92DF92EF92FF9204
:101420000F931F93CF93DF930091260861E081E033
:101430000E948A7DC091230810E0000F111F025204
:10144000104C95E0592E5C0E2AE7E22E26E2F22E91
:10145000D3E0DC1B36E9C32E39E7D32E4CE6A42EAD
:1014600046E2B42E82E0782E7C1A5DE9852E56E2A3
:10147000952E81E0682E6C1A4C2E4194C11137C014
:10148000809122088823B1F080917D02882359F051
:1014900081E090912208911180E024E048E856E232
:1014A000642D0F94FC2ECF5F5C12E8CF84E0809314
:1014B0001C080CC080911B0810921B08882321F384
:1014C0000E947A8580911D088823F1F2DF91CF91E7
:1014D0001F910F91FF90EF90DF90CF90BF90AF9052
:1014E0009F908F907F906F905F904F900895C13044
:1014F00059F5F801859194919093320880933108C1
:1015000080912208813081F080917D02882359F2F8
:101510001F929F928F926F9281E09091220891305A
:1015200009F474C080E072C080911B0810921B08FF
:10153000882351F380912608682F0F94F032809110
:101540001D08882309F3C2CFC23009F042C0F80158
:10155000859194919093320880933108809122086C
:101560008230D1F080917D02882309F49CCFDF92F4
:10157000CF92BF92AF927F9281E0909122089230F9
:1015800009F080E08F930E947C7D0F900F900F9068
:101590000F900F900F9087CF80911B0810921B081F
:1015A000882301F30E94967980911D088823D1F247
:1015B0008DCF80911B0810921B088823C1F0609189
:1015C00026088FEF0F94F03280911D08882379F060
:1015D0007DCFC33009F067CFF80185919491909346
:1015E00032088093310880912208833011F3809172
:1015F0007D02882309F457CF1F92FF92EF92DF9369
:1016000081E090912208933009F08CCF8F930E9453
:101610007C7D0F900F900F900F900F9044CF9F9272
:10162000AF92BF92CF92DF92EF92FF920F931F93F0
:10163000CF93DF9361E081E00E948A7DC09123080F
:10164000CC2E85E0982E9C0E94E2A92E96E2B92E1F
:10165000D7E0DC1B16E01C1B05E00C1B84E0F82E19
:10166000FC1A82E0E82EEC1A81E0D82EDC1AC111B7
:1016700033C0809122088823B9F080917D028823AD
:1016800061F06C2D619581E090912208911180E0CC
:1016900024E047E656E20F94FC2ECF5FC911E7CF56
:1016A00088E080931C080CC080911B0810921B08D6
:1016B000882319F30E947A8580911D088823E9F216
:1016C000DF91CF911F910F91FF90EF90DF90CF901E
:1016D000BF90AF909F900895C13011F5809122087E
:1016E000813079F080917D028823B9F281E0909178
:1016F0002208913009F080E023E046EB5FE36D2D96
:10170000CACF80911B0810921B08882359F382E7E7
:101710009CE80E94578080911D08882319F3D0CF40
:10172000C23009F0BFC090912208923071F08091D0
:101730007D02882309F4B1CF81E0923009F080E086
:1017400020E249E556E26E2DA6CF80911B0810924B
:101750001B08882361F323E636E23093C607209303
:10176000C50780911D08882311F3AACF9091220804
:10177000933079F080917D02882309F48ECF63E065
:101780006C1981E0933009F080E020E24DE456E2EC
:1017900082CF80911B0810921B08882359F324E5FF
:1017A00036E23093C6072093C50780911D08882331
:1017B00009F386CF90912208943071F080917D02D8
:1017C000882309F46ACF81E0943009F080E020E2B8
:1017D00041E456E26F2D5FCF80911B0810921B08E9
:1017E000882361F328E436E23093C6072093C507C7
:1017F00080911D08882311F363CF909122089530C2
:1018000071F080917D02882309F447CF81E0953003
:1018100009F080E020E245E356E2602F3CCF809162
:101820001B0810921B08882361F32CE336E23093E7
:10183000C6072093C50780911D08882311F340CF68
:1018400080912208863081F080917D02882309F4FE
:1018500024CF81E090912208963009F080E023E0C7
:1018600048E256E2612F17CF80911B0810921B08A7
:10187000882351F38EE89DE80E94578080911D08CF
:10188000882311F31DCF80911B0810921B08882319
:10189000D9F0B092C607A092C50780911D08882391
:1018A00099F00ECFC33009F461CFC43009F482CF70
:1018B000C53009F4A2CFC63019F2C73009F0EDCE19
:1018C000909122089730F9F280917D02882309F4E3
:1018D000E4CE81E0973009F080E020E243E156E277
:1018E0006D2FD9CEAF92BF92CF92DF92EF92FF923F
:1018F0000F931F93CF93DF9361E081E00E948A7D75
:10190000C091230885E0C82ECC0ED5E0DC1B93E007
:10191000D92E14E01C1BBD2CBC1A82E0F82EFC1A38
:1019200081E0E82EEC1AAC2EA194C1112BC080915D
:101930002208882381F080917D02882369F181E06B
:1019400090912208911180E024E04CE056E26A2D4B
:101950000F94FC2E21C080911B0810921B08882335
:1019600051F30E947A8580911D08882321F3DF912D
:10197000CF911F910F91FF90EF90DF90CF90BF908C
:10198000AF900895C130A1F590912208913059F09F
:1019900080917D02811119C0CF5FCC11C6CF86E046
:1019A00080931C08E4CF80911B0810921B088823A9
:1019B00079F3809137028C2780933702D0927D0291
:1019C00080911D08882321F3D2CF81E0913009F066
:1019D00080E0909137022BEF35E2911102C027EFA2
:1019E00035E201E04EEF55E26E2D0E948229D4CF00
:1019F000C23009F077C080912208823079F080915E
:101A00007D02882349F281E090912208923009F00A
:101A100080E023E047ED5FE36F2D9ACF80911B08B4
:101A200010921B08882359F385EA99E70E94578092
:101A300080911D08882319F39ACF80912208833062
:101A400081F080917D02882309F4A6CF81E09091F6
:101A50002208933009F080E023E040ED5FE36B2D36
:101A600077CF80911B0810921B08882351F380EADE
:101A700099E70E94578080911D08882311F377CF42
:101A800080912208843081F080917D02882309F4BE
:101A900083CF81E090912208943009F080E023E028
:101AA00049EC5FE3612F54CF80911B0810921B0813
:101AB000882351F38BE999E70E94578080911D0894
:101AC000882311F354CF80911B0810921B088823A0
:101AD000A9F08DE790E80E94578080911D08882327
:101AE00069F045CFC33009F4A8CFC43049F2C530FE
:101AF00009F052CF80912208853029F380917D0230
:101B0000882309F449CF81E090912208953009F0AB
:101B100080E023E040EC5FE36D2F1ACF2F923F92DD
:101B20004F925F926F927F928F929F92AF92BF92ED
:101B3000CF92DF92EF92FF920F931F93CF93DF9399
:101B400000D01F921F92CDB7DEB78091C307877078
:101B500089830E94C533682E61E081E00E948A7DFE
:101B6000209123082C83722E2B5F2A8383E0871910
:101B70008B835524539482E0282E2718452C471830
:101B8000372C31948C81811141C0809122088823A7
:101B9000C9F080917D02882359F081E0909122085C
:101BA000911180E024E04AED50E2632D0F94FC2E69
:101BB000662009F452C08981873009F462C193E03C
:101BC0009D834DC080911B0810921B08882309F348
:101BD0000E947A8580911D088823D9F20F900F907A
:101BE0000F900F900F90DF91CF911F910F91FF9069
:101BF000EF90DF90CF90BF90AF909F908F907F90AD
:101C00006F905F904F903F902F9008959C819130FE
